:100000000C940A300C940F330C943A330C946533EF
:100010000C9490330C94BB330C94E6330C94113451
:100020000C943C340C943B300C943B300C943B309F
:100030000C943B300C943B300C943B300C943B3094
:100040000C943B300C94EACE0C943B300C943B3037
:100050000C943B300C943B300C94A1BF0C943D307D
:100060000C943B300C9469AA0C9415AB0C943B3067
:100070000C943B300C943B300C943B300C943B3054
:100080000C943B300C943B300C943B300C943B3044
:100090000C943B300C943B300C943B300C943B3034
:1000A0000C943B300C943B300C943B300C943B3024
:1000B0000C943B300C943B300C943B300C943B3014
:1000C0000C943B300C943B300C943B300C943B3004
:1000D0000C943B300C943B300C943B300C943B30F4
:1000E0000C943B3085318A318F319931A3311C32E8
:1000F000AD31B531BD31C731D131DB31EA31F43108
:100100001C32FE3108321232403243323232363241
:100110003C327A3247324B325132553259325F32A9
:10012000633267327A326D327132753255683568B2
:100130003B6838683E684168446850684768626850
:100140004A684D68AFA7ADA7D1A7CEA7CCA703A893
:1001500000A8FEA75CA82AA827A825A89CAAA2AA4E
:10016000B3AABEAAC6AADBAACAAADBAACEAAD2AAE8
:10017000DBAAD8AA084AD73B3BCE016E84BCBFFDA0
:10018000C12F3D6C74319ABD56833DDA3D00C77F67
:1001900011BED9E4BB4C3E916BAAAABE0000008000
:1001A0003F05A84CCDB2D44EB93836A9020C50B98F
:1001B000918688083CA6AAAA2ABE000000803F00BB
:1001C0000D94B6550D94B4470D948D0B0D94815A32
:1001D0004E414E494E495459494E46CDCCCC3D0A2C
:1001E000D7233C17B7D13877CC2B329595E6241F0F
:1001F000B14F0A000020410000C84200401C4620C8
:10020000BCBE4CCA1B0E5AAEC59D7400407A10F39A
:100210005A00A0724E18090010A5D4E80000E87634
:1002200048170000E40B54020000CA9A3B0000008B
:10023000E1F505000080969800000040420F0000A4
:1002400000A08601000000102700000000E8030065
:100250000000006400000000000A0000000000012F
:1002600000000000002C76D888DC674F0823DFC12F
:10027000DFAE59E1B1B796E5E3E453C63AE65199EA
:100280007696E8E6C28426EB898C9B62ED407C6F13
:10029000FCEFBC9C9F40F2BAA56FA5F490055A2ACA
:1002A000F75C936B6CF9676DC11BFCE0E40D47FED6
:1002B000F520E6B500D0ED902E03009435770500CB
:1002C00080841E080000204E0A000000C80C333352
:1002D00033330F986E12831141EF8D2114893BE661
:1002E0005516CFFEE6DB18D1844B381BF77C1D90EA
:1002F0001DA4BBE424203284725E228100C9F12453
:10030000ECA1E53D2700000A0B02090C0D0E0807C1
:1003100003040100000000000000000000000000D5
:1003200000000000000000000000000000000000CD
:10033000001211100000000000000000000000008A
:10034000000000000000000000000001021020205A
:100350000808102040102040800201020108040219
:10036000010102040810204080804020100804028F
:1003700001800402018040201008040201080402E8
:1003800001010204081020408001020408102040EE
:100390008005050505070508080808020202020A8B
:1003A0000A08080404040401010101010101010318
:1003B00003030303030303040707070C0C0C0C0CD3
:1003C0000C0C0C0202020206060606060606060BC6
:1003D0000B0B0B0B0B0B0B0000200023002600293E
:1003E000002C002F0032000001000003010601096B
:1003F0000100002200250028002B002E00310034CF
:100400000002010000050108010B01000021002489
:100410000027002A002D00300033000101000004F5
:100420000107010A0101060D00FE09016602D6203E
:10043000FFFE0BFE0AFE0D0060221969808080809D
:100440008080800080183363A0A0A00357675050BD
:10045000F850F850500259692078A0A0702828F070
:100460002002596948A85010204050A890025868AE
:1004700040A0A040A0989068281363808080113B22
:100480006B2040408080808080404020113B6B800A
:100490004040202020202040408006556520A87044
:1004A000A8200455652020F8202011336360408087
:1004B000065161F811336340E040025969080810A1
:1004C00010204040808002596920508888888888A0
:1004D00050200259692060A02020202020F80259D5
:1004E000697088880810204080F8025969F808105F
:1004F000207008088870025969101030505090F828
:100500001010025969F88080B0C808088870025934
:100510006970888080F088888870025969F80810AE
:10052000102020404040025969708888887088886F
:10053000887002596970888888780808887011382E
:100540006840E040000040E04011386840E0400072
:100550000060408002596908102040804020100847
:10056000045464F80000F802596980402010081013
:1005700020408002596970888808102020002002DD
:10058000596970888898A8A8B08078025969205065
:10059000888888F8888888025969F04848487048EF
:1005A0004848F00259697088808080808088700295
:1005B0005969F048484848484848F0025969F88065
:1005C0008080F0808080F8025969F8808080F08017
:1005D0008080800259697088808080988888700245
:1005E000596988888888F888888888123969E0403D
:1005F000404040404040E00259693810101010104F
:10060000109060025969888890A0C0A090888802E4
:1006100059698080808080808080F802596988884C
:10062000D8A8A88888888802596988C8C8A8A898BE
:1006300098888802596970888888888888887002B4
:100640005969F0888888F080808080015A6A7088B3
:100650008888888888A87008025969F0888888F096
:10066000A090888802596970888080700808887016
:10067000025969F820202020202020200259698872
:10068000888888888888887002596988888888500E
:100690005050202002596988888888A8A8A8A850A6
:1006A00002596988885050205050888802596988BA
:1006B0008850502020202020025969F8081010206E
:1006C000404080F8113B6BE080808080808080809B
:1006D00080E0025969808040402010100808113BDA
:1006E0006BE0202020202020202020E008536320E1
:1006F0005088015161F82A226280400256667008D3
:1007000078889868025969808080F088888888F0A5
:1007100002566670888080887002596908080878D7
:1007200088888888780256667088F88088700259B0
:100730006930484040F04040404000586870888828
:100740008878088870025969808080B0C888888855
:10075000881238684000C040404040E0004A6A10BB
:1007600000301010101090906002596980808090C5
:10077000A0C0A09088123969C0404040404040402D
:10078000E0025666D0A8A8A8A888025666B0C88815
:10079000888888025666708888888870005868F053
:1007A000888888F0808080005868788888887808F1
:1007B0000808025666B0C88080808002566670883D
:1007C000601088700258684040F040404048300255
:1007D0005666888888889868025666888888505047
:1007E000200256668888A8A8A8500256668850201D
:1007F0002050880058688888889868088870025651
:1008000066F810204080F8015B6B1820202020C083
:10081000202020201822196980808080808080809C
:1008200080015B6BC0202020201820202020C008E1
:10083000536348A890FFFFFFFFFFFFFFFFFFFFFF8D
:10084000FFFFFFFFFFFFFFFFFFFFFFFFFFFFFFFFB8
:10085000FFFFFFFFFFFF0D0060221969800080800D
:1008600080808080800358682070A8A0A0A8702095
:1008700002596930484040E0404048B0035666881D
:10088000705050708802596988885050F820F820BC
:1008900020221969808080800080808080124A6ACE
:1008A000609080609090601090601A3262A0A00307
:1008B00059697088A8D8C8D8A88870045767700884
:1008C00078887800F80356662850A0A05028045372
:1008D00063F80808163161E00359697088E8D8D8D0
:1008E000E8D888700A5161F81744646090906003FA
:1008F00057672020F8202000F807356540A02040E9
:10090000E007356540A04020C02A226240800058A0
:10091000688888888898E8808002596978E8E8E8DB
:10092000E868282828262161C020226240800735F7
:100930006540C04040E0045767708888887000F8C0
:10094000035666A050282850A0025A6A40C0404072
:10095000E00818283808025A6A40C04040E01028D1
:10096000081038025A6A40A04020A04818283808C9
:10097000025969200020204080888870025A6A400D
:10098000200020508888F88888025A6A10200020A9
:10099000508888F88888025A6A3048002050888831
:1009A000F88888025A6A28500020508888F8888879
:1009B000025A6A50500020508888F88888025A6A83
:1009C00020502020508888F8888802596958A0A0B3
:1009D000A0B0E0A0A0B8005B6B70888080808080B1
:1009E00088702040025A6A402000F88080F08080A1
:1009F000F8025A6A102000F88080F08080F8025ACD
:100A00006A304800F88080F08080F8025A6A5050BE
:100A100000F88080F08080F8123A6A804000E04060
:100A200040404040E0123A6A204000E040404040F0
:100A300040E0124A6A609000E04040404040E012CE
:100A40003A6AA0A000E04040404040E0025969F00E
:100A5000484848E8484848F0025A6A2850008888C0
:100A6000C8A8988888025A6A4020007088888888B8
:100A70008870025A6A1020007088888888887002FE
:100A80005A6A30480070888888888870025A6A28B4
:100A9000500070888888888870025A6A50500070A8
:100AA0008888888888700355658850205088015B45
:100AB0006B08709898A8A8A8C8C87080025A6A40A5
:100AC000200088888888888870025A6A10200088E8
:100AD000888888888870025A6A30480088888888A0
:100AE000888870025A6A5050008888888888887080
:100AF000025A6A102000888850202020200259695C
:100B000080F0888888F0808080025969609090A089
:100B1000A0908888B00259694020007008788898B1
:100B2000680259691020007008788898680259692D
:100B30003048007008788898680259692850007019
:100B40000878889868025969505000700878889829
:100B500068025A6A304830007008788898680256EF
:100B600066702870A0A850005868708880808870CF
:100B700020400259694020007088F880887002592E
:100B8000691020007088F880887002596930480028
:100B90007088F88088700259695050007088F88019
:100BA0008870123969804000C040404040E01239EE
:100BB00069204000C040404040E012496960900018
:100BC000C040404040E0123969A0A000C040404011
:100BD00040E0025A6A50206010708888888870024D
:100BE0005969285000B0C88888888802596940200F
:100BF0000070888888887002596910200070888881
:100C00008888700259693048007088888888700226
:100C10005969285000708888888870025969505036
:100C200000708888888870035767202000F80020AB
:100C300020015868087098A8A8C8708002596940B7
:100C40002000888888889868025969102000888860
:100C50008888986802596930480088888888986828
:100C6000025969505000888888889868005B6B102A
:100C700020008888889868088870005A6A8080B048
:100C8000C88888C8B08080005B6B50500088888816
:100C9000986808887001050700FE0500FB01F22036
:100CA000FFFE05FE05FE0200400215258080800043
:100CB00080053242A0A002556550F850F850014618
:100CC000562070C030E02002556590102040480248
:100CD0005565608068906805122280800225354045
:100CE000808080400225358040404080043343A00E
:100CF00040A003334340E0400122324080043141B0
:100D0000E0021121800255650810204080024555FF
:100D10006090909060022535C040404040024555AB
:100D2000E0106080F0024555E0106010E00245558B
:100D30002060A0F020024555F080E010E00245550B
:100D40006080E09060024555F0102040400245551B
:100D500060906090600245556090701060031323AE
:100D6000800080021424800080800235452040806D
:100D70004020033343E000E00235458040204080BE
:100D8000024555E0106000400255657088B8A870B3
:100D9000024555609090F090024555E090E090E05B
:100DA0000235456080808060024555E0909090E07B
:100DB000023545E080E080E0023545E080E080805B
:100DC0000245557080B090700245559090F090901B
:100DD000023545E0404040E002455530101090603B
:100DE00002455590A0C0A09002354580808080E0EB
:100DF00002556588D8A8888802455590D0B0909053
:100E00000245556090909060024555E09090E080DA
:100E1000014656609090906010024555E09090E039
:100E20009002455570806010E0023545E04040403A
:100E30004002455590909090600245559090A0A03A
:100E40004002556588A8A8A850024555909060902A
:100E5000900245559090701060023545E02040802A
:100E6000E0022535C0808080C0025565804020109A
:100E700008022535C0404040C005324240A0024132
:100E800051F0052232804002445470909070024527
:100E90005580E09090E002344460808060024555C7
:100EA000107090907002445460B0C06002354520CC
:100EB00040E04040004656709090701060024555EA
:100EC00080E0909090021525800080808000273778
:100ED000400040404040800245558090A0E0900294
:100EE00015258080808080025464F0A8A8A8024460
:100EF00054E090909002445460909060004656E018
:100F00009090E080800046567090907010100234EF
:100F100044A0C0808002445470C030E00235454097
:100F2000E0404020024454909090700244549090CD
:100F3000A040025464A8A85050023444A04040A0ED
:100F4000004656909090701060024454F02040F09B
:100F50000235456040804060021525808080808099
:100F6000023545C0402040C005425250A0FFFFFF5F
:100F7000FFFFFFFFFFFFFFFFFFFFFFFFFFFFFFFF81
:100F8000FFFFFFFFFFFFFFFFFFFFFFFFFFFF02006D
:100F900040FFFFFFFFFFFFFFFFFFFFFFFFFFFFFF20
:100FA000FFFFFFFFFFFFFFFFFFFFFFFFFFFFFFFF51
:100FB000FFFFFFFFFFFFFFFFFFFFFFFFFFFFFFFF41
:100FC000FFFFFFFFFFFFFFFFFFFFFFFFFFFFFFFF31
:100FD000FFFFFFFFFFFFFFFFFFFFFFFFFFFFFFFF21
:100FE000FFFFFFFFFFFFFFFFFFFFFFFFFFFFFFFF11
:100FF00001050800FF060121023520FFFF07FF065B
:10100000FF090050221656808080800080153353DF
:10101000A0A0A00257575050F850F8505002575710
:101020002070A07028702013355580A040A02002A9
:10103000475740A0A040A0A05025135380808012A5
:101040002656408080808040122656804040404096
:10105000800245559060F060900255552020F820A0
:1010600020113353604080044151F011335340E06C
:101070004002465610102040808012365640A0A0F4
:10108000A0A04012365640C0404040E002465660A4
:1010900090106080F0024656F0206010906002468A
:1010A000562060A0F02020024656F080E0109060AC
:1010B0000246566080E0909060024656F010202074
:1010C00040400246566090609090600246566090A4
:1010D00090701060122555C0C000C0C01136566017
:1010E00060006040801236562040808040200343DC
:1010F00053F000F0123656804020204080123656C1
:1011000040A020400040015858304898A8A890407E
:1011100030024656609090F09090024656E090E083
:101120009090E0024656609080809060024656E0C3
:1011300090909090E0024656F080E08080F0024669
:1011400056F080E0808080024656609080B09060CB
:101150000246569090F0909090123656E0404040F3
:1011600040E002465670202020A04002465690A043
:10117000C0A0A0900246568080808080F002465633
:1011800090F0F090909002465690D0F0B0B090025F
:101190004656609090909060024656E09090E080B5
:1011A00080014757609090D0B06010024656E090A2
:1011B00090E0909002465660904020906012365623
:1011C000E04040404040024656909090909060022F
:1011D0004656909090906060024656909090F0F045
:1011E00090024656909060609090025656888850C3
:1011F000202020024656F010204080F0123656E0A3
:1012000080808080E0024656808040201010123698
:1012100056E020202020E016325240A0014151F03B
:1012200016225280400244547090907002465680BC
:1012300080E09090E0123454608080600246561046
:10124000107090907002445460B0C0600246562006
:101250005040E04040014555609070106002465695
:101260008080E09090901236564000C04040E011DF
:1012700037572000202020A040024656808090E072
:101280009090123656C040404040E0025454D0A8DE
:10129000A8A8024454E0909090024454609090605A
:1012A000014555E090E08080014555709070101028
:1012B000024454A0D0808012345460C020C0024642
:1012C000564040E0405020024454909090701234B8
:1012D00054A0A0A04002545488A8A850024454909E
:1012E0006060900145559090709060024454F020E9
:1012F00040F0024757304020C02040302216568030
:101300008080808080024757C02040304020C00647
:10131000425250A0FFFFFFFFFFFFFFFFFFFFFFFF55
:10132000FFFFFFFFFFFFFFFFFFFFFFFFFFFFFFFFCD
:10133000FFFFFFFFFF0900502216568000808080CB
:10134000800146562070A0A070200246562050E032
:101350004050A002555588705070880256568850EB
:10136000F820F82022175780808000808080024774
:10137000577080E0907010E0173151A002565670FF
:10138000A8C8C8A87014355560A06000E003435396
:1013900050A050123353E02020143151E002565631
:1013A00070E8D8E8D870173151E015335340A040A9
:1013B00012355540E04000E014355540A02040E093
:1013C000143555C020C020C016225240800145551A
:1013D000909090E08002565678E8E868282824111A
:1013E0005180112252408014355540C04040E014D5
:1013F000355540A04000E0034353A050A00247579A
:10140000808080A060F0200247578080A0D010200C
:101410007002475780408060A0F02012365640008E
:101420004080A04002475740206090F090900247D3
:101430005720406090F0909002475760906090F085
:10144000909002475750A06090F0909002475790BC
:10145000006090F0909002475760906090F09090FC
:1014600002465670A0A0F0A0B0014757609080805F
:101470009060400247574020F080E080F0024757DC
:101480002040F080E080F00247576090F080E080DC
:10149000F00247579000F080E080F012375780400C
:1014A000E0404040E01237572040E0404040E0122A
:1014B000375740A0E0404040E0123757A000E040DE
:1014C0004040E00256567048E8484870024757507E
:1014D000A090D0B0909002475740206090909060CC
:1014E000024757204060909090600247576090609C
:1014F0009090906002475750A06090909060024793
:101500005790006090909060123353A040A0024624
:101510005670B0B0D0D0E0024757402090909090E5
:10152000600247572040909090906002475760902B
:101530009090909060024757900090909090600239
:1015400057571020885020202002465680E0909067
:10155000E0800246566090A0A090A002475740202D
:101560000070909070024757204000709090700279
:1015700047572050007090907002475750A000705D
:1015800090907002465650007090907002475760DD
:10159000906070909070025454F068B07811355596
:1015A000608080604002475740200060B0C0600209
:1015B000475720400060B0C060024757609000600D
:1015C000B0C060024656500060B0C060123757800D
:1015D0004000C04040E0123757204000C04040E08B
:1015E00012375740A000C04040E0123656A000C05D
:1015F0004040E0024757A040A0107090600247575B
:1016000050A000E0909090024757402000609090DA
:1016100060024757204000609090600247576090FA
:10162000006090906002475750A000609090600268
:1016300046569000609090601235554000E00040A2
:1016400002445470B0D0E002475740200090909080
:10165000700247572040009090907002475760906A
:1016600000909090700246569000909090700148C3
:101670005820400090907090600147578080E09023
:10168000E080800147579000909070906025753AF7
:101690002530327500253032753A253032750020FC
:1016A0002020200025202000252000253164002551
:1016B0003264002533640025346400253564002538
:1016C0003664000000007E006000600060F87ECCA0
:1016D00060CC60CC60F860CC00CC00CC00CC0000CA
:1016E0000000000000FE7F0E702664724E7A5E32AB
:1016F0004C8241324C7A5E724E26640E70FE7F0040
:101700000000000000FE7F0E70C663C24382411AD3
:1017100058BA5D1A588241C243C6630E70FE7F00FC
:1017200000000000008808880810112022202210E4
:101730001188088808101100000000000000000057
:1017400000000000002022101188088808101120D5
:101750002220221011880800000000000000000074
:101760000000000000000000000000000000000079
:10177000000000000000000000FE7FFE7F06600009
:1017800000000000000000F00FF81FF81FF81FF025
:101790000FF00FF81FF81FF81FE007C003800100CB
:1017A000000000304848304572723A20757466383F
:1017B00020666F6E74206E6F7420696E6974696143
:1017C0006C697A65642E004572723A2075746638C9
:1017D00020666F6E74206E6F7420696E6974696123
:1017E0006C697A65642E004572723A2075746638A9
:1017F00020666F6E74206E6F7420696E6974696103
:101800006C697A65642E00506C6561736520526561
:10181000736574005052494E5445522048414C540F
:10182000454400687474703A2F2F6D61726C696E54
:1018300066772E6F726700322E302E302E313731A0
:10184000007F80FFC0FFC0FFC07F807F80FFC0FFA0
:10185000C0FFC03F001E000C00FFFFFF0E000E0087
:101860000E000E000E000E000E000E007FC03F8026
:101870001F000E00040004000E001F003F807FC008
:101880000E000E000E000E000E000E000E000E00E8
:1018900000FE0003FF800783C00E01C00E00E01CA5
:1018A00000E07F00E03E00E01C00E00800E00000F7
:1018B000E00001C00E01C00F078007FF0001FC001F
:1018C00001FC0007FF000F07800E01C00001C000EF
:1018D00000E00800E01C00E03E00E07F00E01C00AB
:1018E000E00E00E00E01C00783C003FF8000FE0091
:1018F000000C0D00FE07022603BC017FFE08FE0857
:10190000FE05080806000040F0C888889878100591
:101910000808060000C0F88888888888F80505054A
:101920000600012030F8302005080806000020706D
:10193000F820202020E00509090600FF2070A8A853
:10194000B888887020050606060001E08CEA8C8ABB
:101950000A0509090600FFF8A88888888888A8F879
:10196000050A0A0600FE205050505088A8A888702A
:1019700003030306000340A040FFFFFFFFFFFFFF3C
:10198000FFFFFFFFFFFFFFFFFFFFFFFFFFFFFF0066
:1019900000000605FF0107070602008080808080A6
:1019A0000080030303060105A0A0A00506060600AB
:1019B0000050F85050F8500509090600FF2070A8A3
:1019C000A07028A87020050707060000C8C81020CE
:1019D00040989805070706000040A0A040A890681E
:1019E0000103030602058080800309090601FF2028
:1019F00040408080804040200309090601FF80406C
:101A00004020202040408005070706000020A870E5
:101A10002070A8200505050600012020F8202002DE
:101A200003030601FFC04080050101060003F80220
:101A30000202060100C0C0050707060000081010DA
:101A400020404080050707060000708898A8C888D5
:101A50007003070706010040C040404040E0050712
:101A600007060000708808102040F80507070600E8
:101A700000F80810300888700507070600001030CD
:101A80005090F81010050707060000F880F00808CD
:101A90008870050707060000304080F088887005D0
:101AA0000707060000F80810102020200507070689
:101AB000000070888870888870050707060000702D
:101AC000888878081060020505060100C0C000C0C3
:101AD000C00206060601FFC0C000C0408003050525
:101AE0000601012040804020050303060002F800A3
:101AF000F803050506010180402040800507070620
:101B000000007088102020002005070706000070E4
:101B100088B8A8B88070050707060000708888F8A4
:101B2000888888050707060000F04848704848F094
:101B30000507070600007088808080887005070709
:101B4000060000F04848484848F00507070600002E
:101B5000F88080F08080F8050707060000F8808094
:101B6000F0808080050707060000708880809888D4
:101B700070050707060000888888F88888880307AA
:101B800007060100E04040404040E005070706002E
:101B900000381010101090600507070600008890AC
:101BA000A0C0A09088050707060000808080808084
:101BB00080F805070706000088D8A8888888880567
:101BC00007070600008888C8A898888805070706C0
:101BD000000070888888888870050707060000F074
:101BE0008888F08080800507070600007088888854
:101BF000A89068050707060000F08888F0A0908884
:101C000005070706000070888070088870050707C0
:101C1000060000F8202020202020050707060000ED
:101C20008888888888887005070706000088888863
:101C30008850502005070706000088888888A8A8D3
:101C4000500507070600008888502050888805073F
:101C5000070600008888502020202005070706007E
:101C600000F80810204080F80309090601FFE08011
:101C7000808080808080E00507070600008040406B
:101C8000201010080309090601FFE0202020202071
:101C90002020E00503030600052050880501010609
:101CA00000FEF80303030601058040200505050634
:101CB000000070087888780507070600008080F02B
:101CC000888888F00505050600007080808870050A
:101CD0000707060000080878888888780505050643
:101CE00000007088F080700507070600003048404B
:101CF000E04040400507070600FE708888887808A5
:101D0000700507070600008080F088888888030730
:101D1000070601004000C0404040E00409090601F8
:101D2000FE1000301010101090600507070600002C
:101D300080808890E09088030707060100C040403B
:101D4000404040E0050505060000D0A8A8A8A80569
:101D50000505060000B0C88888880505050600004E
:101D600070888888700507070600FEF0888888F06C
:101D700080800507070600FE7888888878080805AF
:101D80000505060000B0C880808005050506000036
:101D900078807008F00507070600002020F8202052
:101DA000201805050506000088888898680505053F
:101DB00006000088888850200505050600008888F0
:101DC000A8A8500505050600008850205088050782
:101DD000070600FE8888885020408005050506001B
:101DE00000F8102040F80309090601FF2040404098
:101DF00080404040200109090602FF8080808080E9
:101E0000808080800309090601FF80404040204017
:101E100040408005030306000248A890FF1FFFFF13
:101E2000FFFFFFFF600000000001FF400000000016
:101E300000FF8000000000007F83CF00000C303FD7
:101E400087FF80000C301F867980000C000F8C30DB
:101E5000C7838C30E78C30CFC7CC31F38C30DCECCF
:101E6000EC33B98C30D86C6C33198C30D06C0C33AB
:101E7000198C30D86C0C33198C30DC6C0E3B198CFF
:101E800030CF7C079F198C30C77C038F194000002E
:101E900000000002600000000000061FFFFFFFFFBF
:101EA000FFF800060900FE06018902FE20FFFE077A
:101EB000FE06FE000000060007010606060200807E
:101EC0008080800080030303060103A0A0A0050713
:101ED000070600FF5050F850F85050050909060059
:101EE000FE2070A8A07028A870200608080600FF31
:101EF00040A84810204854080507070600FF6090D6
:101F000090609890680103030602038080800207B6
:101F1000070602FF4080808080804002070706029B
:101F2000FF80404040404080050505060000885085
:101F3000F850880505050600002020F8202002043E
:101F4000040602FEC0404080050101060002F802BE
:101F50000202060200C0C00406060601001010209E
:101F60004080800406060601006090909090600317
:101F7000060606010040C0404040E0040606060197
:101F8000006090102040F0040606060100F020607A
:101F90001010E005060606000010305090F81004FE
:101FA0000606060100F080E01010E00406060601B7
:101FB000006080E0909060040606060100F01010BA
:101FC0002040400406060601006090609090600486
:101FD000060606010060909070106002050506027A
:101FE00000C0C000C0C00207070602FEC0C000C09B
:101FF0004040800505050600001860806018050354
:1020000003060001F800F8050505060000C03008C9
:1020100030C00407070601006090106040004005D2
:1020200006060600007090A8B0807005060606003F
:1020300000205088F88888050606060000F088F021
:102040008888F00406060601006090808090600495
:102050000606060100E090909090E0040606060156
:1020600000F080E08080F0040606060100F080E0C9
:10207000808080040606060100609080B0906004B5
:1020800006060601009090F0909090030606060167
:1020900000E040404040E005060606000038101011
:1020A00010906004060606010090A0C0A090900465
:1020B00006060601008080808080F0050606060086
:1020C0000088D8A8A8888804060606010090D0B029
:1020D0009090900506060600007088888888700435
:1020E0000606060100E09090E080800407070601E4
:1020F000FF609090D0B06010040606060100E090EA
:1021000090E09090040606060100609040209060E8
:10211000050606060000F8202020202004060606FA
:102120000100909090909060040606060100909047
:1021300090F060600506060600008888A8A8D88888
:102140000506060600008850202050880506060671
:102150000000888850202020040606060100F010A8
:10216000204080F0030606060100E080808080E0C9
:1021700004060606010080804020101003060606B3
:102180000100E020202020E005030306000320508A
:10219000880501010600FEF80202020602048040E2
:1021A0000404040601007090907004060606010005
:1021B0008080E09090E0040404060100708080704C
:1021C00004060606010010107090907004040406C6
:1021D000010060B0C070040606060100205040E017
:1021E00040400406060601FE6090907010600406F0
:1021F000060601008080E09090900306060601002C
:102200004000C04040E00308080601FE20006020B6
:102210002020A0400406060601008080A0C0A090F7
:10222000030606060100C040404040E005040406E5
:102230000000D0A8A888040404060100E090909053
:10224000040404060100609090600406060601FE86
:10225000E09090E080800406060601FE7090907089
:102260001010040404060100A0D0808004040406B9
:10227000010070C030E00406060601004040E04066
:102280005020040404060100909090700404040699
:1022900001009090606005040406000088A8A85022
:1022A000040404060100906060900406060601FE26
:1022B000909090709060040404060100F02040F0BB
:1022C0000307070601002040408040402001070727
:1022D0000602FF808080808080800307070601005F
:1022E0008040402040408004020206010350A0FFCD
:1022F000FFFFFFFFFFFFFFFFFFFFFFFFFFFFFFFFEE
:10230000FFFFFFFFFFFFFFFFFFFFFFFFFFFFFFFFDD
:10231000000000060007010606060200800080801B
:1023200080800406060601FF2070A0A0702005072B
:10233000070600FF304840F04040F805050506005C
:1023400000A8508850A80506060600008850F8200E
:10235000F8200107070602FF80808000808080044B
:1023600007070601FF708060906010E0030101061E
:102370000105A0060707060000788494A4948478D9
:1023800003050506010160A06000E00505050600E3
:10239000002850A05028040303060100F010100488
:1023A0000101060102F00607070600007884B4A4C4
:1023B000A48478040101060105F004030306010268
:1023C0006090600507070600FF2020F8202000F835
:1023D00003050506010140A02040E00305050601B4
:1023E00001C0204020C00202020602044080040511
:1023F000050601FF9090B0D0800506060600007823
:10240000E8E86828280101010602028002020206AB
:1024100002FE408003050506010140C04040E00384
:10242000050506010140A04000E005050506000085
:10243000A0502850A00508080600FF40C04050707A
:102440003078100508080600FF40C04050680810AA
:10245000380508080600FFC0204030F0307810042E
:10246000070706010020002060809060050707062E
:1024700000004020205070888805070706000010E3
:102480002020507088880507070600002050205043
:10249000708888050707060000285020507088883B
:1024A00005070706000050002050708888050707C0
:1024B000060000205020507088880506060600009F
:1024C00078A0F0A0A0B80408080601FE6090808003
:1024D000906020400407070601004020F080E08063
:1024E000F00407070601002040F080E080F00407B8
:1024F000070601002050F080E080F0040707060185
:10250000005000F080E080F00307070601008040E3
:10251000E0404040E00307070601002040E0404063
:1025200040E003070706010040A0E0404040E00310
:102530000707060100A000E0404040E0050606064F
:1025400000007048E848487004070706010050A0E2
:1025500090D0B09090040707060100402060909052
:10256000906004070706010020406090909060048E
:10257000070706010020506090909060040707064E
:10258000010050A060909090600407070601005081
:10259000006090909060050505060000885020506E
:1025A000880408080601FF1070B0B0D0D0E08004A5
:1025B00007070601004020909090906004070706EE
:1025C00001002040909090906004070706010020D1
:1025D0005090909090600407070601005000909082
:1025E00090906005070706000010208850202020EA
:1025F00004060606010080E09090E08004060606CE
:1026000001006090A0A090A00407070601004020F0
:102610000070909070040707060100204000709041
:10262000907004070706010020500070909070041D
:10263000070706010050A00070909070040606067F
:1026400001005000709090700407070601002050B0
:10265000207090907005040406000070A8B0780403
:1026600006060601FE708080702040040707060100
:102670000040200060B0C070040707060100204041
:102680000060B0C07004070706010020500060B071
:10269000C070040606060100500060B0C070030759
:1026A00007060100804000C04040E0030707060124
:1026B00000204000C04040E003070706010040A0A2
:1026C00000C04040E0030606060100A000C04040F4
:1026D000E004070706010030601070909060040766
:1026E0000706010050A000E0909090040707060143
:1026F0000040200060909060040707060100204021
:102700000060909060040707060100205000609070
:10271000906004070706010050A0006090906004DC
:102720000606060100500060909060050505060051
:10273000002000F8002004040406010070B0D0E07E
:1027400004070706010040200090909070040707DE
:1027500006010020400090909070040707060100D9
:1027600020500090909070040606060100500090E2
:102770009090700409090601FE204000909090702E
:1027800090600408080601FE8080E09090E0808060
:102790000408080601FE5000909090709060536EFF
:1027A000346B3300496E76616465727300427269FE
:1027B000636B6F7574004D61696E00536D6F6F745C
:1027C00068696E6700536D6F6F7468696E67005A51
:1027D000005A005900590058005800436F72726542
:1027E0006374696F6E00436F7272656374696F6EB4
:1027F000004D61696E00456E6473746F70204162B4
:102800006F7274004F6666004F6E00456E6473749D
:102810006F702041626F72740046696C616D656E05
:10282000740054656D706572617475726500426103
:10283000636B6C6173680053746570732F6D6D000A
:102840004A65726B00416363656C65726174696FA0
:102850006E0056656C6F6369747900436F6E6669CC
:102860006775726174696F6E004573746570732F5C
:102870006D6D004573746570732F6D6D005A7374C0
:102880006570732F6D6D005A73746570732F6D6D65
:10289000005973746570732F6D6D00597374657092
:1028A000732F6D6D005873746570732F6D6D0058C4
:1028B00073746570732F6D6D00416476616E63652E
:1028C000642053657474696E67730056652D4A659C
:1028D000726B0056652D4A65726B00567A2D4A65FB
:1028E000726B00567A2D4A65726B0056792D4A65D7
:1028F000726B0056792D4A65726B0056782D4A65C9
:10290000726B0056782D4A65726B00416476616E79
:102910006365642053657474696E677300416D610B
:1029200078204500416D6178204500416D61782037
:102930005A00416D6178205A00416D61782059003C
:10294000416D6178205900416D6178205800416DDA
:102950006178205800412D54726176656C00412DDC
:1029600054726176656C00412D52657472616374B6
:1029700000412D5265747261637400416363656C3C
:1029800000416363656C00416476616E6365642039
:1029900053657474696E6773005654726176204D86
:1029A000696E005654726176204D696E00566D69ED
:1029B0006E00566D696E00566D6178204500566D4B
:1029C0006178204500566D6178205A00566D617817
:1029D000205A00566D6178205900566D6178205953
:1029E00000566D6178205800566D6178205800417E
:1029F0006476616E6365642053657474696E677391
:102A0000002008204661637400200820466163743A
:102A1000002008204D6178002008204D61780020BA
:102A200008204D696E002008204D696E00417574C4
:102A30006F74656D70004F6666004F6E004175746F
:102A40006F74656D7000416476616E6365642053D8
:102A5000657474696E6773004C6F6164206D6D00FE
:102A60004C6F6164206D6D00556E6C6F6164206DFC
:102A70006D00556E6C6F6164206D6D004164766110
:102A80006E6365204B00416476616E6365204B0088
:102A9000416476616E6365642053657474696E6722
:102AA000730044697361626C65205374657070656E
:102AB0007273004D3834004175746F2043616C6946
:102AC0006272617465004D313137205374617274E4
:102AD000696E67204175746F2D43616C6962726124
:102AE00074696F6E0A54300A4732380A4D313137F3
:102AF000204C6576656C696E672058204178697353
:102B00000A473020583135302046393939390A479B
:102B10003238205A300A4D313137204C6576656C99
:102B2000696E6720646F6E652E0A4731320A4D3137
:102B300031372043616C6962726174696E672E2E51
:102B40002E0A473432350A4D3530300A4D3131378F
:102B50002043616C6962726174696F6E2064617494
:102B600061207361766564004175746F20486F6DF4
:102B70006500473238004C6576656C2058204178F6
:102B80006973004D313137204C6576656C696E672D
:102B9000205820417869730A473020583135302059
:102BA00046393939390A473238205A300A4D3131DD
:102BB00037204C6576656C696E6720646F6E652E94
:102BC000004D6F76652041786973004D61696E0034
:102BD000457874727564657220004175746F204881
:102BE0006F6D6500473238004D6F7665205A004D95
:102BF0006F76652059004D6F76652058004D6F74D3
:102C0000696F6E00457874727564657220004D6F4F
:102C100076652025736D6D00004D6F766520302E32
:102C2000316D6D004D6F766520316D6D004D6F76A5
:102C3000652031306D6D004D6F7665204178697388
:102C400000486F74656E6420746F6F20636F6C64EE
:102C500000457874727564657220004D6F7665204A
:102C60005A004D6F76652059004D6F7665205800EB
:102C70004D6F7665205A004D6F76652059004D6F77
:102C800076652058005072696E742066726F6D20F0
:102C90004D65646961005072696E742066726F6D73
:102CA000204D6564696100022E2E004D61696E0041
:102CB0005072696E740043616E63656C0053746199
:102CC0007274205072696E7420003F0057616974FD
:102CD00020666F720066696C616D656E7420707538
:102CE0007267650000506C65617365207761697477
:102CF0002E00507265737320427574746F6E007489
:102D00006F20726573756D65207072696E740057FF
:102D100061697420666F720066696C616D656E74BE
:102D2000206C6F616400496E736572742066696C13
:102D3000616D656E7400616E6420707265737320DE
:102D4000627574746F6E00746F20636F6E74696E59
:102D5000756500507265737320627574746F6E00D0
:102D6000746F2068656174206E6F7A7A6C65004EAE
:102D70006F7A7A6C652068656174696E6700506C63
:102D80006561736520776169742E2E2E0057616925
:102D90007420666F720066696C616D656E74207573
:102DA0006E6C6F6164005761697420666F720066B3
:102DB000696C616D656E74206368616E676500742F
:102DC0006F207374617274005061726B696E672E4C
:102DD0002E2E004368616E67696E672046696C61DC
:102DE0006D656E7400554E4C4F41442046494C4130
:102DF0004D454E54004C4F41442046494C414D45B1
:102E00004E540020204E6F7A7A6C653A20002000E4
:102E1000456E642066696C616D656E7420636861DF
:102E20006E6765005075726765206D6F7265000092
:102E30004368616E67652046696C616D656E7400FC
:102E4000556E6C6F61642046696C616D656E7400CF
:102E50004C6F61642046696C616D656E74004D361F
:102E6000303020423020542564004D373032203B32
:102E70002564004D37303220542564004D37303101
:102E80002054256400507265686561742043757331
:102E9000746F6D005072656865617420437573745A
:102EA0006F6D005072656865617420414253005037
:102EB00072656865617420504C41004261636B002B
:102EC0004E6F204D65646961005072696E742066B2
:102ED000726F6D204D65646961004368616E67655E
:102EE000204D65646961004D32310041626F757437
:102EF000205072696E746572004368616E67652068
:102F000046696C616D656E74004368616E6765202B
:102F100046696C616D656E74004D3630302042300C
:102F200000436F6E66696775726174696F6E0054F5
:102F3000656D7065726174757265004D6F74696F4F
:102F40006E00526573756D65205072696E74005421
:102F5000756E650053746F70205072696E74005006
:102F600061757365205072696E7400496E666F20DA
:102F700053637265656E0053746F70004261636BDA
:102F80000053746F70205072696E74003F0050726D
:102F90006F6265205A204F666673657400426162F5
:102FA0007973746570205900426162797374657039
:102FB000205800466C6F7700466C6F770046616E54
:102FC00020537065656420310046616E2053706542
:102FD000656420310042656400426564004E6F7A8A
:102FE0007A6C65004E6F7A7A6C6500537065656423
:102FF000005370656564004D61696E0042616279DD
:103000007374657020590042616279737465702031
:10301000580047616D6573005072696E7465722067
:103020005374617473004669726D776172652056DE
:10303000657273696F6E004D61696E00256973007A
:1030400025696D20256973002569682025696D2033
:1030500025697300256964202569682025696D202C
:103060002569730025697920256964202569682010
:1030700025696D20256973003E20004578747275BE
:1030800064656420546F74616C3A00256C642E256D
:10309000696D003E20004C6F6E67657374204A6F47
:1030A000622054696D653A003E2000546F74616C73
:1030B000205072696E742074696D653A00436F6DBB
:1030C000706C657465643A20005072696E742043B8
:1030D0006F756E743A2000436F6F6C646F776E008B
:1030E00046616E20537065656420310046616E2034
:1030F0005370656564203100426564004265640078
:103100004E6F7A7A6C65004E6F7A7A6C65004D610D
:10311000696E006F6F6F0000001FC07FF0DDD8FF89
:10312000F87FF04440248000003180000024804477
:1031300040107CFEFEFE04000E000E007FC0FFE08B
:10314000FFE0FFE0FFE006000F001F8036C03FC039
:1031500009001680294006000F001F8036C03FC0BE
:10316000168020401080104008801FC037607FF01C
:103170005FD050500D80104048905FD077707FF046
:103180001FC0104020200F007FE0FFF0E670FFF02E
:10319000198036C0C0300F007FE0FFF0E670FFF00E
:1031A000198036C0198047414D45204F5645520081
:1031B000526573746F7265206661696C73616665D0
:1031C000004C6F61642053657474696E67730053BB
:1031D000746F72652053657474696E677300507202
:1031E0006F6265205A204F6666736574004164768D
:1031F000616E6365642053657474696E6773004D16
:1032000061696E0050726F6265205A204F66667366
:103210006574004D6F76696E672E2E2E004D323428
:10322000004D323520500A4D3234005072696E74B0
:10323000205061757365640050617573652050722C
:10324000696E74005072696E742041626F727465A9
:1032500064004C756C7A426F74204C756C7A426FC6
:10326000742054415A2072656164792E005072694D
:103270006E74696E672E2E2E005072696E74205027
:103280006175736564004D656469612052656D6F99
:10329000766564004D6564696120496E736572747A
:1032A0006564004D313137004D33310043616E6E3E
:1032B0006F7420656E746572207375626469723A0A
:1032C00020002E0A006F70656E206661696C65646F
:1032D0002C2046696C653A20006175746F25632E59
:1032E00067006572726F722077726974696E672009
:1032F000746F2066696C650A004E6F742053442019
:103300007072696E74696E670A0053442070726946
:103310006E74696E67206279746520002E0A00441D
:10332000656C6574696F6E206661696C65642C20DC
:1033300046696C653A200046696C652064656C6579
:103340007465643A0057726974696E6720746F20FF
:1033500066696C653A20002E0A006F70656E206603
:1033600061696C65642C2046696C653A20002E0A00
:10337000006F70656E206661696C65642C2046691B
:103380006C653A200046696C652073656C656374F2
:1033900065640A002053697A653A200046696C65C5
:1033A000206F70656E65643A20002066696C653A2E
:1033B0002000667265736800646F696E67004E6F07
:1033C000772000454E4420535542524F5554494EA4
:1033D000450A002220706F73002220706172656EB2
:1033E000743A2200535542524F5554494E4520439A
:1033F000414C4C207461726765743A220074727992
:10340000696E6720746F2063616C6C207375622D28
:1034100067636F64652066696C657320776974689B
:1034200020746F6F206D616E79206C6576656C73AA
:103430002E204D4158206C6576656C2069733A31B9
:103440000A004D3234004D3233202573005344209E
:1034500063617264206F6B0A006F70656E526F6FEC
:1034600074206661696C65640A00766F6C756D65C1
:103470002E696E6974206661696C65640A00534444
:1034800020696E6974206661696C0A00286E6F207D
:1034900066696C65290043616E6E6F74206F70659C
:1034A0006E2073756264697220007C3C3E5E2B3D29
:1034B0003F2F5B5D3B2C2A225C000A003B204545E8
:1034C00050524F4D20496E6465783A200055706423
:1034D0006174696E67207A6F666673657420696EC1
:1034E00020454550524F4D3A200034746820707288
:1034F0006F626520706F696E742C206469737461EB
:103500006E63652066726F6D20706C616E653A2027
:1035100000000000000000000000000000000000AB
:10352000000000000000000000000000000000009B
:10353000000000000C000000000000000C00000073
:103540000000000012000000000000002300000046
:103550000000000021000000000000004C8000007E
:10356000000000005E8000000000000092400000AB
:1035700000000000A1400000000000012120000028
:10358000000000027F900000000000020010000018
:1035900000000007FFF80000000000040008000021
:1035A0000000000800040000000000080006000001
:1035B0000000001000020000000000301E010000AA
:1035C000000000207F81000000000041FFE080003B
:1035D00000000043FCF08000000000873B784000C2
:1035E0000000018EDBFC60000000010FEBCC20002E
:1035F0000000021FEDB610000000021FDEB6100032
:1036000000000439CD7F080000000436E0FF080008
:103610000000087EC0BB84000000187F005D8600AB
:103620000000107FC0ED82000000203CC07301004C
:103630000000203B337F01000000701BE77E038009
:103640000000C81DEEDE04C00000880FDEDC044070
:103650000001240FDF3C092000012607DBF81920B8
:1036600000027203E7F0139000025101FFE0229084
:10367000000489007F802448000904801E0048243B
:10368000000BFE400000DFF400100040000080024C
:10369000001FFFFFFFFFFFFE000000000000000012
:1036A000000000000000000000000000000000001A
:1036B000001022103C3C0E1F0010221004221104A6
:1036C000001022100822110400102210083C1104DE
:1036D00000102210102211040010221020221104C8
:1036E000001E1C1E3C3C0E040000000000000000F8
:1036F00000000000000000000000000000000000CA
:1037000000000000000000000000000000000000B9
:1037100000000000000000000000000000000000A9
:103720000000000000000000000000000000000099
:103730000000000000000000000000000000000089
:103740000000000000000000000000000000000079
:103750000C0D00FE07022603BC017FFE08FE08FEDA
:1037600005080806000040F0C88888987810050809
:1037700008060000C0F88888888888F805050506CE
:1037800000012030F830200508080600002070F8FD
:1037900020202020E00509090600FF2070A8A8B815
:1037A00088887020050606060001E08CEA8C8A0AEB
:1037B0000509090600FFF8A88888888888A8F80500
:1037C0000A0A0600FE205050505088A8A8887003AE
:1037D000030306000340A040FFFFFFFFFFFFFFFFC2
:1037E000FFFFFFFFFFFFFFFFFFFFFFFFFFFF0000E7
:1037F000000605FF01070706020080808080800028
:1038000080030303060105A0A0A00506060600002C
:1038100050F85050F8500509090600FF2070A8A084
:103820007028A87020050707060000C8C8102040AF
:10383000989805070706000040A0A040A8906801DE
:1038400003030602058080800309090601FF20406A
:10385000408080804040200309090601FF804040ED
:1038600020202040408005070706000020A8702087
:1038700070A8200505050600012020F8202002037D
:10388000030601FFC04080050101060003F80202A3
:1038900002060100C0C0050707060000081010203E
:1038A000404080050707060000708898A8C8887007
:1038B00003070706010040C040404040E0050707FD
:1038C000060000708808102040F805070706000071
:1038D000F8081030088870050707060000103050FF
:1038E00090F81010050707060000F880F008088817
:1038F00070050707060000304080F08888700507D3
:1039000007060000F8081010202020050707060011
:103910000070888870888870050707060000708826
:103920008878081060020505060100C0C000C0C00C
:103930000206060601FFC0C000C040800305050660
:1039400001012040804020050303060002F800F832
:103950000305050601018040204080050707060099
:1039600000708810202000200507070600007088DE
:10397000B8A8B88070050707060000708888F88826
:103980008888050707060000F04848704848F00599
:10399000070706000070888080808870050707068A
:1039A0000000F04848484848F0050707060000F8BE
:1039B0008080F08080F8050707060000F88080F01E
:1039C00080808005070706000070888080988870D6
:1039D000050707060000888888F888888803070795
:1039E000060100E04040404040E0050707060000B7
:1039F000381010101090600507070600008890A08E
:103A0000C0A0908805070706000080808080808025
:103A1000F805070706000088D8A888888888050761
:103A2000070600008888C8A8988888050707060048
:103A30000070888888888870050707060000F0886D
:103A400088F080808005070706000070888888A8B5
:103A50009068050707060000F08888F0A0908805A8
:103A60000707060000708880700888700507070641
:103A70000000F820202020202005070706000088ED
:103A800088888888887005070706000088888888E5
:103A900050502005070706000088888888A8A8508D
:103AA000050707060000888850205088880507070A
:103AB0000600008888502020202005070706000007
:103AC000F80810204080F80309090601FFE0808013
:103AD0008080808080E0050707060000804040204D
:103AE0001010080309090601FFE0202020202020F3
:103AF00020E00503030600052050880501010600AB
:103B0000FEF80303030601058040200505050600B5
:103B10000070087888780507070600008080F08824
:103B20008888F0050505060000708080887005070C
:103B300007060000080878888888780505050600CB
:103B4000007088F08070050707060000304840E0EC
:103B50004040400507070600FE7088888878087096
:103B60000507070600008080F0888888880307071B
:103B70000601004000C0404040E00409090601FE83
:103B8000100030101010109060050707060000802C
:103B9000808890E09088030707060100C0404040FD
:103BA0004040E0050505060000D0A8A8A8A8050526
:103BB00005060000B0C88888880505050600007065
:103BC000888888700507070600FEF0888888F080DE
:103BD000800507070600FE788888887808080505AC
:103BE00005060000B0C88080800505050600007845
:103BF000807008F00507070600002020F82020202C
:103C000018050505060000888888986805050506DA
:103C1000000088888850200505050600008888A8CF
:103C2000A8500505050600008850205088050707A4
:103C30000600FE88888850204080050505060000A3
:103C4000F8102040F80309090601FF204040408099
:103C5000404040200109090602FF8080808080806A
:103C60008080800309090601FF80404040204040D9
:103C7000408005030306000248A890FF4F46460017
:103C80004F4E006563686F3A004572726F723A007A
:103C90004572726F722077726974696E6720746FF3
:103CA00020454550524F4D210A00507265737320D4
:103CB000627574746F6E20286F72204D3130382910
:103CC00020746F2068656174206E6F7A7A6C650A63
:103CD00000507265737320627574746F6E20286F64
:103CE00072204D3130382920746F20726573756DE4
:103CF000650A00496E736572742066696C616D6552
:103D00006E7420616E6420707265737320627574C6
:103D1000746F6E20286F72204D313038290A004DA3
:103D20003630303A20546F6F20436F6C6400486F18
:103D300074656E6420746F6F20636F6C640A004852
:103D40006F74656E6420746F6F20636F6C640A001B
:103D5000496E736572742066696C616D656E74205E
:103D6000616E6420707265737320627574746F6E17
:103D700020286F72204D313038290A0063616E634C
:103D8000656C00726573756D656400726573756D41
:103D9000650070617573656400706F7765726F663A
:103DA00066002F2F616374696F6E3A0020573A00E6
:103DB00020573A00486F74656E6420436F6F6C69DA
:103DC0006E672E2E2E00486F74656E642048656104
:103DD00074696E672E2E2E00202F002042403A007C
:103DE00020403A00546865726D616C2052756E61B6
:103DF00077617900486F74656E6420544845524D70
:103E0000414C2052554E415741590042454420549F
:103E10004845524D414C2052554E41574159002082
:103E20002D20496E76616C696420657874727564C2
:103E30006572206E756D62657220210A00486561A9
:103E400074696E67206661696C6564004265642010
:103E500048656174696E67204661696C65640054E9
:103E60006865726D616C2052756E61776179004290
:103E7000454420544845524D414C2052554E4157DF
:103E800041590048656174696E67206661696C65B7
:103E90006400486F74656E642048656174696E677C
:103EA000204661696C656400546865726D616C20C0
:103EB00052756E6177617900486F74656E64205445
:103EC0004845524D414C2052554E41574159004DA5
:103ED000494E54454D502074726967676572656438
:103EE00000486F74656E64204572723A204D494EE9
:103EF00054454D50004572723A204D494E54454D3F
:103F00005020424544004D415854454D5020747254
:103F10006967676572656400486F74656E64204503
:103F200072723A204D415854454D50004572723AD4
:103F3000204D415854454D5020424544006265642F
:103F4000002C2073797374656D2073746F707065C5
:103F50006421204865617465725F49443A200023FA
:103F6000646566696E652044454641554C545F0062
:103F70004B6420004B6920004B7020000062656498
:103F800000504944204175746F74756E65206669F0
:103F90006E697368656421205075742074686520AB
:103FA0006C617374204B702C204B6920616E64200F
:103FB0004B6420636F6E7374616E74732066726FEE
:103FC0006D2062656C6F7720696E746F20436F6E31
:103FD00066696775726174696F6E2E680A00504970
:103FE00044204175746F74756E65206661696C65F7
:103FF00064212074696D656F75740A005468657278
:104000006D616C2052756E6177617900486F7465DF
:104010006E6420544845524D414C2052554E4157F4
:1040200041590042454420544845524D414C20528C
:10403000554E415741590048656174696E67206665
:1040400061696C656400486F74656E6420486561E1
:1040500074696E67204661696C656400426564201E
:1040600048656174696E67204661696C65640050DB
:104070004944204175746F74756E65206661696C82
:104080006564212054656D70657261747572652078
:10409000746F6F20686967680A00204B643A2000DB
:1040A000204B693A2000204B703A20000A20436CD4
:1040B000617373696320504944200A00204B643ABD
:1040C0002000204B693A2000204B703A20000A2043
:1040D0004E6F206F76657273686F6F740A0020549C
:1040E000753A2000204B753A2000206D61783A2007
:1040F00000206D696E3A200020643A200020626939
:1041000061733A2000504944204175746F74756E94
:10411000652073746172740A0050494420417574BB
:104120006F74756E65206661696C656421205465E5
:104130006D706572617475726520746F6F20686947
:1041400067680A001000AD0330016A0150022B01BC
:1041500070030A019004F500B005E500D006D80010
:10416000F007CE001009C500300ABE00500BB700A2
:10417000700CB100900DAB00B00EA600D00FA200E5
:10418000F0109D0010129900301395005014920009
:1041900070158E0090168B00B0178700D018840021
:1041A000F0198100101B7E00301C7B00501D79002F
:1041B000701E7600901F7300B0207000D0216E003A
:1041C000F0226B0010246900302566005026630041
:1041D0007027610090285E00B0295C00D02A590049
:1041E000F02B5600102D5400302E5100502F4E0051
:1041F00070304B0090314800B0324500D03342005F
:10420000F0343E0010363B00303737005038330072
:1042100070392E00903A2900B03B2300D03C1B009F
:10422000F03D1100103F0100F03F00001000C902F6
:1042300010012C014001220170011801B0010E0192
:10424000F00104015002FA00B002F0003003E60071
:10425000D003DC009004D2007005C800A006BE00A8
:104260000008B400B009AA00D00BA000600E9600B0
:1042700060118C000015820020197800C01D6E00AE
:10428000A0226400B0275A00902C50000031460054
:10429000E0343C0010383200903A2800603C1E00A8
:1042A000A03D1400803E0A00203F00006F70656E44
:1042B00000545249474745524544003A20007A5F2E
:1042C0006D6178007A5F6D696E00795F6D696E006F
:1042D000785F6D696E005265706F7274696E6720E9
:1042E000656E6473746F70207374617475730A0003
:1042F000456E6473746F70732025632025632025D9
:104300006320256300205A3A0020593A0020583A89
:1043100000656E6473746F7073206869743A20006E
:10432000486F6D696E67204661696C6564000A5369
:10433000746174733A2046696C616D656E742075A2
:104340007365643A20002C204C6F6E67657374208F
:104350006A6F623A2000546F74616C2074696D65F5
:104360003A200053746174733A20002C204661692E
:104370006C65643A20002C2046696E697368656438
:104380003A20005072696E74733A2000537461745D
:10439000733A2000496E76616C69642065787472A6
:1043A000756465720A0045313A200045303A2000B4
:1043B0005A3A2000593A20004D53312C4D53322C9B
:1043C0004D53332050696E730A583A20004D69638B
:1043D000726F737465707320756E617661696C615C
:1043E000626C650A00205A3A0020593A0020436F57
:1043F000756E7420583A00C23100001C260000F48B
:10440000190000D80F0000EB080000C00400007580
:104410000200004001000024F4D43050C38E20C2BA
:10442000A24017828B7011127A910D816CD90AA863
:1044300061E108C7586607615143061E4B5D05C11F
:1044400045A7041A411104093D980371393103400D
:1044500036DB0265339102D4305402802E1D026394
:104460002CEE01752AC501B028A001102781018F0B
:104470002564012B244B01E0223401AC211F018D66
:10448000200D01801FFC00841EED00971DDF00B889
:104490001CD200E61BC600201BBC00641AB200B28E
:1044A00019A8000A19A0006A189900D117910040B4
:1044B000178B00B516840031167E00B31579003ACB
:1044C000157300C7146F0058146A00EE1366008855
:1044D00013630025135E00C7125B006C12570015B2
:1044E000125400C111510070114F0021114B00D620
:1044F0001049008D1047004610440002104200C0D1
:104500000F4000800F3E00420F3C00060F3B00CBE7
:104510000E3800930E37005C0E3500270E3400F382
:104520000D3200C10D3100900D3000600D2E0032B3
:104530000D2D00050D2C00D90C2B00AE0C2900858B
:104540000C29005C0C2700350C27000E0C2600E817
:104550000B2400C40B2400A00B23007D0B23005A66
:104560000B2100390B2100180B2000F80A1F00D97D
:104570000A1E00BB0A1E009D0A1D00800A1D006362
:104580000A1C00470A1B002C0A1B00110A1A00F71C
:10459000091A00DD091900C4091900AB09190092B4
:1045A0000917007B091800630917004C091600362B
:1045B000091600200916000A091500F5081500E083
:1045C000081400CC081400B8081400A408140090C3
:1045D0000813007D0812006B0813005808120046EB
:1045E00008120034081100230811001208110001FC
:1045F000081100F0071000E0071000D0071000C0FD
:10460000071000B0070F00A107100091070E0083EC
:10461000070F0074070F0065070E0057070E0049CB
:10462000070E003B070D002E070E0020070D00139C
:10463000070D0006070D00F9060C00ED060D00E061
:10464000060C00D4060C00C8060C00BC060C00B01A
:10465000060C00A4060B0099060C008D060B0082C8
:10466000060B0077060B006C060B0061060A00576C
:10467000060B004C060A0042060A0038060A002E05
:10468000060A0024060A001A060A00100609000796
:10469000060A00FD050900F4050900EB050900E222
:1046A000050900D9050900D0050900C7050900BEA4
:1046B000050900B5050800AD050800A50509009C21
:1046C000050800940508008C050800840508007C96
:1046D000050800740508006C050700650508005D05
:1046E000050700560508004E05070047050700406E
:1046F00005080038050700310507002A05070023D3
:104700000507001C050600160507000F0507000831
:1047100005060002050700FB040600F5040700EE8D
:10472000040600E8040600E2040700DB040600D5E6
:10473000040600CF040600C9040600C3040600BD39
:10474000040600B7040600B1040500AC040600A688
:10475000040600A00405009B0406009504050090D3
:104760000406008A04050085040500800406007A1A
:1047700004050075040500700405006B040500665F
:10478000040500610405005C04050057040500529F
:104790000405004D04050048040500430405003EDF
:1047A0000404003A04050035040500300404002C1C
:1047B00004050027040400230405001E0404001A55
:1047C00004040016040500110404000D040400098B
:1047D0000405000404040000040400FC030400F8C1
:1047E000030400F4030400F0030400EC030400E8F5
:1047F000030400E4030400E0030400DC030400D825
:10480000030400D4030400D0030400CC030400C854
:10481000030300C503030024F404D9201BC40C5C6B
:104820000E9804C4095F0265077101F405F900FBE5
:1048300004B30048048700C103690058035500030E
:10484000034500BE023A008402310053022A0029C7
:1048500002250004022000E4011C00C8011900AF79
:104860000117009801140084011300710110006108
:1048700001100051010E0043010D0036010B002B09
:10488000010B0020010B00150109000C01090003B8
:10489000010800FB000800F3000800EB000700E43B
:1048A000000600DE000600D8000600D2000600CC9C
:1048B000000500C7000500C2000500BD000400B9E6
:1048C000000400B5000400B1000400AD000400A91C
:1048D000000400A5000300A20003009F0004009B49
:1048E000000300980003009500020093000300906D
:1048F0000003008D0002008B000300880002008688
:1049000000020084000300810002007F0002007D9D
:104910000002007B000200790002007700010076AF
:104920000002007400020072000100710002006FBA
:104930000002006D0001006C0002006A00010069C5
:1049400000020067000100660001006500010064CC
:104950000002006200010061000100600001005FD0
:104960000002005D0001005C0001005B0001005AD4
:1049700000010059000100580001005700010056D5
:1049800000010055000100540001005300000053D5
:104990000001005200010051000100500001004FD1
:1049A0000001004E0000004E0001004D0001004CCF
:1049B0000001004B0000004B0001004A00010049CB
:1049C00000010048000000480001004700010046C7
:1049D00000000046000100450000004500010044C1
:1049E00000010043000000430001004200000042BB
:1049F0000001004100000041000100400001003FB3
:104A00000000003F0001003E0000003E0001003DAC
:104A10000000003D0001003C0000003C0000003CA4
:104A20000001003B0000003B0001003A0000003A9A
:104A30000001003900000039000100380000003892
:104A40000000003800010037000000370001003688
:104A5000000000360000003600010035000000357F
:104A60000000003500010034000000340000003474
:104A70000001003300000033000000330001003269
:104A8000000000320000003200010031000000315F
:104A90000000003100010030000000300000003054
:104AA0000001002F0000002F0000002F0000002F49
:104AB0000001002E0000002E0000002E0001002D3D
:104AC0000000002D0000002D0000002D0001002C32
:104AD0000000002C0000002C0000002C0001002B26
:104AE0000000002B0000002B0000002B0001002A1A
:104AF0000000002A0000002A0000002A000100290E
:104B00000000002900000029000000290000002901
:104B100000010028000000280000002800000028F4
:104B200000000028000100270000002700000027E7
:104B300000000027000000270001002600000026DA
:104B400000000026000000260000002600010025CD
:104B500000000025000000250000002500000025C1
:104B600000000025000100240000002400000024B3
:104B700000000024000000240001002300000023A6
:104B80000000002300000023000000230000002399
:104B9000000000230001002200000022000000228B
:104BA000000000220000002200000022000100217D
:104BB0000000002100000021000000210000002171
:104BC0000000002100000021000100200000002062
:104BD0000000002000000020000000200000002055
:104BE00000000020000000200001001F0000001F46
:104BF0000000001F0000001F0000001F0000001F39
:104C00000000001F0001001E0000001E0000001E2A
:104C10000000001E00000020204D36303320003AF6
:104C20000A0020286D6D2900205300205A002059C9
:104C30000020580020204D34323520460042616368
:104C40006B6C61736820636F6D70656E73617469FE
:104C50006F6E3A0A002055004C0046696C616D6524
:104C60006E74206C6F61642F756E6C6F6164206C64
:104C7000656E677468733A0A0020204D3930302021
:104C80004B004C696E65617220416476616E6365AC
:104C90003A0A0020204D383531205A005A2D5072E2
:104CA0006F6265204F66667365740020440020497A
:104CB0000020204D33303420500020440020490093
:104CC00020204D333031205000504944207365740A
:104CD00074696E67733A0A0020460020420020483B
:104CE0000020204D3134352053004D6174657269C8
:104CF000616C2068656174757020706172616D65AA
:104D0000746572733A0A0020204D3432302053000B
:104D10004175746F20426564204C6576656C696EE0
:104D2000673A0A00204500205A0020590020580008
:104D300020540020530020204D32303520420020E6
:104D4000453C6D61785F655F6A65726B3E00205817
:104D50003C6D61785F785F6A65726B3E20593C6D8F
:104D600061785F795F6A65726B3E205A3C6D61784D
:104D70005F7A5F6A65726B3E00416476616E63655F
:104D8000643A20423C6D696E5F7365676D656E7451
:104D90005F74696D655F75733E20533C6D696E5F2E
:104DA00066656564726174653E20543C6D696E5F32
:104DB00074726176656C5F66656564726174653E88
:104DC0000020540020520020204D3230342050006A
:104DD000416363656C65726174696F6E2028756EDE
:104DE0006974732F7332293A20503C7072696E7463
:104DF0005F616363656C3E20523C726574726163EF
:104E0000745F616363656C3E20543C7472617665C7
:104E10006C5F616363656C3E0A00204500205A00A8
:104E200020590020204D3230312058004D617869E2
:104E30006D756D20416363656C65726174696F6E39
:104E40002028756E6974732F7332293A0A00204541
:104E500000205A0020590020204D323033205800C5
:104E60004D6178696D756D20666565647261746504
:104E7000732028756E6974732F73293A0A0053746E
:104E80006570732070657220756E69743A0A00202F
:104E9000204D3134392043203B20556E69747320F6
:104EA000696E2043656C736975730A002020473270
:104EB00031202020203B20556E69747320696E20BC
:104EC0006D6D0048617264636F646564204465665B
:104ED00061756C742053657474696E6773204C6FD0
:104EE000616465640A002823000028230000C800CC
:104EF00000002823000000009643000096430000B5
:104F0000F0410000C8410000C8420000C842000053
:104F1000FA430000D243454550524F4D20496E6937
:104F20007469616C697A65640A00290A00206279F3
:104F30007465733B2063726320002073746F726525
:104F4000642073657474696E677320726574726926
:104F500065766564202800202863616C63756C6148
:104F600074656429210A0020213D200045455052E6
:104F70004F4D20435243206D69736D617463682007
:104F80002D202873746F7265642920002053697A7C
:104F9000653A2000496E6465783A2000204D6172C0
:104FA0006C696E3D563639290A00454550524F4DC1
:104FB0002076657273696F6E206D69736D617463BD
:104FC000682028454550524F4D3D004E6F204545C5
:104FD00050524F4D2E0A00290A00206279746573E1
:104FE0003B20637263200053657474696E6773209D
:104FF00053746F7265642028004E6F2045455052EF
:105000004F4D2E0A00454550524F4D20646174614A
:1050100073697A65206572726F722E0A0041757429
:105020006F6C6576656C206661696C65640A004129
:1050300075746F6C6576656C206661696C6564007B
:10504000205A3A200020593A200042656420583AFC
:1050500020005761726E696E673A20486F6D696E05
:10506000672042756D702044697669736F72203CC9
:1050700020310A00020204486F6D652025732573F4
:105080002573204669727374002046697273740A2E
:1050900000486F6D65200020746F6F206C6F6E6725
:1050A00020657874727573696F6E207072657665AD
:1050B0006E7465640A0020636F6C64206578747296
:1050C0007573696F6E2070726576656E7465640ABB
:1050D0000020453A00205A3A0020593A00583A0038
:1050E00000004842000048420000F041FFFF01007C
:1050F00000A0400000A040000000400080AC430041
:1051000080A24300809643000048C2000088C1008E
:105110008095430080934300009A430080954300AC
:105120000048C2000088C1000000C020746F6F20DA
:105130006C6F6E6720657874727573696F6E20701E
:10514000726576656E7465640A0020636F6C642016
:10515000657874727573696F6E2070726576656EAE
:105160007465640A00627573793A207061757365BD
:105170006420666F7220696E7075740A00627573C0
:10518000793A2070617573656420666F722075735B
:1051900065720A00627573793A2070726F63657385
:1051A00073696E670A004D3131372050726F626546
:1051B000207375636365737366756C0020496E7642
:1051C000616C696420657874727564657220002072
:1051D0005A3A200020593A200042656420583A206B
:1051E0000050726F6265205A204F66667365743A8C
:1051F00020003F5A206F7574206F662072616E67C1
:105200006520282D3220746F2035290A004D313455
:105210003520533C696E6465783E206F7574206F4D
:10522000662072616E67652028302D31290A00439F
:105230006C69636B20746F20526573756D652E2EDB
:105240002E00220A00556E6B6E6F776E20636F6DB5
:105250006D616E643A202200454550524F4D204FFB
:105260004B0A004E6F204D6F76652E004543484F28
:1052700000494E464F004552524F52530044525936
:1052800052554E00434F4D4D554E49434154494FA1
:105290004E006F6666006C52715276527D52845297
:1052A00044454255473A0054415A20576F726B6843
:1052B0006F7273652045646974696F6E204F46464E
:1052C0002E00205A00205900580020204D61783AC5
:1052D0002000205A00205900580020204D696E3AC5
:1052E0002000536F667420656E6473746F70733A38
:1052F00020005072696E742074696D653A20004D0B
:105300003131332053002F2F20004361703A004386
:1053100048414D4245525F54454D504552415455C8
:105320005245004D4F54494F4E5F4D4F4445530039
:10533000544845524D414C5F50524F544543544997
:105340004F4E004155544F5245504F52545F5344B5
:105350005F5354415455530050524F4D50545F5376
:105360005550504F525400454D455247454E4359B4
:105370005F50415253455200434153455F4C4947AA
:1053800048545F4252494748544E45535300544F86
:1053900047474C455F4C494748545300534F465488
:1053A000574152455F504F574552004255494C4472
:1053B0005F50455243454E54004C4556454C494E6E
:1053C000475F44415441005A5F50524F42450041AB
:1053D00055544F4C4556454C005052494E545F4A27
:1053E0004F420050524F4752455353004155544F7E
:1053F0005245504F52545F54454D5000564F4C55F6
:105400004D455452494300454550524F4D00424985
:105410004E4152595F46494C455F5452414E5346A6
:1054200045520053455249414C5F584F4E5F584FCB
:105430004646004649524D574152455F4E414D4503
:105440003A4D61726C696E20322E302E302E31371B
:105450003120284769746875622920534F5552439B
:10546000455F434F44455F55524C3A6874747073BE
:105470003A2F2F636F64652E616C6570686F626A86
:10548000656374732E636F6D2F64696666757369E7
:105490006F6E2F4D41524C494E2050524F544F4346
:1054A0004F4C5F56455253494F4E3A312E30204DA6
:1054B000414348494E455F545950453A54415A205A
:1054C000576F726B686F7273652045646974696F9A
:1054D0006E2045585452554445525F434F554E54E3
:1054E0003A3120555549443A356565373938666251
:1054F0002D343036322D346433352D383232342D5C
:105500003565383436666662343561350A002028E0
:105510004E6F7420796574206D6561737572656472
:105520002900202041766572616765206D65617391
:1055300075726564206261636B6C61736820286DAD
:105540006D293A002020536D6F6F7468696E672073
:10555000286D6D293A202020202020202020202086
:10556000202020202020530020204261636B6C61AA
:1055700073682044697374616E636520286D6D29BA
:105580003A202020202020202000202846312E30C4
:10559000203D2066756C6C2C2046302E30203D203E
:1055A0006E6F6E65290A002020436F727265637406
:1055B000696F6E20416D6F756E742F466164652D45
:1055C0006F75743A2020202020460061637469764C
:1055D000653A0A00696E004261636B6C6173682012
:1055E000436F7272656374696F6E2000205A0020E9
:1055F000580020506F736974696F6E616C2045723A
:10560000726F723A0A002058004E6F7A7A6C6520E9
:10561000546970204F757465722044696D656E73AE
:10562000696F6E733A0A002020546F703A20002090
:10563000204261636B3A2000202052696768743A07
:10564000200020204C6566743A20004261636B6C38
:105650006173683A0A00205A0020580043656E744E
:1056600065723A0A0020204261636B3A20002020D4
:1056700052696768743A200020204C6566743A20AD
:10568000002020546F703A200053696465733A0A11
:1056900000426564204C6576656C696E6720004643
:1056A00061696C656420746F20656E61626C652051
:1056B000426564204C6576656C696E670A004265D8
:1056C00064204C6576656C20436F72726563746903
:1056D0006F6E204D61747269783A000A0A426564FF
:1056E000204C6576656C20436F7272656374696FD8
:1056F0006E204D61747269783A00202B000A436F66
:1057000072726563746564204265642048656967E8
:1057100068742076732E2042656420546F706F6C1D
:105720006F67793A0A00202B000A426564204865B9
:105730006967687420546F706F6772617068793A36
:105740000A2020202B2D2D2D204241434B202D2D92
:105750002B0A2020207C20202020202020202020F8
:10576000207C0A204C207C20202020282B2920204F
:1057700020207C20520A2045207C20202020202030
:1057800020202020207C20490A2046207C20282D13
:1057900029204E20282B29207C20470A2054207CB9
:1057A00020202020202020202020207C20480A208B
:1057B00020207C20202020282D29202020207C2013
:1057C000540A2020207C202020202020202020205F
:1057D000207C0A2020204F2D2D2046524F4E542051
:1057E0002D2D2B0A2028302C30290A000A4D656106
:1057F0006E206F662073616D706C656420706F69D8
:105800006E74733A200020643A200020623A20002F
:1058100045716E20636F656666696369656E747352
:105820003A20613A200050726F62696E6720506FB3
:10583000696E742025692F2569002E0A002F0050FB
:10584000726F62696E67206D65736820706F696E34
:10585000742000202844525952554E2900473239AD
:10586000204175746F20426564204C6576656C69D3
:105870006E67003F20284C2C522C462C4229206F6A
:105880007574206F6620626F756E64732E0A003F18
:1058900050726F626520706F696E74732028592989
:1058A00020696D706C61757369626C652028322D9A
:1058B00032292E0A003F50726F626520706F696E48
:1058C00074732028582920696D706C617573696242
:1058D0006C652028322D32292E0A003F2856296572
:1058E00072626F7365206C6576656C20696D706C93
:1058F00061757369626C652028302D34292E0A0089
:1059000043757272656E742066696C653A20004555
:105910006E642066696C65206C6973740A00426568
:1059200067696E2066696C65206C6973740A004152
:105930006476616E6365204B3D003F4B2076616C61
:105940007565206F7574206F662072616E676520C3
:1059500028302D3130292E0A004D31313720486F43
:105960007420656E642068656174696E672E2E2EE2
:105970000A4D31303420533137300A473238204F06
:10598000310A4D31313720576970696E67206E6F6B
:105990007A7A6C650A54300A473120582D31372005
:1059A000593235205A31302046343030300A4D31AA
:1059B000303920523137300A4731205A310A4D31BF
:1059C00031340A473120582D3137205932350A47B2
:1059D0003120582D3137205939350A473120582D7B
:1059E0003137205932350A473120582D3137205967
:1059F00039350A473120582D3137205932350A4779
:105A00003120582D3137205939350A473120582D4A
:105A10003137205932350A473120582D3137205936
:105A200039350A473120582D3137205932350A4748
:105A30003120582D3137205939350A473120582D1A
:105A40003137205932350A473120582D3137205906
:105A500039350A4731205A31350A4D3430300A4D34
:105A600031303620533235350A473020582D313009
:105A700020592D394D31303920523136300A4D31CF
:105A8000303700473238004D6163726F20746F6F9A
:105A9000206C6F6E672E0A0020466C6F773A2000EC
:105AA00020643A0020693A0020703A002045002026
:105AB0005A00205900204D393220580043290A004D
:105AC00061626C656420286D696E2074656D70205C
:105AD0000064697300656E00436F6C6420657874C0
:105AE0007275646573206172652000205400205235
:105AF00000416363656C65726174696F6E3A205032
:105B000000496E76616C69642065787472756465AD
:105B1000720A0020643A0020693A0020703A00536B
:105B20006C6565702E2E2E0047322F473320626140
:105B30006420706172616D65746572730A005072E1
:105B40006F6265205A204F66667365743A20004480
:105B50006F6E6520736176696E672066696C652E6D
:105B60000A0053442072656164206572726F720A84
:105B700000446F6E65207072696E74696E6720668E
:105B8000696C650A004D32390053544F50504544FA
:105B90002E20005072696E7465722073746F70707D
:105BA00065642064756520746F206572726F72730E
:105BB0002E2046697820746865206572726F7220A5
:105BC000616E6420757365204D39393920746F20FA
:105BD000726573746172742E202854656D706572DD
:105BE00061747572652069732072657365742E2007
:105BF00053657420697420616674657220726573E0
:105C000074617274696E67290A004E6F204368657B
:105C1000636B73756D2077697468206C696E65209D
:105C20006E756D6265722C204C617374204C696EC8
:105C3000653A20004E6F20436865636B73756D2075
:105C400077697468206C696E65206E756D62657227
:105C50002C204C617374204C696E653A2000636897
:105C600065636B73756D206D69736D617463682C0A
:105C7000204C617374204C696E653A20004C696E4B
:105C800065204E756D626572206973206E6F742099
:105C90004C617374204C696E65204E756D6265723F
:105CA0002B312C204C617374204C696E653A2000B6
:105CB0004D31313000526573656E643A20002042E8
:105CC000002050006F6B00220A00656E71756575CB
:105CD00065696E67202200504944204175746F74D5
:105CE000756E65206661696C65642120426164207F
:105CF0006578747275646572206E756D6265720A7E
:105D00000042656420436F6F6C696E672E2E2E0013
:105D10004265642048656174696E672E2E2E006F9F
:105D20006B004739310A4730205A3135204636302A
:105D3000300A4739300A473020583137302059323D
:105D400039302046333030300A4D313137205072EF
:105D5000696E742061626F727465642E0047323818
:105D6000205A002020506C616E6E65724275666626
:105D7000657242797465733A200020467265652029
:105D80004D656D6F72793A2000436F6D70696C6577
:105D9000643A204F637420203820323031390A00B1
:105DA000207C20417574686F723A2028416C6570C0
:105DB00068204F626A6563747320496E632E2C20DD
:105DC0004C756C7A426F7420476974205265706F0D
:105DD0007369746F7279290A004F63742020382028
:105DE0003230313931323A34393A313800204C616D
:105DF000737420557064617465643A2000322E30EB
:105E00002E302E3137310A004D61726C696E0020E0
:105E1000536F6674776172652052657365740A000A
:105E2000205761746368646F672052657365740AF4
:105E3000002042726F776E206F7574205265736513
:105E4000740A002045787465726E616C2052657327
:105E500065740A00506F77657255700A007374613B
:105E600072740A004B494C4C45442E200050726914
:105E70006E7465722068616C7465642E206B696C49
:105E80006C28292063616C6C6564210A004B494CC5
:105E90004C2063617573656420627920746F6F2094
:105EA0006D75636820696E616374697665207469D5
:105EB0006D65202D2063757272656E7420636F6D41
:105EC0006D616E643A20004D3130342053313730EB
:105ED0000A4D313137204C6576656C696E67205804
:105EE00020417869730A47302058313530204639CF
:105EF0003939390A473238205A300A4D3131372082
:105F00004C6576656C696E6720646F6E652E0A4716
:105F100031320A4D31303920523136300A4D343069
:105F2000300A4D3131372050726F62696E672062DE
:105F300065640070726F62655F7265776970650095
:105F40004175746F6C6576656C206661696C65641B
:105F5000004D31313720426564206C6576656C698F
:105F60006E67206661696C65642E0A4730205A317D
:105F7000300A47302045300A4D333030205032351A
:105F800020533838300A4D333030205035302053CC
:105F9000300A4D3330302050323520533838300AF3
:105FA0004D333030205035302053300A4D333030AF
:105FB0002050323520533838300A473420533100CE
:105FC00070726F62655F6661696C65640050726FC4
:105FD0007465637465642050696E0A0025301D0C79
:105FE000282924311C0B4527232F1B0A1E4443223A
:105FF0002B1A4142033809FF36030806020200014A
:106000002F49F78B2A96A0AD55CAE400E200E000C4
:10601000E6004A9611241FBECFEFD1E2DEBFCDBF0E
:1060200000E00CBF13E0A0E0B2E0E2E6F3ED02E036
:106030000BBF02C007900D92AA3EB107D9F727E126
:10604000AAEEB3E001C01D92A53FB207E1F710E34D
:10605000C9E0D0E300E006C021970109802FFE01CE
:106060000F94E75EC030D10780E00807A9F70E94CF
:10607000A53C0D949F690C9400001F920F920FB6DF
:106080000F9211242F933F938F939F93AF93BF93BE
:106090008091EB039091EC03A091ED03B091EE039E
:1060A0003091EA0323E0230F2D3720F40196A11D40
:1060B000B11D05C026E8230F0296A11DB11D209336
:1060C000EA038093EB039093EC03A093ED03B0936A
:1060D000EE038091EF039091F003A091F103B09152
:1060E000F2030196A11DB11D8093EF039093F0037D
:1060F000A093F103B093F203BF91AF919F918F9161
:106100003F912F910F900FBE0F901F9018952FB7B2
:10611000F8946091EB037091EC038091ED03909102
:10612000EE032FBF08953FB7F8948091EF0390914D
:10613000F003A091F103B091F20326B5A89B05C02E
:106140002F3F19F00196A11DB11D3FBFBA2FA92FF6
:10615000982F8827820F911DA11DB11DBC01CD0173
:1061600042E0660F771F881F991F4A95D1F708955F
:106170008F929F92AF92BF92CF92DF92EF92FF9257
:106180006B017C01D0DF4B015C01C114D104E1043F
:10619000F104F1F09CD3C7DFDC01CB018819990928
:1061A000AA09BB09883E9340A105B10570F321E01F
:1061B000C21AD108E108F10888EE880E83E0981E23
:1061C000A11CB11CC114D104E104F10421F7DDCFFD
:1061D000FF90EF90DF90CF90BF90AF909F908F9007
:1061E00008958230910538F0880F991F880F991F04
:1061F00005970197F1F70895789484B5826084BD7E
:1062000084B5816084BD85B5826085BD85B58160BA
:1062100085BDEEE6F0E0808181608083E1E8F0E01A
:106220001082808182608083808181608083E0E849
:10623000F0E0808181608083E1EBF0E08081846028
:106240008083E0EBF0E0808181608083E1E9F0E031
:10625000808182608083808181608083E0E9F0E0DA
:10626000808181608083E1EAF0E0808182608083C8
:10627000808181608083E0EAF0E0808181608083BA
:10628000E1E2F1E0808182608083808181608083AF
:10629000E0E2F1E0808181608083EAE7F0E08081E4
:1062A000846080838081826080838081816080833C
:1062B0008081806880831092C10008951F93CF93DE
:1062C000DF93182FEB0161E016D1209711F460E005
:1062D00004C0CF3FD10531F461E0812FDF91CF9130
:1062E0001F9145C1E12FF0E0EB5FFC4FE4914E2F91
:1062F00050E0FA013197E231F10508F09DC088279E
:10630000EE58FF4F8F4F0D94E75E84B5806884BDD3
:10631000C7BD97C084B5806284BDC8BD92C080915E
:106320008000806880938000D0938900C0938800AB
:1063300088C080918000806280938000D0938B0021
:10634000C0938A007EC08091800088608093800026
:10635000D0938D00C0938C0074C08091B000806891
:106360008093B000C093B3006CC08091B000806295
:106370008093B000C093B40064C0809190008068A6
:1063800080939000D0939900C09398005AC0809158
:106390009000806280939000D0939B00C0939A00FD
:1063A00050C080919000886080939000D0939D00B1
:1063B000C0939C0046C08091A00080688093A0009C
:1063C0008091A0008F7B8093A000D093A900C09300
:1063D000A80037C08091A00080628093A000D09375
:1063E000AB00C093AA002DC08091A000886080936C
:1063F000A000D093AD00C093AC0023C080912001D9
:10640000806880932001D0932901C093280119C08E
:1064100080912001806280932001D0932B01C09352
:106420002A010FC080912001886080932001D093C1
:106430002D01C0932C0105C0C038D1050CF04CCF04
:1064400046CFDF91CF911F91089590E0FC013197E5
:10645000E231F10508F04EC08827EC57FF4F8F4F0F
:106460000D94E75E809180008F7703C0809180005B
:106470008F7D80938000089580918000877FF9CF81
:1064800084B58F7702C084B58F7D84BD08958091D7
:10649000B0008F7703C08091B0008F7D8093B000F3
:1064A0000895809190008F7707C0809190008F7D34
:1064B00003C080919000877F809390000895809121
:1064C000A0008F7707C08091A0008F7D03C08091CE
:1064D000A000877F8093A0000895809120018F778E
:1064E00007C0809120018F7D03C080912001877FAC
:1064F000809320010895CF93DF9390E0FC01E55B4A
:10650000FC4F2491FC01EF56FC4F8491882361F1EC
:1065100090E0880F991FFC01E55FFB4FC591D49176
:10652000FC01EF50FC4FA591B491611109C09FB7D8
:10653000F8948881209582238883EC912E230BC0C8
:10654000623061F49FB7F8943881822F809583235D
:106550008883EC912E2B2C939FBF06C08FB7F894A5
:10656000E8812E2B28838FBFDF91CF9108951F9351
:10657000CF93DF93282F30E0F901EB5FFC4F84913C
:10658000F901E55BFC4FD491F901EF56FC4FC49142
:10659000CC23C1F0162F811158DFEC2FF0E0EE0F65
:1065A000FF1FEF50FC4FA591B4918FB7F8941111D4
:1065B00005C09C91ED2FE095E92302C0EC91ED2BF5
:1065C000EC938FBFDF91CF911F910895CF93DF930D
:1065D000282F30E0F901EB5FFC4F8491F901E55B76
:1065E000FC4FD491F901EF56FC4FC491CC2389F0B4
:1065F00081112BDFEC2FF0E0EE0FFF1FE952FC4F73
:10660000A591B491EC91ED2381E090E021F480E03C
:1066100002C080E090E0DF91CF91089508951F922D
:106620000F920FB60F9211240BB60F922F933F9338
:106630004F935F936F937F938F939F93AF93BF938A
:10664000EF93FF93E0910802F09109021995FF91F1
:10665000EF91BF91AF919F918F917F916F915F91DA
:106660004F913F912F910F900BBE0F900FBE0F9047
:106670001F9018951F920F920FB60F9211240BB610
:106680000F922F933F934F935F936F937F938F93CB
:106690009F93AF93BF93EF93FF93E0910A02F09122
:1066A0000B021995FF91EF91BF91AF919F918F913F
:1066B0007F916F915F914F913F912F910F900BBE02
:1066C0000F900FBE0F901F9018951F920F920FB64C
:1066D0000F9211240BB60F922F933F934F935F931A
:1066E0006F937F938F939F93AF93BF93EF93FF939A
:1066F000E0910C02F0910D021995FF91EF91BF917D
:10670000AF919F918F917F916F915F914F913F9149
:106710002F910F900BBE0F900FBE0F901F901895EA
:106720001F920F920FB60F9211240BB60F922F9358
:106730003F934F935F936F937F938F939F93AF9309
:10674000BF93EF93FF93E0910E02F0910F02199522
:10675000FF91EF91BF91AF919F918F917F916F9139
:106760005F914F913F912F910F900BBE0F900FBEF5
:106770000F901F9018951F920F920FB60F92112431
:106780000BB60F922F933F934F935F936F937F932B
:106790008F939F93AF93BF93EF93FF93E091040286
:1067A000F09105021995FF91EF91BF91AF919F91E3
:1067B0008F917F916F915F914F913F912F910F90AA
:1067C0000BBE0F900FBE0F901F9018951F920F9247
:1067D0000FB60F9211240BB60F922F933F934F9346
:1067E0005F936F937F938F939F93AF93BF93EF9339
:1067F000FF93E0910602F09107021995FF91EF9146
:10680000BF91AF919F918F917F916F915F914F91C8
:106810003F912F910F900BBE0F900FBE0F901F90C6
:1068200018951F920F920FB60F9211240BB60F926C
:106830002F933F934F935F936F937F938F939F9388
:10684000AF93BF93EF93FF93E0911002F091110289
:106850001995FF91EF91BF91AF919F918F917F918A
:106860006F915F914F913F912F910F900BBE0F90C1
:106870000FBE0F901F9018951F920F920FB60F9298
:1068800011240BB60F922F933F934F935F936F9307
:106890007F938F939F93AF93BF93EF93FF93E09179
:1068A0001202F09113021995FF91EF91BF91AF91F0
:1068B0009F918F917F916F915F914F913F912F9118
:1068C0000F900BBE0F900FBE0F901F90189508955C
:1068D0001F93CF93DF93EC011D821C821F821E82C7
:1068E000198681E0888782E28A871F861E86FE01DC
:1068F000B396CE01C1962FEF2193E817F907E1F780
:1069000011E018A3CE0113D61F8B188E198E80E4C8
:106910008A8F1B8E88E698E39AAB89ABDF91CF9183
:106920001F910895DB01ED91FC911994EF92FF9274
:106930001F93CF93DF931F921F92CDB7DEB77C01D9
:10694000DC01D196ED91FC91D29782E069837A8344
:10695000199520E030E04AE069817A81C701E2DFE1
:10696000182FD701D196ED91FC91D29783E019951C
:10697000D701D196ED91FC91D29780E01995812FA6
:106980000F900F90DF91CF911F91FF90EF9008959E
:106990000F931F93CF93DF93EC018B01E9A9FAA921
:1069A00082E01995E9A9FAA981E0199520E030E083
:1069B00044E1B801CE01B6DF9E012D5C3F4F47E1B7
:1069C000B801CE01AFDFE9A9FAA980E0DF91CF914C
:1069D0001F910F911994EF92FF921F93CF93DF9322
:1069E000EC017B01E9A9FAA982E01995E9A9FAA9C4
:1069F00081E0199520E030E045E1B701CE0192DF5A
:106A0000182F882339F09E012D5C3F4F47E1B701D5
:106A1000CE0188DFE9A9FAA980E01995812FDF91DD
:106A2000CF911F91FF90EF900895CF93DF931F9226
:106A3000CDB7DEB79E012F5F3F4F46E473DF8981FC
:106A40000F90DF91CF910895CF93DF931F92CDB731
:106A5000DEB79E012F5F3F4F47E464DF89810F90CF
:106A6000DF91CF91089520E030E048E45BCFCF93F1
:106A7000DF93EC016A817B81D8DF88836A817B8127
:106A8000CE01E2DF89836A817B81CE01ECDF8B87D7
:106A90009E012D5C3F4F6A817B8147E1CE01DF91F2
:106AA000CF9140CFCF93DF93EC016A817B813EDFB2
:106AB000882319F0CE01DBDF81E0DF91CF910895CB
:106AC0008F929F92AF92BF92CF92EF920F93CF93FC
:106AD000DF931F921F92CDB7DEB74C015B012A8373
:106AE0004983F6DEF401B382A282498147A32A8159
:106AF00020A705A3E4A2C3A2C4010F900F90DF91C9
:106B0000CF910F91EF90CF90BF90AF909F908F90CB
:106B1000C9CFFC01628173813BCFCF93DF93EC013E
:106B2000EE85FF85309709F019956A817B81CE014A
:106B3000DF91CF9150CF0F93FC0182819381648FBD
:106B4000458F278F068F9F01245E3F4F4BE3BC018B
:106B5000CF010F91E7CEFC0160A30895BF92CF92C1
:106B6000DF92EF92FF920F931F93CF93DF936C010D
:106B7000D62FB42EC22F7801CC2369F0F7010491EF
:106B800020E04B2D6D2FC601D6DFFFEFEF1AFF0A75
:106B9000C150D85FF1CFDF91CF911F910F91FF903E
:106BA000EF90DF90CF90BF9008958F929F92AF9219
:106BB000BF92CF92DF92EF92FF920F931F93CF93EA
:106BC000DF935C01C62EC42FD22ED02F220F220FAE
:106BD000220F1ED0882379F0DC0F8D2C912CCD173D
:106BE00051F087012D2D4C2F6C2DC501B7DFE80C1E
:106BF000F91CCF5FF4CFDF91CF911F910F91FF90E0
:106C0000EF90DF90CF90BF90AF909F908F900895BE
:106C10000F93FC010150040F84A996A9941718F052
:106C2000081728F402C0081750F0041740F4215048
:106C3000260F83A995A9961720F4281720F480E041
:106C400007C0281720F481E0261710F0F8CF81E064
:106C50000F91089581E008952EE93FE0009729F013
:106C6000F9013197F1F70197F9CF0895FC011282EC
:106C700080818150838314820895FC0180819281F8
:106C8000980F92832181921760F494819F5F94837F
:106C90009381890F821710F08FEF820F838381E039
:106CA000089580E00895FC0191E08381861708F43F
:106CB00090E031E0461708F030E0832F892B21E087
:106CC0005281451708F420E02823832F8923822B43
:106CD0000895DC01FB01108212968C91129781833A
:106CE00015968C9115978150828313968C9183838E
:106CF0000895FB0141812381213029F0233031F4B3
:106D000068EF640F04C0642F485F01C0642FCBCFCD
:106D1000DC0115962C9115971696ED91FC9117971D
:106D2000CF01820F911D820F911D1192E817F90773
:106D3000E1F70895FC01A681B7818281481B858116
:106D4000483018F0A80FB11D4770382F369536958A
:106D50003695562F577080E890E002C0959587953C
:106D60005A95E2F7439F402D1124669566956695E6
:106D7000E62FF0E0E40FF11DEA0FFB1F3081222324
:106D800011F0832B02C08095832380830895FB013B
:106D90004181DC0112962C911297421760F01396F4
:106DA0002C911397241738F0608115962C91621757
:106DB00010F42481BFCF0895CF92DF92FF920F93FA
:106DC0001F93CF93DF936C01EB01FA809B8191308D
:106DD00051F030F0923049F0933051F41FEF09C078
:106DE00010E001E007C011E004C010E00FEF02C0A6
:106DF00010E000E0F7FE03C0BE01C601C8DF9881C5
:106E0000900F98839981910F9983FF0C99F7DF91E7
:106E1000CF911F910F91FF90DF90CF9008950F9326
:106E20001F93CF93DF938901FB01C281D38142334A
:106E3000D9F058F44531E1F0473109F1443141F5D9
:106E4000CE0166DFCE0112DF23C04634E1F04734C5
:106E5000E1F04B33E9F4B901CE014BDF8823C1F0F7
:106E6000B801CE01A9DF14C0B901CE0190DF10C076
:106E7000CE0103DF882369F0CE014ADF09C0B901E2
:106E8000CE0127DF05C08D8101C08981F801808393
:106E900081E0DF91CF911F910F910895CF92DF9202
:106EA000EF92FF920F931F93CF93DF937C01D62F26
:106EB000D42EC22F122FC62EC20E6C2D611B18307D
:106EC00038F00FEF20E04D2DC70135DE1850F5CF1B
:106ED0006C2F687F6D0F2C2F277071F097E029279A
:106EE0002F5F27700FEF10E001C0000F2A95EAF71F
:106EF00020E04D2DC7011FDEDF91CF911F910F9133
:106F0000FF90EF90DF90CF900895CF92DF92EF92B5
:106F1000FF920F931F93CF93DF937C01D62ED42F34
:106F2000C22F122FC42EC20E4C2D411B183038F028
:106F30000FEF21E06D2DC701FEDD1850F5CF4C2F6E
:106F4000487F4D0F2C2F277071F097E029272F5F76
:106F500027700FEF10E001C0000F2A95EAF721E03B
:106F60006D2DC701E8DDDF91CF911F910F91FF904B
:106F7000EF90DF90CF900895EF92FF920F931F93C1
:106F8000CF93DF93EC01162FF42EE22E01E040DECA
:106F9000882359F02E2D4F2D612FCE01DF91CF91F7
:106FA0001F910F91FF90EF9079CFDF91CF911F91BB
:106FB0000F91FF90EF900895EF92FF920F931F9320
:106FC000CF93DF93EC01162FF42EE22E022F21E057
:106FD0001FDE882359F02E2D4F2D612FCE01DF911A
:106FE000CF911F910F91FF90EF908FCFDF91CF91B5
:106FF0001F910F91FF90EF900895DF92EF92FF9213
:107000000F931F93CF93DF937C01162FC42FD22EA3
:10701000D02FFEDD8823F9F02D2D4C2F612FC701D5
:107020003DDF2D2F4C2F612FC7016FDF6FEF6D0DEF
:10703000610F2D2F4C2FC70168DF4FEF4D0F4C0F05
:107040002D2D612FC701DF91CF911F910F91FF90DF
:10705000EF90DF9023CFDF91CF911F910F91FF90A1
:10706000EF90DF900895EF92FF920F931F93CF93CD
:10707000DF937C01D62F122FC42F040F212F4C2F0A
:107080006D2FC7010BDFCF5F0C13F8CFDF91CF91CE
:107090001F910F91FF90EF900895DF92EF92FF9272
:1070A0000F931F93CF93DF93EC01162FF42EE22E54
:1070B000AFDD882329F02E2D4F2D612FCE01D3DF98
:1070C000DF91CF911F910F91FF90EF90DF90089586
:1070D0000895FC01E60FF11D849190E0982F882718
:1070E0003196E4918E0F911D0895FC0184910895CD
:1070F000FCDF882321F0823011F083E0089586E0E0
:10710000089580E00895FC018081089566E0E1CF54
:1071100068E0DFCF0A96FC01849108950B96FC018C
:1071200084910895DC011496ED91FC9115973196A8
:1071300084910895BF92CF92DF92EF92FF920F93C6
:107140001F93CF93DF938C01E62EDC011496CD9133
:10715000DC911597CE01C9DFF82EF8018481958165
:10716000C7DFC82EF1E0FF1203C02FE0B22E02C02D
:10717000BB24BA94D80114968D919C911597CADFBF
:10718000F82EF80184819581C9DFD82ED801149694
:107190008D919C911597BCDFB0E6BE1538F4009731
:1071A00029F0C80FD91F91E6F92E0FC0F80184818C
:1071B0009581ACDFF0E4FE1538F4009729F0C80F94
:1071C000D91F81E4F82E01C06196DE1490F4D80135
:1071D00050961C92509753961C92539754961C921B
:1071E000549751961C92519752961C9280E090E0D1
:1071F00066C0DF1460F38C2D90E0FE0124912F3FD8
:1072000011F4219657C0FE104CC0D80114968D91F0
:107210009C9115976ADF9E012F5F3F4FFE018823E7
:1072200011F08230E1F48491D80153968C935397F6
:10723000F901249154962C935497FE013396E491CE
:107240005096EC935097FE013496E4915196EC934E
:107250005197FE013596E4915296EC9320C08491AB
:10726000982F9F709250D80152969C935297829576
:107270008F7051968C935197F9012491822F8F70C2
:1072800054968C93549722952F7053962C93539722
:10729000FE013296E491E295EF705096EC93CE01A8
:1072A0000EC0FE013296E491EB219C012E0F311DA0
:1072B000C20FD31FFD1409F48ACFF3949ECFDF9140
:1072C000CF911F910F91FF90EF90DF90CF90BF90E3
:1072D00008954F925F926F927F929F92AF92BF926A
:1072E000CF92DF92EF92FF920F931F93CF93DF9392
:1072F0001F92CDB7DEB72C01C62E942E622F1ADF57
:107300007C01892B09F43AC0F20184819581F0DE79
:10731000B82EF201138904898189C80E8289981ACE
:10732000D92CD01A212F4D2D6C2DC20171DC882350
:1073300011F1EB0CF11C195F169516951695612E3F
:10734000712CD914C1F03C2D57018A2D8E1981174B
:1073500070F4F501049120E04D2D632FC2013983B3
:10736000EADBFFEFAF1ABF0A3981385FEECFE60CD8
:10737000F71CD394E6CFF201808901C080E00F9022
:10738000DF91CF911F910F91FF90EF90DF90CF9001
:10739000BF90AF909F907F906F905F904F900895B7
:1073A0000F931F93CF93DF9300D0CDB7DEB78C013F
:1073B000DC015596ED91FC9156972B834A836983A6
:1073C00019954A81480F2B816981C8010F900F9050
:1073D0000F90DF91CF911F910F917BCFAF92BF9212
:1073E000DF92EF92FF920F931F93CF93DF931F9241
:1073F0001F92CDB7DEB77C01D62E042FDC01559647
:10740000ED91FC91569729833A831995080F2981AC
:10741000A22E3A81B32E10E0F50121915F012223C3
:1074200039F0402F6D2DC70154DFD80E180FF4CF5F
:10743000812F0F900F90DF91CF911F910F91FF90AF
:10744000EF90DF90BF90AF900895DF92EF92FF92A0
:107450000F931F93CF93DF937C01D62FD42E8901F6
:10746000DC015596ED91FC9156971995D80EC0E028
:10747000F8012491222349F04D2D6D2FC70129DFFA
:10748000D80FC80F0F5F1F4FF3CF8C2FDF91CF9115
:107490001F910F91FF90EF90DF900895DC011496FB
:1074A0002D913C9115972115310509F43FC0579650
:1074B0008C915797F901811108C03596E49158963F
:1074C000EC935897F9013C9611C0813041F43F96F6
:1074D000E4915896EC935897F901709607C03D9641
:1074E000E4915896EC935897F9013E96E491599699
:1074F000EC93599758968C915897082E000C990B3D
:1075000059962C915997821B910927FD93955A966C
:107510002C915A97203441F0829FC001112426E01B
:10752000969587952A95E1F75B968C93089521E8C7
:1075300038E3FC01368B258B0895CF92DF92EF92D2
:10754000FF920F931F93CF93DF938C017B016A010E
:10755000CB01FA011995D82F882311F1682FC801A2
:10756000E9DDF801C189C195FFEFEF1AFF0AC701F4
:10757000F6011995F801882351F08089C80FC701D9
:10758000F6011995D82F682FC801D4DDEDCFD03280
:1075900021F091898389890F01C080898C0F01C0F6
:1075A00080E0DF91CF911F910F91FF90EF90DF90DE
:1075B000CF90089543E858E3C0CFCF93DF93FC0109
:1075C000248135812617370741F0EC0175836483E8
:1075D00065DF81E898E39E8B8D8BDF91CF910895D5
:1075E000CF93DF9300D01F92CDB7DEB76115710541
:1075F0008105910579F09B01AC0169833A834B8346
:107600005C830F94765F29813A814B815C810F9472
:10761000CB5E03C060E070E0CB010F900F900F9045
:107620000F90DF91CF910895CF92DF92EF92FF926A
:107630000F931F9362177307840795077CF48901E2
:107640009A016B017C01C901B8016C197D098E0991
:107650009F09C6DF6C0D7D1D8E1D9F1D1F910F9113
:10766000FF90EF90DF90CF9008954F925F926F92CE
:107670007F92AF92BF92CF92DF92EF92FF920F93E1
:107680001F93CF93DF93CDB7DEB729013A019B015A
:10769000AC0124193509460957098A899B89AC89A7
:1076A000BD89BC01CD016A197B098C099D090F9424
:1076B000675EA801970124193509460957090F94F7
:1076C000CB5ECA01B9016A0D7B1D8C1D9D1DDF912A
:1076D000CF911F910F91FF90EF90DF90CF90BF90CF
:1076E000AF907F906F905F904F90089580E090E012
:1076F00008950895CF92DF92EF92FF920F931F9318
:10770000CF93DF936C017A018B01C0E0D0E0CE15FE
:10771000DF0589F0D8016D918D01D601ED91FC91C5
:107720000190F081E02DC6011995892B11F47E019D
:1077300002C02196ECCFC701DF91CF911F910F912D
:10774000FF90EF90DF90CF9008956115710579F06B
:10775000FB0101900020E9F73197AF01461B570B61
:10776000DC01ED91FC910280F381E02D199480E021
:1077700090E00895EACFDC01ED91FC910190F08159
:10778000E02D19944F925F926F927F92EF92FF9249
:107790000F931F93CF93DF93CDB7DEB7A1970FB6AB
:1077A000F894DEBF0FBECDBF7C01FA01CB0119A258
:1077B000223008F42AE08E010F5D1F4F422E512C1B
:1077C000612C712CBF01A30192010F94A95EF901F4
:1077D000CA01015011096A3014F4605D01C0695C8E
:1077E000D8016C93232B242B252B61F7B801C701FB
:1077F000ACDFA1960FB6F894DEBF0FBECDBFDF9110
:10780000CF911F910F91FF90EF907F906F905F90BD
:107810004F900895CF92DF92EF92FF920F931F93B4
:10782000CF93DF93EC016A017B012115310579F4D7
:10783000E881F9810190F081E02D642FDF91CF91F3
:107840001F910F91FF90EF90DF90CF9019942A3005
:107850003105D9F477FF18C06DE28DDF8C01442724
:107860005527BA014C195D096E097F092AE0CE013E
:1078700089DF800F911FDF91CF911F910F91FF90B2
:10788000EF90DF90CF9008952AE0B701A601CE01D6
:10789000DF91CF911F910F91FF90EF90DF90CF90EC
:1078A00071CF9A01AB01770F660B770BB3CFCF93F4
:1078B000CFB7F8948091F303811127C0E6ECF3E091
:1078C0008491E0E8F3E09491E82FF0E0EE0FFF1FE1
:1078D000E55FFB4FA591B491EC91E92321F461E0C0
:1078E00085E30E94B73261E085E30E947B328CB56C
:1078F00080618CBD8CB580648CBD61E084E30E94A6
:107900007B3261E083E30E947B328091F3038F5FDF
:107910008093F303CFBFCF910895CF92EF920F934F
:10792000FC0113AE14AE15AE0496CAD80F91EF90B9
:10793000CF9008958EBD00000DB407FEFDCF8EB52B
:10794000089580E090E0089508950E94FC30FCDFE7
:107950000F94C859C0E0D0E00F945B5A2097E1F330
:107960000E940000F9CFCF93DF931F92CDB7DEB70F
:107970009091FA03292F2370233041F09160926097
:107980009093FA0389830E94034B89810F90DF91C2
:10799000CF910C94114B8091FA03982F93709130F2
:1079A00031F081608D7F8093FA030C940A4B089527
:1079B000CF93DF93EC018991882319F00E94114B3A
:1079C000FACFDF91CF9108950F931F93CF938C013E
:1079D000C62FF80181918F01882331F0CC2321F04B
:1079E0000E94114BC150F5CFCF911F910F91089577
:1079F000CF93DF93FC018491EF012196882321F03E
:107A00000E94114BFE01F7CFDF91CF9108950F93A4
:107A10001F93CF93DF93CDB7DEB727970FB6F894B8
:107A2000DEBF0FBECDBF6330B1F038F46130B1F0CE
:107A3000623049F52FEA36E113C0653031F040F08D
:107A4000663009F52FEB36E10BC02BEB36E108C0B1
:107A500027EB36E105C023EB36E102C02BEA36E125
:107A60009F938F933F932F938E010F5F1F4F1F9311
:107A70000F930F942064C8019BDF0F900F900F901D
:107A80000F900F900F9027960FB6F894DEBF0FBEA1
:107A9000CDBFDF91CF911F910F9108951F93CF9389
:107AA000DF931F92CDB7DEB7182F811102C080E29D
:107AB00001C084E2611102C090E001C092E0892B14
:107AC000698351DF9091FA0310FB92F9892F698144
:107AD00060FB83F98093FA030F90DF91CF911F91A0
:107AE00008956091FA0362FB992790F9891721F0B4
:107AF00063FB662760F9D2CF0895CF93C82F81E04A
:107B0000F0DFC11102C082E001C083E02CDF909160
:107B1000FA03C0FB94F99093FA03CF9108959091E2
:107B2000FA03929591708913E8CF0895CF93C82FE7
:107B300080E0D7DF8C2F8F738068CF9114CFCF93E5
:107B4000C82F80E0CEDF8C2F8F738064CF910BCF56
:107B50001F93CF93DF931F92CDB7DEB7182F81E02D
:107B60006983BFDF6981862F8068FDDE812F8F707A
:107B700080680F90DF91CF911F91F5CE80E0B1DF4B
:107B800081E0F1DE6FE070E080E090E00C94B830CE
:107B9000CF93DF93C0E06C2F80E0DADFFCDED1E131
:107BA000D15039F080E00E94114B80E00E94114BCF
:107BB000F7CFCF5FC03279F7DF91CF910895CF92A1
:107BC000DF92EF92FF921F93CF93DF931F921F924A
:107BD000CDB7DEB769837A83B2DFDDDE6981C62E79
:107BE0007A81D72E11E1115069F0F601E590F490F9
:107BF0008F2D0E94114B8E2D0E94114B82E0C80EDA
:107C0000D11CF1CF0F900F90DF91CF911F91FF907A
:107C1000EF90DF90CF900895CF92DF92EF92FF9296
:107C20000F931F93CF93DF931F92CDB7DEB7982F9B
:107C3000623010F06250985FC62EC29480EFC82266
:107C40008A01D12C6D2D6C0D892F998381DFA3DEE4
:107C5000F801E590F4908F2D0E94114B8E2D0E941B
:107C6000114BD3940E5F1F4F998180E1D812EACF58
:107C70000F90DF91CF911F910F91FF90EF90DF90C8
:107C8000CF900895CF92DF92EF92FF920F931F93C0
:107C9000CF93DF93C42E623010F06250805F982F34
:107CA0009170D92EC82FC695D62FD295D07F83EA52
:107CB000E82E87E1F82E01E0F7011491602F6D0F97
:107CC0008C2F46DF68DECC2059F0D11002C0812F06
:107CD00001C080E00E94114BDD2029F0812F04C0FB
:107CE00080E00E94114B80E00E94114B0F5FFFEF7C
:107CF000EF1AFF0A053001F7DF91CF911F910F9125
:107D0000FF90EF90DF90CF9008958F929F92AF9267
:107D1000BF92DF92EF92FF920F931F93CF93DF9367
:107D2000D82E69E10F94765E20E1929FC001112464
:107D300069E170E00F94965E80E090E85C0102C01B
:107D4000B594A7946A95E2F711E0ED2CF12C612F20
:107D50008CE0FEDE20DE20E030E000E0490189E139
:107D6000880E911CE814F90434F42E153F0534F004
:107D7000C0E0D0E004C0CFEFDFEF01C0E50111307B
:107D800051F01D3041F0033011F4C16006C0011103
:107D900004C0D06802C0CFEFDFEF8D2F0E94114BDF
:107DA0008C2F0E94114B0F5F940124363105B1F6E0
:107DB0001F5F1E3061F68CE0B9DEEDDD80E20E94CF
:107DC000114B29E02D1530F464E0C70120DE88EA6C
:107DD00096E105C063E0C7011ADE84EA96E1DF910F
:107DE000CF911F910F91FF90EF90DF90BF90AF90D8
:107DF0009F908F90FDCDCF93C82F85E097DECBDD90
:107E0000C11102C0C6E001C0C4E080E00E94114B75
:107E10008C2FCF910C94114B80E081DE63E477E1ED
:107E200080E090E0CCDE63E277E180E190E0C7DEC5
:107E300063E077E180E290E0C2DE63EE76E180E32A
:107E400090E0BDDE43E857E160E080E0E5DE43E638
:107E500057E161E080E0E0DE43EC56E161E085E07F
:107E6000DBDE80E0C8CF1F93CF93DF931F92CDB7A7
:107E7000DEB7182F80E1698359DE8DDD69816623C5
:107E800051F0111102C012E001C010E080E00E9428
:107E9000114B812F04C080E20E94114B80E20F90B1
:107EA000DF91CF911F910C94114BCF92DF92EF9203
:107EB000FF920F93CF93DF93C82F6B017A01D22FDC
:107EC000813049F028F0823049F0833039F008C021
:107ED00081E02CDE05C081E129DE02C089E026DEDA
:107EE0005ADD63E0C60193DDDD2349F08AE10E949B
:107EF000114B63E0C7018BDD011106C015C00023E3
:107F000099F08FE996E174DD41E04D276C2F85E013
:107F1000B9DE4D2F6C2F89E0DF91CF910F91FF904B
:107F2000EF90DF90CF90AECEDF91CF910F91FF9089
:107F3000EF90DF90CF9008950F93CF936115710567
:107F400089F0C1E0681779073CF49C01261B370BC8
:107F50002330310544F406C09B01281B390B233024
:107F600031050CF4C0E02091140221702C1711F09F
:107F700001E001C0042F2C2FAB01BC0180E095DF94
:107F800080911402C0FB80F980931402CF910F916D
:107F900008950F93CF936115710589F0C1E06817BB
:107FA00079073CF49C01261B370B2330310544F440
:107FB00006C09B01281B390B233031050CF4C0E0AF
:107FC0002091140222FB222720F92C1711F001E046
:107FD00001C0042F2C2FAB01BC0181E066DF809132
:107FE0001402C0FB82F980931402CF910F9108957F
:107FF000CF93C82F86E09ADDCEDC63E08C2F90E033
:1080000006DD85E2CF910C94114BCF92DF92EF9277
:10801000FF920F931F93CF93DF93CDB7DEB72797D0
:108020000FB6F894DEBF0FBECDBF8C0188E07EDDB9
:10803000F80160817181828193812CE3C22ED12C61
:10804000E12CF12CA70196010F94A95ECA01B90198
:10805000A70196010F94A95E8E010F5F1F4F243672
:10806000310598F47F936F933F932F9385E996E1C1
:108070009F938F931F930F930F9420640FB6F894E0
:10808000DEBF0FBECDBF85E012C07F936F933F93DD
:108090002F938DE896E19F938F931F930F930F94E7
:1080A00020640FB6F894DEBF0FBECDBF86E0F801A6
:1080B000E80FF11D80E280836EDC66E0C80184DC9D
:1080C00027960FB6F894DEBF0FBECDBFDF91CF91DC
:1080D0001F910F91FF90EF90DF90CF900895CF9375
:1080E000DF93EC0186E122DD56DC63E0CE018FDC1C
:1080F00085E2DF91CF910C94114B1F93CF93DF93C7
:108100001F92CDB7DEB788E111DD45DC86E496E04D
:108110000E945584182F813150F486E496E048DCA3
:108120001031F9F080E20E94114B1F5FF9CFCE01B0
:1081300001960E94F78760E147DC8981803178F4FD
:108140008EE20E94114B19811F3049F08EE20E948D
:10815000114B6EE0611B19F086E496E035DC0E945D
:10816000D9870F90DF91CF911F9108950E94948637
:108170006091AC0C90913D024091B60C5091B70CBF
:1081800020916802309169022427352740918D0C97
:1081900050918E0C24273527969FA0011124440F5F
:1081A000452F441F550B51952427A9014827CA0183
:1081B0002091F8033091F9032817390731F0909393
:1081C000F9038093F80381E0089580E008954F92C9
:1081D0005F926F927F928F929F92AF92BF92CF9257
:1081E000DF92EF92FF921F93CF93DF9300D01F9205
:1081F000CDB7DEB7F82E811104C0B8DF882309F4AB
:1082000067C00E949486182F0F940D5669837A8355
:108210008B839C83A0906802B09069026091890C66
:1082200070918A0C80918B0C90918C0C0F94CE5B8A
:108230002B013C01C0908D0CD0908E0C8090B60C20
:108240009090B70C6091B20C7091B30C8091B40C0B
:108250009091B50C0F94CE5BDC01CB014F2DB40196
:108260006BDE4F2DB601C20194DE2091AC0CE22EE4
:10827000F12C11110DC090913D0297FD09C0929F04
:10828000900111247901EE0CEF2CEE1CFF08F19403
:1082900024E62E9DC0012F9D900D112481589F4FE3
:1082A0006FEF70E00F94965E862FA2DECE010196EE
:1082B000ACDEC50114DFEF2811F0812F9CDD61E0F9
:1082C0001C141D041CF060E080E001C0812FCBDD98
:1082D0000F900F900F900F90DF91CF911F91FF9013
:1082E000EF90DF90CF90BF90AF909F908F907F9056
:1082F0006F905F904F900895E6E4F6E090E08191F2
:10830000882311F09827FBCF81E02091F7032913F0
:1083100002C080E008959093F70308950E94948628
:10832000982F81E02091F603291302C080E0089580
:108330009093F6030895811107C0DEDF811104C018
:10834000EDDF882329F0D9CE10928A06D6DEE6CF5B
:108350000895CF93C82F0E94C58BC11104C090917E
:10836000F503981721F08093F503CF91CECCCF91F0
:108370000895CF93C82F0E94FD4A8091FA038E7F03
:108380008093FA038C2F23DF8C2FD5DF8C2FE1DF36
:108390000E94FD4A8091FA038E7F8093FA03CF9169
:1083A000089561E081E07ADB61E081E077DB80E0E5
:1083B000A4CB0E94FD4A8091FA038E7F8093FA033A
:1083C000F0DFDCDBE5DB28DD81E0D3DF0E94FD4A66
:1083D0008091FA038E7F8093FA0308950E94FD4AEC
:1083E0008091FA038E7F8093FA03C8DB61E081E01D
:1083F00055DB0E94FD4A8091FA038E7F8093FA0339
:1084000008950E94FD4A8091FA038E7F8093FA03BB
:10841000C8DFB4DB61E081E041DB0E94FD4A80916E
:10842000FA038E7F8093FA03089580E0A2CF9091A3
:10843000F403981729F08093F4038111BACFCECFBB
:108440000895E8E0F4E083AF64AF08954AE050E0B7
:10845000BC0188E094E025CAEF92FF920F931F932E
:10846000CF93DF937A016F3F71058105910509F084
:1084700048F488E094E07FD98CE094E00E94923840
:1084800090E014C0C0914304D09144044D2F50E0BB
:10849000EC2FF0E08B019C01BF018CE094E0AED1A9
:1084A000C80FC0934304D09344049927DF91CF9120
:1084B0001F910F91FF90EF900895EF92FF920F930D
:1084C0001F93CF93DF938B01C8E0D4E0FBACECACFF
:1084D0004E2D50E06F2D70E09C018CE094E0E6D1D1
:1084E000F80EFBAEECAE9927DF91CF911F910F9163
:1084F000FF90EF900895EF92FF920F931F93CF9309
:10850000DF938B01C8E0D4E0FBACECAC4E2D50E027
:108510006F2D70E09C018CE094E014D2F80EFBAE5D
:10852000ECAE9927DF91CF911F910F91FF90EF90C3
:1085300008950F931F93CF93DF93CDB7DEB728979E
:108540000FB6F894DEBF0FBECDBF8A0123E0660FE1
:10855000771F2A95E1F7680F791F48E050E0CE01B8
:1085600001960F94546329813A81F80180819181A9
:108570002817390790F08217930760F09C81828159
:10858000981758F081E090E03B812381231738F061
:1085900080E005C081E090E002C08FEF9FEF289659
:1085A0000FB6F894DEBF0FBECDBFDF91CF911F9104
:1085B0000F910895EF92FF920F931F93CF93DF9344
:1085C000EC018B017A018A859B858617970731F02C
:1085D000888199810E94DD3A1B870A878885998561
:1085E000019689F00E811F81B701888199810E94CF
:1085F000DA3A080F111D888599858017910718F4BC
:1086000081E090E011C06E818A81680F97014C81F2
:10861000888199810E94EE392E813F81280F311D7A
:108620003F832E8380E090E0DF91CF911F910F91E7
:10863000FF90EF9008954F925F926F927F928F928A
:108640009F92AF92BF92CF92DF92EF92FF920F93E1
:108650001F93CF93DF93CDB7DEB72D970FB6F89466
:10866000DEBF0FBECDBF6C012A013B01490158019D
:108670001B861C86CE0101967C0188E0F7011192D1
:108680008A95E9F7DB01CA0127E0B695A79597958A
:1086900087952A95D1F79A838983F42FFF77FD87F1
:1086A0008F2F80588B838C831A8619864F3F5105F4
:1086B0006105710509F018F460E070E026C0609172
:1086C000FD037091FE038E01075F1F4F970149E97B
:1086D00052E48091FB039091FC030E94A68297FDD7
:1086E000EBCF69857A8583E0660F771F8A95E1F77E
:1086F0008091FB039091FC03680F791F48E050E0E4
:10870000C7010F9454636F8178856115710519F461
:108710004B86B60106C0C616D70619F08D8580684F
:108720008B87AE01455F5F4FC401F50119952D960A
:108730000FB6F894DEBF0FBECDBFDF91CF911F9172
:108740000F91FF90EF90DF90CF90BF90AF909F90F0
:108750008F907F906F905F904F9008956F927F926F
:108760008F929F92AF92BF92CF92DF92EF92FF9241
:108770000F931F93CF93DF9300D01F92CDB7DEB737
:108780006C017B013A015901480119821A821B824E
:108790001C82AE014F5F5F4FB301C7010E94068389
:1087A0007C0149815A816B817C81411551056105AC
:1087B000710529F084019501C6013DDFE6CF0F90D8
:1087C0000F900F900F90DF91CF911F910F91FF901D
:1087D000EF90DF90CF90BF90AF909F908F907F9061
:1087E0006F90089521E02093FF03EBEFF3E0918376
:1087F00080837383628380E090E008957F92AF92DC
:10880000BF92CF92DF92EF92FF920F931F93CF937D
:10881000DF93CDB7DEB72C970FB6F894DEBF0FBE4F
:10882000CDBF6C01762EF72F842FE52FB901A8015B
:10883000D6011496AD90BC9015979091FF039111BD
:108840000AC027EE37E1482F672DC6010E94253A5E
:1088500080E090E019C0DA82C9827B82FC838D833C
:10886000EE8318861F82FA86E9861C861B860AED2F
:1088700012E49E012F5F3F4FC501DDDEB501C60149
:108880000E94DD3A8F8198852C960FB6F894DEBF52
:108890000FBECDBFDF91CF911F910F91FF90EF9051
:1088A000DF90CF90BF90AF907F900895CF92DF92EE
:1088B000EF92FF920F931F93CF93DF93CDB7DEB765
:1088C0002C970FB6F894DEBF0FBECDBF7C01C90157
:1088D000F701C480D5802091FF03211108C027EC47
:1088E00037E1C7010E94253A80E090E01CC0FA827F
:1088F000E9826B837C834D835E8318861F821A878F
:1089000009871C861B860AED12E49E012F5F3F4FEC
:1089100040EA52E8BC01C60121DFB601C7010E944E
:10892000DD3A8F8198852C960FB6F894DEBF0FBE86
:10893000CDBFDF91CF911F910F91FF90EF90DF900E
:10894000CF900895CF92DF92EF92FF920F931F93F3
:10895000CF93DF93CDB7DEB72C970FB6F894DEBF79
:108960000FBECDBF7C01C901F701C480D580209125
:10897000FF03211108C027EA37E1C7010E94253A09
:1089800080E090E01CC0FA82E9826B837C834D8397
:108990005E8318861F821A8709871C861B860AED4C
:1089A00012E49E012F5F3F4F43EA52E8BC01C6012B
:1089B000D5DEB601C7010E94DD3A8F8198852C96DD
:1089C0000FB6F894DEBF0FBECDBFDF91CF911F91E0
:1089D0000F91FF90EF90DF90CF900895CF93DF93AA
:1089E000EC01262F4CAD6BAD04960E94D0392BAD17
:1089F000082E000C990B820F911D8BAF81E090E047
:108A0000DF91CF9108950F939CE0899F802D1124D1
:108A100021E0280F20930704845F8093060490E0F0
:108A200002964091400450E08417950714F480E0CA
:108A300033C0822F90E02091420430E082179307E8
:108A4000B4F76623A9F061E08CE094E00E94AB35B6
:108A5000409107044E5F0BE020E860E08CE094E07A
:108A60000E944D3860E08CE094E00E94AB3505C078
:108A700061E08CE094E00E94AB3560910604809147
:108A800040046817A0F2909107048091420489176E
:108A900070F280E0D6DC81E00F910895CF93DF93F0
:108AA000FC0185ADEF012496811105C081E085AF01
:108AB000CE010E945235CE01DF91CF910C948935C1
:108AC000CF93DF93EA01BDDC6FEF7FEFCE01DF9143
:108AD000CF9111CD6FEF7FEFF0CC4FEF5FEFBCCCBC
:108AE000482F50E020910504022E000C330B421752
:108AF000530781F080930504813031F462EA7EE10E
:108B00008CE094E00C94DD3A60EF78E18CE094E046
:108B10000C94DD3A089581E0089588E094E0BEDF8A
:108B200080E00E947EA58CE094E00E948D3581114A
:108B3000F7CF64EC79E080E090E00C94D6A5EF925A
:108B4000FF920F9380914504811107C081E08093CB
:108B500045048CE094E00E9452358CE094E00E9441
:108B600089358DE1E82E8EE1F82E03E127E047E01C
:108B700064E28CE094E00E94D53583E0B1DF47E306
:108B800058E16BE285E29CDF43E258E167E387E06E
:108B900097DF8CE094E00E948D358111E2CF0F9138
:108BA000FF90EF90089581E0CADF64EC79E080E007
:108BB00090E00C94D6A5B1DFF6CF60E070E082EAD9
:108BC0009EE110CE1F93CF93DF931BDCC0910D0469
:108BD000C695C69588E094E061DFDC2FDD0F1D2F80
:108BE0001C0F83E07DDF6C2F80E02BDC86E496E0B9
:108BF00071DF44E158E16D2F80E062DF47E058E12A
:108C0000612F80E05DDF8CE094E00E948D35811162
:108C1000E8CFDF91CF911F9108950895CF93E62F6C
:108C20006CE0869F602D112481E0860F80930704FD
:108C3000645F60930604462F50E04E5F5F4F2091C3
:108C4000400430E0421753070CF445C090E02091F7
:108C5000420430E0821793070CF03DC0CE2F8EE324
:108C6000F0DB65E470E080E090E037DF61E36C0FFB
:108C7000062E000C770B880B990B2FDF60E270E05B
:108C800080E090E02ADF6091B20C7091B30C80918B
:108C9000B40C9091B50C0F94CE5BCB010F94245083
:108CA00019DF6FE270E080E090E017DF0E949486A9
:108CB000811109C085E0C89FF0011124E456F34FEB
:108CC0008481811108C08091B60C9091B70C0F94EB
:108CD0002450CF91FFCECF910895CF92DF92EF92A3
:108CE000FF920F931F93CF93DF931F921F92CDB7E5
:108CF000DEB77B01622F498386DE4981882309F430
:108D000040C0442309F101151105F1F4C7010E9487
:108D1000768425E130E0281B310937FF02C02F5F40
:108D20003F4F3595279530E82158822F830F87FDD7
:108D30000CC060E270E080E090E02A833983CDDEF1
:108D4000398131502A81F1CF30E8C32ED12CB601C0
:108D5000C701D1DB7601E81AF90A0115110511F4F2
:108D60001E2D06C0FF24B701C801A7DB1E2D181B4E
:108D7000173038F060E270E080E090E0AEDE181B63
:108D8000F7CF0F900F90DF91CF911F910F91FF9030
:108D9000EF90DF90CF9008950F93CF93DF93982FAC
:108DA000862FEA01692F2FDE882309F162E770E040
:108DB000CE01A1DBC2E7C81BC73038F060E270E02B
:108DC00080E090E08ADEC81BF7CF609106048AE756
:108DD00038DB602F000F770B880B990B7EDE60E28B
:108DE00070E080E090E0DF91CF910F9176CEDF913F
:108DF000CF910F910895CF92DF92EF92FF920F9350
:108E00001F93CF93DF93982F862F6A017901692FE3
:108E1000FADD882309F445C0C701002321F00E9430
:108E20007684182F03C00E945584182FC3E1D0E028
:108E3000C11BD1098C2F880FC80FCC0FD0E0BE0109
:108E4000C60159DBC81B6AE370E080E090E045DEB4
:108E5000C73038F060E270E080E090E03EDEC81B92
:108E6000F7CF8AEF189F802D112460910604805857
:108E7000E8DA002361F06FEF7FEFC701DF91CF9158
:108E80001F910F91FF90EF90DF90CF9034CBC701EF
:108E9000DF91CF911F910F91FF90EF90DF90CF90D6
:108EA00019CEDF91CF911F910F91FF90EF90DF903E
:108EB000CF900895BF92CF92DF92EF92FF920F93DF
:108EC0001F93CF93DF936C017B010E947684C82FA0
:108ED000C7010E94558403E110E0081B11098C2F83
:108EE00090E0BB24B394081719071CF0B12CC5E21D
:108EF00001C0CFE12C2F30E0A9014E5F5F4F809180
:108F0000400490E04817590744F029503109609116
:108F1000420470E0621773079CF5D0E0E114F1049D
:108F2000A9F16AE370E080E090E0D7DDBB2081F03A
:108F3000C45F80914004C81748F12C2F30E02950BD
:108F400031098091420490E0821793071CF41EC0FF
:108F5000DD23E1F0802F880F800F6C2F880F71DAEE
:108F600060E270E080E090E0B8DDC701DF91CF9172
:108F70001F910F91FF90EF90DF90CF90BF90AACDFF
:108F8000A6016C2F80E09CDDD1E0C8CFDF91CF91AE
:108F90001F910F91FF90EF90DF90CF90BF900895B9
:108FA000CF92DF92EF92FF920F931F93CF93DF93B5
:108FB0001F92CDB7DEB7182F7A01D22ECA0169836E
:108FC0000E947684082F812F880F810FC82ECC0C29
:108FD0001CE06981169F100D1124DD20C1F061E0B5
:108FE0008CE094E00E94AB35202F220F200F220F3F
:108FF0002E5F0BE047EF410F6FEF6C0D8CE094E0BC
:109000000E944D3860E08CE094E00E94AB35A701EF
:10901000612F8C2D55DDDD2071F061E08CE094E056
:109020000F90DF91CF911F910F91FF90EF90DF9004
:10903000CF900C94AB350F90DF91CF911F910F9192
:10904000FF90EF90DF90CF900895AF92BF92DF92A4
:10905000EF92FF920F931F93CF93DF93EC015B018D
:10906000D42EC901B801A7010E94258691E02D2DBB
:109070002927A50164E081E093DFCE010E94768478
:109080002D2DAE0164E094E1981B892FDF91CF91E3
:109090001F910F91FF90EF90DF90BF90AF9080CF26
:1090A000EF92FF920F93CF93DF93D82FC62F7901C2
:1090B000682F8C2FA8DC8823D9F0002329F062E0E8
:1090C00070E080E090E009DD2D2F4C2F64E1C701B6
:1090D0000E94018568E770E0F0D9C8E7C81BC73077
:1090E00038F060E270E080E090E0F7DCC81BF7CF7A
:1090F000DF91CF910F91FF90EF9008958F929F9203
:10910000AF92BF92CF92DF92EF92FF920F936B01DB
:109110007C018090010490900204A0900304B09020
:109120000404A50194010F945F5B882301F120E002
:1091300030E0A901C701B6010F945F5B882351F0AD
:10914000A5019401C701B6010F945F5B87FD04C0C0
:1091500081E003C080E001C08FEF80930004C092E3
:109160000104D0920204E0920304F092040480917E
:109170004004813128F480914204833008F048C0D3
:1091800080914004853128F480914204843108F0B4
:109190004FC0809140048F3308F057C08091420443
:1091A0008F3208F452C08091000440E3481B86E7E8
:1091B000E82E88E1F82E0DE022E06AE58CE094E0EC
:1091C0000E94D5358091000441E3481B9CE5E92EBF
:1091D00098E1F92E22E065E08CE094E00E94D5351C
:1091E00020E9E22E28E1F22E00E123E04FE262E1E5
:1091F0008CE094E00E94D53530ECE32E38E1F32E7C
:1092000023E04FE267E68CE094E00E94D5351DC074
:109210008091000444E0481B51E4E52E58E1F52E0E
:109220000CE022E062E48CE094E00E94D535A8CF07
:1092300049E5E42E48E1F42E01E023E044E16CE34B
:109240008CE094E00E94D535A4CF0F91FF90EF9071
:10925000DF90CF90BF90AF909F908F900895CF9266
:10926000EF920F93CF93DF93C8E0D4E01B821A8272
:1092700084E593E099838883CC24CA94EE24EA940D
:1092800006E427E448E465E172E0CE010E948D3CEB
:1092900080E693E099838883DF91CF910F91EF90DF
:1092A000CF9008959091050194709093030187FDEC
:1092B00076C0A398909105019095947090930301C6
:1092C00090910501947090930301982F990F86FD5A
:1092D00072C0A398809105018095847080930301EA
:1092E00080910501847080930301292F220F96FD40
:1092F00060C0A398809105018095847080930301DC
:1093000080910501847080930301922F990F26FDAF
:109310004EC0A398809105018095847080930301CD
:1093200080910501847080930301292F220F96FDFF
:109330003CC0A398809105018095847080930301BF
:1093400080910501847080930301922F990F26FD6F
:109350002AC0A398809105018095847080930301B1
:1093600080910501847080930301292F220F96FDBF
:1093700018C0A398809105018095847080930301A3
:109380008091050184708093030126FD16C0A39887
:109390008091050180958470809303010895A39ABC
:1093A00089CFA39AE7CFA39AD5CFA39AC3CFA39A85
:1093B000B1CFA39A9FCFA39A8DCFA39A8091050195
:1093C000809584708093030108952F923F925F925D
:1093D0007F929F92AF92BF92CF92DF92EF92FF92D5
:1093E0000F931F93CF93DF937C011B01942E690190
:1093F0008AE0481709F47BC0A5E14A134EC0DB019F
:109400001296ED91FC9113971281C681D781A49A8F
:1094100088E28A950000E9F700EE010F80E1582EFE
:10942000510E98E2792E88EF3DDF872D8A95000056
:10943000E9F7103208F046C0812F8077806832DF6C
:10944000812F8295807F2EDF872D8A950000E9F796
:1094500080E828DF80E026DF872D8A950000E9F785
:109460008AEF20DF872D8A950000E9F75E01B0E1E1
:10947000AB0EB11C8881807F15DF89918295807F3A
:1094800011DFCA15DB05B1F7872D8A950000E9F7D2
:109490001F5F0F5F1511C7CFA4989601492DB10129
:1094A000C701DF91CF911F910F91FF90EF90DF9057
:1094B000CF90BF90AF909F907F905F903F902F9004
:1094C0000C940F37802F80778068ECDE802F829598
:1094D000807FE8DE872D8A950000E9F780E8E2DEEC
:1094E00080E8E0DE872D8A950000E9F7B9CF9C9AE5
:1094F000A4989B9AA39880910401846080930401AE
:10950000809105018095847080930301A49AC8E23C
:109510008C2F8A950000E9F788E790E00E942C36AE
:1095200088EFC0DE8C2F8A950000E9F780E2BADE72
:1095300080E0B8DE8C2F8A950000E9F780E0B2DE8B
:1095400080E8B0DE8C2F8A950000E9F780E0AADE83
:1095500080E1A8DE8C2F8A950000E9F78FE090E08B
:109560000E942C3680E29EDE80E49CDE8C2F8A9561
:109570000000E9F780E296DE80E694DECA950000FE
:10958000E9F710E0D8E208E2812F807780688ADE70
:10959000812F8295807F86DE8D2F8A950000E9F7E6
:1095A00080E880DE80E07EDE8D2F8A950000E9F77E
:1095B0008AEF78DE8D2F8A950000E9F7C0E280E01F
:1095C00071DE80E06FDE9D2F9A950000E9F7C150B3
:1095D000B1F788EF67DE802F8A950000E9F71F5FFB
:1095E000103209F0D1CF80E05DDE80EC5BDE88E2F6
:1095F0008A950000E9F7A49850CFA49A88E28A954A
:109600000000E9F7089588EF4DDE88E28A950000B2
:10961000E9F708958AEF46DE88E28A950000E9F7C7
:109620000895CF93C82F807F3DDE8C2F8295807F59
:1096300039DE88E28A950000E9F7CF910895CF934B
:10964000DF931F921F92CDB7DEB789839A830E9462
:109650006C7F20E040E060E070E089819A810F90AB
:109660000F90DF91CF910C941F800F93CF93DF93D6
:1096700061E081E00E943881D0911406C0E0D111F0
:1096800017C080911306811104C00E944B8581117F
:1096900065C080912302882309F457C081E090912E
:1096A0001306911180E004E024E046EB57E24BC042
:1096B000D130C1F480911306813021F40E944B8592
:1096C000811155C080912302882309F43EC081E0B6
:1096D00090911306913009F080E003E02EE34DEA0B
:1096E00057E231C0D230B9F480911306823021F4B0
:1096F0000E944B85811144C080912302882329F167
:1097000081E090911306923009F080E003E02EE3AF
:1097100044EA57E218C0D330C1F480911306833075
:1097200021F40E944B85811134C08091230288234B
:1097300061F081E090911306933009F080E003E03E
:109740002EE34EE957E26C2F27DBCF5FDF5FC5309A
:1097500009F095CF84E08093120622C081E00E9438
:1097600052808091E005882309F493CF19C08FE3DC
:1097700095E765DF8091E005882309F4A3CF10C049
:1097800081E69AE75CDF8091E005882309F4B4CF95
:1097900007C089E79EE753DF8091E005882329F21F
:1097A000DF91CF910F910895CF93DF93EC01CB011F
:1097B000BA010F94015C23E333E343E250E40F94D6
:1097C0009D5D0F94D35B6883DF91CF910895CF9314
:1097D000DF93EC01CB01BA010F94015C2FE632E17B
:1097E00043E85AE30F949D5D688379838A839B8362
:1097F000DF91CF91089564ED7BE487E09CE40C94C5
:10980000768067EE7BE48AE29CE40C9476800F9489
:10981000015C23E333E343E250E40F949D5D0F9436
:10982000D35B862F0D94794FCF93DF9300D01F9297
:10983000CDB7DEB769837A838B839C8360E2CE01E8
:1098400001960F9462520F900F900F900F90DF913E
:10985000CF9108950F94015C2FE632E143E85AE37B
:109860000F949D5DE1CF2F923F924F925F926F9246
:109870007F928F929F92AF92BF92CF92DF92EF92A0
:10988000FF920F931F93CF93DF93CDB7DEB7299746
:109890000FB6F894DEBF0FBECDBF1C017987688775
:1098A000CA01B901E982FA820B831C83DE82CD8270
:1098B000AF8220E030E04AE754E40F949D5D6B01F5
:1098C0007C0120E030E040E057EC0F94625D181618
:1098D0002CF0C12CD12CE12C27ECF22EC701B601C3
:1098E0000F94CE5B2B013C0120E030E04AE754E4CA
:1098F00069817A818B819C810F949D5D4B015C0114
:1099000020E03EEF4FEF56E40F945F5B87FD07C00A
:10991000812C9EEF992EAA24AA9496E4B92E20E0D9
:1099200030E04AE754E4E885F985608171818281FD
:1099300093810F949D5D6B017C01C301B2010F9473
:10994000015C9B01AC01C701B6010F94855A0F94CD
:10995000D35B69837A838B839C83C501B4010F94A5
:10996000CE5B7B018C01E418F50806091709FF811D
:10997000FF938D809E8081E0A82E8CE4B82EC98054
:10998000DA80A301920168857985C1010E94937FE5
:109990000F9029960FB6F894DEBF0FBECDBFDF91B2
:1099A000CF911F910F91FF90EF90DF90CF90BF90DC
:1099B000AF909F908F907F906F905F904F903F906F
:1099C0002F9008958F929F92AF92BF92CF92DF9285
:1099D000EF92FF920F931F93CF93DF9361E081E0AB
:1099E0000E943881D0911406C0E0D11119C0809135
:1099F0001306811104C00E944B858111C4C080915F
:109A00002302882309F4B6C081E0909113069111D6
:109A100080E004E024E041EF57E26C2FBDD9AAC0FA
:109A2000D130E1F480911306813021F40E944B85FE
:109A30008111B2C080912302882309F49BC011E0F8
:109A400080911306813009F010E08091240C0F946E
:109A5000794F00E09C014BED57E289C0D23009F507
:109A600080911306823021F40E944B858111C3C07E
:109A700080912302882309F47DC011E080911306B0
:109A8000823009F010E06091250C7091260C8091D5
:109A9000270C9091280CC8DE00E09C0147ED57E2AE
:109AA00066C0D33009F580911306833021F40E94FB
:109AB0004B858111B9C080912302882309F45AC0D3
:109AC00011E080911306833009F010E06091290CB9
:109AD00070912A0C80912B0C90912C0CA5DE00E04B
:109AE0009C0143ED57E243C0D43001F58091130649
:109AF000843021F40E944B858111AFC080912302F4
:109B00008823C1F111E080911306843009F010E040
:109B100060912D0C70912E0C80912F0C9091300C37
:109B200083DE00E09C014FEC57E221C0D53011F5F7
:109B300080911306853021F40E944B858111A6C0C7
:109B4000809123028823B1F011E0809113068530C3
:109B500009F010E06091290270912A0280912B0295
:109B600090912C0261DE00E09C014BEB57E26C2FE0
:109B7000812F41D9CF5FDF5FC53009F036CF86E056
:109B8000809312069BC081E00E9452808091E00584
:109B9000882309F434CF92C081E00E94408560910F
:109BA000240C70E080E090E00F94FF5B29EC38EC2F
:109BB00048EC5EE30F949D5D0F94D35B1F92812C64
:109BC000912C4BEFA42E4BE4B42E6B0114E6E12E46
:109BD000F12C00E010E020E030E0A90164E27CE03C
:109BE00086EE97E20E94937F0F908091E005882394
:109BF00009F420CF63C081E00E944085A12CC12CD4
:109C0000D12C16E6E12EFE2C0EE111E420E030E02E
:109C1000A90165E27CE089ED97E225DE8091E0050F
:109C2000882309F425CF4AC081E00E944085A12CF9
:109C3000C12CD12C16E6E12EFE2C0EE111E420E021
:109C400030E0A90169E27CE085ED97E20CDE8091CD
:109C5000E005882309F42FCF31C081E00E944085C0
:109C6000A12CC12CD12C16E6E12EFE2C0EE111E424
:109C700020E030E0A9016DE27CE081ED97E2F3DDC8
:109C80008091E005882309F439CF18C081E00E9453
:109C90004085A12CC12CD12C16E6E12EFE2C0EE124
:109CA00011E420E030E0A90169E272E085EC97E27E
:109CB000DADD8091E005882309F442CFDF91CF916E
:109CC0001F910F91FF90EF90DF90CF90BF90AF90DA
:109CD0009F908F900895CF93DF93EC01CB01BA0151
:109CE0000F94015C2AE037ED43E25CE30F949D5D45
:109CF000688379838A839B83DF91CF910895CF9383
:109D0000DF93EC01CB01BA010F94015C6883798386
:109D10008A839B83DF91CF910895CF93DF93EC01EA
:109D2000CB01BA010F94015C20E030E048EC51E433
:109D30000F949D5D688379838A839B83DF91CF91A4
:109D40000895CF93DF93EC01CB01BA010F94015C2E
:109D5000688379838A839B83DF91CF910895CF9322
:109D6000DF93EC01CB01BA010F94015C20E030E0FD
:109D700048EC51E40F949D5D0F94D35B6883798325
:109D80008A839B83DF91CF910895CF93DF93EC017A
:109D9000CB01BA010F94015C20E030E048EC52E4C2
:109DA0000F949D5D0F94D35B688379838A839B8333
:109DB000DF91CF910895CF93DF93EC01CB01BA01EE
:109DC0000F94015C2AE037ED43E25CE30F949D5D64
:109DD000688379838A839B83DF91CF910895CF93A2
:109DE000DF93EC01CB01BA010F94015C2DEC3CEC4C
:109DF0004CEC5DE30F949D5D688379838A839B833C
:109E0000DF91CF9108956BE67EE488E89FE40C949F
:109E100076806FE77EE486E090E50C94768061EAD8
:109E20007EE487E39FE40C9476806DE87EE485EA27
:109E30009FE40C9476806FEA7EE482E290E50C94D5
:109E4000768065EC7EE482EC9FE40C9476806BED8A
:109E50007EE48EE49FE40C9476806FEE7EE48BE6E5
:109E60009FE40C9476800D94EC0A0D94330BCF9301
:109E7000DF9300D01F92CDB7DEB70F94015C6983EA
:109E80007A838B839C83CE0101960F94A9530F9004
:109E90000F900F900F90DF91CF910895CF93DF93A4
:109EA00000D01F92CDB7DEB70F94015C2AE037EDEA
:109EB00043E25CE30F949D5D69837A838B839C838B
:109EC000CE0101960F94DB530F900F900F900F90DF
:109ED000DF91CF910895CF93DF9300D01F92CDB73C
:109EE000DEB70F94015C2DEC3CEC4CEC5DE30F9481
:109EF0009D5D69837A838B839C83CE0101960F9449
:109F000078540F900F900F900F90DF91CF9108959C
:109F1000CF93DF9300D01F92CDB7DEB70F94015CD3
:109F20002AE037ED43E25CE30F949D5D69837A8319
:109F30008B839C83CE0101960F9424510F900F9038
:109F40000F900F90DF91CF910895CF93DF9300D0C2
:109F50001F92CDB7DEB70F94015C20E030E048ECF3
:109F600051E40F949D5D69837A838B839C83CE013A
:109F700001960F94A9530F900F900F900F90DF91BF
:109F8000CF910895CF93DF9300D01F92CDB7DEB766
:109F90000F94015C20E030E048EC52E40F949D5DAA
:109FA0000F94D35B0F94FF5B69837A838B839C83CD
:109FB000CE0101960F94A9530F900F900F900F9020
:109FC000DF91CF910895CF92DF92EF92FF926B01D4
:109FD0007C0120E030E0A9010F945F5B87FD05C0A4
:109FE00020E030E040E05FE304C020E030E040E00B
:109FF0005FEBC701B6010F94865A0F94CE5BCB017D
:10A00000FF90EF90DF90CF900D9424500F94015C5F
:10A01000DACFCF93DF9300D01F92CDB7DEB70F9486
:10A02000D35B0F94FF5B69837A838B839C83CE0120
:10A0300001960F94A9530F900F900F900F90DF91FE
:10A04000CF9108950F94015C20E030E048EC51E49A
:10A050000F949D5DDECF81E00C9452806F927F92D1
:10A060008F929F92AF92BF92CF92DF92EF92FF9228
:10A070000F931F93CF93DF9300D01F92CDB7DEB71E
:10A0800061E081E00E94388160901406712C6110BB
:10A090001AC080911306811104C00E944B85811162
:10A0A00059C180912302882309F44BC181E090912A
:10A0B0001306911180E004E024E047E859E2672D9F
:10A0C0000E94CC463EC181E068122CC080911306EC
:10A0D000813021F40E944B85811143C1809123027C
:10A0E000882309F42EC111E080911306813009F014
:10A0F00010E080916D0E90916E0EA0916F0EB09158
:10A10000700E89839A83AB83BC83CE0101960F9432
:10A11000A95300E09C014BE759E2672D812F0E9473
:10A12000FB460FC182E068122CC08091130682307A
:10A1300021F40E944B8581114CC180912302882318
:10A1400009F4FFC011E080911306823009F010E09D
:10A150008091710E9091720EA091730EB091740E59
:10A1600089839A83AB83BC83CE0101960F94A95354
:10A1700000E09C0147E659E2672D812F0E94FB46D3
:10A18000E0C083E068122CC080911306833021F474
:10A190000E944B8581114FC180912302882309F4CD
:10A1A000D0C011E080911306833009F010E0809157
:10A1B000750E9091760EA091770EB091780E8983EE
:10A1C0009A83AB83BC83CE0101960F94A95300E020
:10A1D0009C0145E559E2672D812F0E94FB46B1C0E5
:10A1E00084E0681227C080911306843021F40E9415
:10A1F0004B85811158C180912302882309F4A1C0A5
:10A2000011E080911306843009F010E06091390E5E
:10A2100070913A0E80913B0E90913C0E0F94FF5B33
:10A22000F8DE00E09C0147E459E2672D812F0E948F
:10A23000FB4687C085E0681227C0809113068530F1
:10A2400021F40E944B8581116AC1809123028823E9
:10A2500009F477C011E080911306853009F010E011
:10A2600060913D0E70913E0E80913F0E9091400E98
:10A270000F94FF5BCEDE00E09C0149E359E2672DBD
:10A28000812F0E94FB465DC086E0681227C0809146
:10A290001306863021F40E944B8581117CC1809188
:10A2A0002302882309F44DC011E080911306863003
:10A2B00009F010E06091410E7091420E8091430EC2
:10A2C0009091440E0F94FF5BA4DE00E09C014BE2F2
:10A2D00059E2672D812F0E94FB4633C087E0681248
:10A2E00030C080911306873021F40E944B85811184
:10A2F00087C180912302882321F111E08091130608
:10A30000873009F010E06091450E7091460E809103
:10A31000470E9091480E0F94FF5B0F94D35B0F9400
:10A32000FF5B69837A838B839C83CE0101960F94B4
:10A33000A95300E09C014DE159E2672D812F0E9455
:10A34000FB467394639485E07812A1CE88E08093F5
:10A35000120691C180DE8091E005882309F4A1CE28
:10A360008AC181E00E9440852AE037ED43E25DE347
:10A3700060916D0E70916E0E80916F0E9091700EC7
:10A380000F949D5D20E030E040E85FE30F94855A34
:10A390000F94D35B1F92812C912C55E1A52E5FE485
:10A3A000B52E6B0117E7E12E1FE0F12E00E010E063
:10A3B00021E030E040E050E06DE67EE081E899E2A7
:10A3C0000E94937F0F908091E005882309F486CE48
:10A3D00052C181E00E94408520E030E048EC52E428
:10A3E0006091710E7091720E8091730E9091740E47
:10A3F0000F94855A0F94D35B1F92812C912C3FE0D0
:10A40000A32E3FE4B32E6B011BE9E12E1FE7F12ED3
:10A4100000E010E024E630E040E050E061E77EE05C
:10A4200081E799E20E94937F0F908091E005882355
:10A4300009F483CE20C181E00E9440852AE037EDF7
:10A4400043E25DE36091750E7091760E8091770E18
:10A450009091780E0F949D5D20E030E040E85FE33E
:10A460000F94855A0F94D35B1F92812C912C95E108
:10A47000A92E9FE4B92E6B0117E7E12E1FE0F12E04
:10A4800000E010E021E030E040E050E065E77EE0F1
:10A490008EE599E20E94937F0F908091E0058823DA
:10A4A00009F47ACEE8C081E00E9440856091390EBF
:10A4B00070913A0E80913B0E90913C0E0F94FF5B91
:10A4C0002AE037ED43E25DE30F949D5D20E030E04C
:10A4D00040E850E40F94855A0F94D35B1F92B3E386
:10A4E0008B2EBFE49B2E1BE1A12E1FE4B12E6B012E
:10A4F00014E7E12E1FE0F12E00E010E024E030E050
:10A5000040E050E069E37EE08EE499E20E94937FB0
:10A510000F908091E005882309F46DCEACC081E0F6
:10A520000E94408560913D0E70913E0E80913F0EDD
:10A530009091400E0F94FF5B2AE037ED43E25DE31C
:10A540000F949D5D20E030E040E850E40F94855A80
:10A550000F94D35B1F92E3E38E2EEFE49E2EFBE17C
:10A56000AF2EFFE4BF2E6B0114E7E12E1FE0F12EAA
:10A5700000E010E024E030E040E050E06DE37EE0F9
:10A5800080E499E20E94937F0F908091E0058823F8
:10A5900009F45BCE70C081E00E9440856091410E5D
:10A5A0007091420E8091430E9091440E0F94FF5B88
:10A5B0002AE037ED43E25DE30F949D5D0F94D35B9A
:10A5C0001F9233E3832E3FE4932E4BE1A42E4FE4FE
:10A5D000B42E6B0118E7E12E1FE0F12E00E010E031
:10A5E00020E030E0A90161E47EE082E399E20E948C
:10A5F000937F0F908091E005882309F450CE3BC0F3
:10A6000081E00E9440856091450E7091460E8091D8
:10A61000470E9091480E0F94FF5B2AE037ED43E21E
:10A620005CE30F949D5D20E030E040E85FE30F9431
:10A63000855A0F94D35B1F9283E3882E8FE4982E64
:10A6400091E2A92E9FE4B92E6B011DEDE12E13E0DE
:10A65000F12E00E010E021E030E040E050E065E461
:10A660007EE084E299E20E94937F0F908091E00562
:10A67000882309F43ECE0F900F900F900F90DF913A
:10A68000CF911F910F91FF90EF90DF90CF90BF90EF
:10A69000AF909F908F907F906F9008950F931F932E
:10A6A000CF93DF9361E081E00E943881C09114066E
:10A6B000D0E0C1111AC080911306811104C00E941C
:10A6C0004B8581110CC180912302882309F461C05C
:10A6D00081E090911306911180E004E024E04BE5C5
:10A6E00058E26D2F0E94CC4654C0C130D9F48091FD
:10A6F0001306813021F40E944B858111F7C08091AF
:10A700002302882309F445C081E09091130691301B
:10A7100009F080E003E02EE342E558E26D2F0E944D
:10A72000CC4637C0C230D1F480911306823021F478
:10A730000E944B858111E4C080912302882349F156
:10A7400081E090911306923009F080E003E02EE35F
:10A7500045E458E26D2F0E94CC461BC0C330C9F4BB
:10A7600080911306833021F40E944B858111D2C061
:10A7700080912302882369F081E090911306933041
:10A7800009F080E003E02EE340E458E26D2F0E94E0
:10A79000CC460E94088081111DC0C430E9F480912C
:10A7A0001306843021F40E944B858111BDC0809135
:10A7B0002302882309F4C2C081E0909113069430EB
:10A7C00009F080E003E02EE347E358E26D2F0E949A
:10A7D000CC46B4C014E001C015E0C1131BC0809189
:10A7E00013068C1304C00E944B858111A9C080916F
:10A7F0002302882371F081E0909113069C1380E07E
:10A8000003E02EE34EE258E26D2F0E94CC461C2F4F
:10A8100001C01C2F81E0810FC81318C0809113065E
:10A820008C1304C00E944B85811194C08091230237
:10A83000882361F081E0909113069C1380E003E08F
:10A840002EE342E258E26D2F0E94CC4682E0810F57
:10A85000C81318C0809113068C1304C00E944B8546
:10A86000811182C080912302882361F081E0909160
:10A8700013069C1380E003E02EE349E158E26D2FBC
:10A880000E94CC4683E0810FC81320C0809113063C
:10A890008C1304C00E944B85811170C080912302EB
:10A8A0008823A1F08091080E811103C024E038E2D2
:10A8B00002C028E038E281E0909113069C1380E00A
:10A8C00001E046EF57E26D2F0E94FB46DF5FCF5F4E
:10A8D000D53009F0EECE1C5F109312065CC0BBDBD6
:10A8E0008091E005882309F4EECE55C08CEE97E503
:10A8F0000E941F4B8091E005882309F400CF4BC0D4
:10A900008EE290E50E941F4B8091E005882309F4B8
:10A9100013CF41C08AEB99E50E941F4B8091E0055F
:10A92000882309F425CF37C08EEE9BE50E941F4B8C
:10A930008091E005882309F43ACF2DC015E06ACF55
:10A9400082EE9CE40E941F4B8091E005882309F46D
:10A950004ECF21C08DE896E50E941F4B8091E00507
:10A96000882309F463CF17C08BE595E50E941F4B40
:10A970008091E005882309F475CF0DC040E050E0D8
:10A9800068E07EE08BE098E20E94FA7F8091E0052B
:10A99000882309F483CFDF91CF911F910F91089500
:10A9A0002F923F924F925F926F927F928F929F92DF
:10A9B000AF92BF92CF92DF92EF92FF920F931F93CD
:10A9C000CF93DF9300D000D0CDB7DEB71C017E83DC
:10A9D0006D8329013A01460120E030E040E057EC68
:10A9E000B201C3010F94625D18162CF0412C512C5A
:10A9F000612C27EC01C0272DB201862D922F0F94D8
:10AA0000CE5B2B013C0120E03EEF4FEF56E4B70157
:10AA1000C8010F945F5B87FD06C0B12C9EEFF92E35
:10AA20000FEF16E401C0BE2CC301B2010F94015C0C
:10AA30009B01AC01ED81FE816081718182819381F6
:10AA40000F94855A0F94D35B69837A838B839C839D
:10AA50006B2D7F2DC8010F94CE5B7B018C01E41818
:10AA6000F50806091709AF9289E0A82E8FE4B82EE1
:10AA7000C980DA80A30192016D817E81C1010E94AB
:10AA8000937F0F9026960FB6F894DEBF0FBECDBF12
:10AA9000DF91CF911F910F91FF90EF90DF90CF90BA
:10AAA000BF90AF909F908F907F906F905F904F90EE
:10AAB0003F902F9008956F927F928F929F92AF92C6
:10AAC000BF92CF92DF92EF92FF920F931F93CF939B
:10AAD000DF9300D01F92CDB7DEB761E081E00E9426
:10AAE000388160901406712C61101AC08091130691
:10AAF000811104C00E944B85811198C0809123026E
:10AB0000882309F48AC081E090911306911180E0B6
:10AB100004E024E040E95AE2672D0E94CC467DC063
:10AB200081E068122CC080911306813021F40E94CC
:10AB30004B85811182C080912302882309F46DC066
:10AB400011E080911306813009F010E08091A90D89
:10AB50009091AA0DA091AB0DB091AC0D89839A8311
:10AB6000AB83BC83CE0101960F94245100E09C017D
:10AB70004CE75AE2672D812F0E94FB464EC082E0CF
:10AB8000681225C080911306823021F40E944B8503
:10AB9000811181C080912302882309F43EC011E015
:10ABA00080911306823009F010E06091EE0B7091F5
:10ABB000EF0B8091F00B9091F10B05DA00E09C0116
:10ABC00048E65AE2672D812F0E94FB4626C083E0AB
:10ABD000681223C080911306833021F40E944B85B4
:10ABE000811171C0809123028823B9F011E0809116
:10ABF0001306833009F010E06091F20B7091F30BB3
:10AC00008091F40B9091F50BDED900E09C0148E5B2
:10AC10005AE2672D812F0E94FB467394639485E06E
:10AC2000781262CF84E08093120664C014DA8091B7
:10AC3000E005882309F462CF5DC020E030E048ECF5
:10AC400052E46091A90D7091AA0D8091AB0D909185
:10AC5000AC0D0F949D5D0F94D35B1F92812C912CB2
:10AC600023E0A22E2FE4B22E6B01EE24EA941FE71C
:10AC7000F12E00E010E020E030E0A90169EA7DE07B
:10AC800086E89AE20E94937F0F908091E0058823E6
:10AC900009F451CF2FC081E00E944085A12CC12C26
:10ACA000D12CE12CF12C08E413E420E030E0A901E0
:10ACB0006EEE7BE082E79AE273DE8091E005882306
:10ACC00009F468CF17C081E00E944085A12CC12CF7
:10ACD000D12CE12CF12C08E413E420E030E0A901B0
:10ACE00062EF7BE080E69AE25BDE8091E0058823FC
:10ACF00009F478CF0F900F900F900F90DF91CF91C4
:10AD00001F910F91FF90EF90DF90CF90BF90AF9089
:10AD10009F908F907F906F9008956F927F928F9207
:10AD20009F92AF92BF92CF92DF92EF92FF920F93DA
:10AD30001F93CF93DF9300D01F92CDB7DEB761E0B2
:10AD400081E00E94388160901406712C61101AC055
:10AD500080911306811104C00E944B858111BDC0F2
:10AD600080912302882309F4B0C081E090911306FA
:10AD7000911180E004E024E046E45AE2672D0E944D
:10AD8000CC46A3C081E0681223C0809113068130B5
:10AD900021F40E944B858111A7C080912302882352
:10ADA00009F493C08091D60D811103C026E33AE2E5
:10ADB00002C02AE33AE281E090911306913009F053
:10ADC00080E001E04DE25AE2672D0E94FB467DC023
:10ADD00082E0681225C080911306823021F40E941F
:10ADE0004B8581118FC080912302882309F46DC0A7
:10ADF00011E080911306823009F010E06091820228
:10AE0000709183028091840290918502DCD800E0E9
:10AE10009C014FE15AE2672D812F0E94FB4655C0ED
:10AE200083E0681225C080911306833021F40E94CC
:10AE30004B8581117CC080912302882309F445C091
:10AE400011E080911306833009F010E060918602D2
:10AE5000709187028091880290918902B4D800E0B5
:10AE60009C0141E15AE2672D812F0E94FB462DC0D3
:10AE700084E068122AC080911306843021F40E9475
:10AE80004B85811169C0809123028823F1F011E084
:10AE900080911306843009F010E080917E02909139
:10AEA0007F02A0918002B091810289839A83AB8353
:10AEB000BC83CE0101960F94245100E09C0141E037
:10AEC0005AE2672D812F0E94FB467394639485E0BC
:10AED00078123CCF709212066CC0BDD88091E0050C
:10AEE000882309F43DCF65C040E050E066ED7DE089
:10AEF0008DE39AE20E94FA7F8091E005882309F4AD
:10AF00004CCF57C0A12CC12CD12CE12CF12C01E944
:10AF100013E420E030E0A90162E872E086E29AE200
:10AF20003FDD8091E005882309F45DCF42C0A12C6C
:10AF3000C12CD12CE12CF12C01E913E420E030E00C
:10AF4000A90166E872E088E19AE22ADD8091E005D5
:10AF5000882309F470CF2DC020E030E048EC52E4A3
:10AF600060917E0270917F028091800290918102B7
:10AF70000F949D5D0F94D35B1F92812C912C83E0E5
:10AF8000A82E8FE4B82E6B0118EEE12E13E0F12EFF
:10AF900000E010E020E030E0A9016EE772E089E017
:10AFA0009AE20E94937F0F908091E005882309F434
:10AFB0006ACF0F900F900F900F90DF91CF911F915C
:10AFC0000F91FF90EF90DF90CF90BF90AF909F9048
:10AFD0008F907F906F900895AF92CF92DF92EF9213
:10AFE000FF920F931F93CF93DF9361E081E00E9464
:10AFF0003881D0911406C0E0D1111AC08091130697
:10B00000811104C00E944B85811109C180912302E6
:10B01000882309F4FBC081E090911306911180E030
:10B0200004E024E04FEE59E26C2F0E94CC46EEC0C3
:10B03000D13031F580911306813021F40E944B8587
:10B040008111F5C080912302882309F4DFC011E04B
:10B0500080911306813009F010E060915D0E7091CF
:10B060005E0E80915F0E9091600E0E94E34F00E0B3
:10B070009C0141EE59E26C2F812F0E94FB46C6C015
:10B08000D23031F580911306823021F40E944B8535
:10B090008111E7C080912302882309F4B7C011E031
:10B0A00080911306823009F010E06091610E70917A
:10B0B000620E8091630E9091640E0E94E34F00E057
:10B0C0009C0143ED59E26C2F812F0E94FB469EC0EC
:10B0D000D33031F580911306833021F40E944B85E3
:10B0E0008111D9C080912302882309F48FC011E017
:10B0F00080911306833009F010E06091650E709125
:10B10000660E8091670E9091680E0E94E34F00E0FA
:10B110009C0145EC59E26C2F812F0E94FB4676C0C2
:10B12000D43031F580911306843021F40E944B8590
:10B130008111CBC080912302882309F467C011E0FC
:10B1400080911306843009F010E06091690E7091CF
:10B150006A0E80916B0E90916C0E0E94E34F00E09E
:10B160009C0147EB59E26C2F812F0E94FB464EC099
:10B17000D53031F580911306853021F40E944B853E
:10B180008111BDC080912302882309F43FC011E0E2
:10B1900080911306853009F010E06091790E70916E
:10B1A0007A0E80917B0E90917C0E0E94E34F00E01E
:10B1B0009C014DEA59E26C2F812F0E94FB4626C06C
:10B1C000D63021F580911306863021F40E944B85FC
:10B1D0008111AEC0809123028823C1F011E08091DB
:10B1E0001306863009F010E060917D0E70917E0E9E
:10B1F00080917F0E9091800E0E94E34F00E09C01B1
:10B2000049E959E26C2F812F0E94FB46CF5FDF5F37
:10B21000C53009F0F1CE87E080931206A1C00E94EC
:10B220002B508091E005882309F4F0CE99C081E08D
:10B230000E944085A12CC12CD12CE12C10ECF12EC8
:10B2400009E714E420E030E040E85FE36DE57EE0EC
:10B2500088EE99E2A5DB8091E005882309F4F2CE1F
:10B260007FC081E00E944085A12CC12CD12CE12C13
:10B2700010ECF12E09E714E420E030E040E85FE351
:10B2800061E67EE08AED99E28BDB8091E005882320
:10B2900009F400CF65C081E00E944085A12CC12C3B
:10B2A000D12CE12C10ECF12E09E714E420E030E081
:10B2B00040E85FE365E67EE08CEC99E271DB80912B
:10B2C000E005882309F40ECF4BC081E00E94408541
:10B2D000A12CC12CD12CE12C10ECF12E09E714E4A7
:10B2E00020E030E040E85FE369E67EE08EEB99E243
:10B2F00057DB8091E005882309F41CCF31C081E041
:10B300000E944085A12CC12CD12CE12C10ECF12EF7
:10B3100009E714E420E030E0A90169E77EE082EB70
:10B3200099E23EDB8091E005882309F42BCF18C019
:10B3300081E00E944085A12CC12CD12CE12C10EC85
:10B34000F12E09E714E420E030E0A9016DE77EE08A
:10B3500083EA99E225DB8091E005882309F43ACF5E
:10B36000DF91CF911F910F91FF90EF90DF90CF90E1
:10B37000AF9008956F927F928F929F92AF92BF92FB
:10B38000CF92DF92EF92FF920F931F93CF93DF93B1
:10B3900000D01F92CDB7DEB761E081E00E94388116
:10B3A00060901406712C61101AC0809113068111EF
:10B3B00004C00E944B858111C2C080912302882362
:10B3C00009F4B5C081E090911306911180E004E08A
:10B3D00024E04BE059E2672D0E94CC46A8C081E0F2
:10B3E000681226C080911306813021F40E944B859B
:10B3F0008111ADC080912302882309F498C011E027
:10B4000080911306813009F010E06091090E70916F
:10B410000A0E80910B0E90910C0E0E94E34F00E0FB
:10B420009C014BEF58E2672D812F0E94FB467FC0A5
:10B4300082E0681226C080911306823021F40E94B7
:10B440004B8581119EC080912302882309F46FC02F
:10B4500011E080911306823009F010E060910D0E2A
:10B4600070910E0E80910F0E9091100E0E94E34F7E
:10B4700000E09C014BEE58E2672D812F0E94FB46B5
:10B4800056C083E068122CC080911306833021F4EB
:10B490000E944B8581118FC080912302882309F47B
:10B4A00046C011E080911306833009F010E08091CE
:10B4B000110E9091120EA091130EB091140E89836B
:10B4C0009A83AB83BC83CE0101960F94DB5300E0DB
:10B4D0009C014BED58E2672D812F0E94FB4627C04F
:10B4E00084E0681224C080911306843021F40E9405
:10B4F0004B85811198C0809123028823C1F011E00F
:10B5000080911306843009F010E06091150E70915F
:10B51000160E8091170E9091180E0E94E34F00E0D6
:10B520009C014BEC58E2672D812F0E94FB467394DF
:10B53000639485E0781237CF709212068DC00E9416
:10B540002B508091E005882309F437CF85C081E036
:10B550000E944085A12CC12CD12CE12C10E8F12EA9
:10B5600007E714E420E030E040E85FE369E07EE0D4
:10B5700083E099E215DA8091E005882309F43ACF57
:10B580006BC081E00E944085A12CC12CD12CE12C04
:10B5900010E8F12E07E714E420E030E040E85FE334
:10B5A0006DE07EE083EF98E2FBD98091E00588238F
:10B5B00009F449CF51C081E00E94408520E030E08D
:10B5C00048EC52E46091110E7091120E8091130EAE
:10B5D0009091140E0F949D5D20E030E040E251E424
:10B5E0000F94855A0F94D35B1F92812C912C97E274
:10B5F000A92E9FE4B92E6B0115EFE12E1FE7F12E66
:10B6000000E010E02AE030E040E050E061E17EE060
:10B6100083EE98E20E94937F0F908091E00588234B
:10B6200009F43ACF19C081E00E944085A12CC12CB9
:10B63000D12CE12C10E8F12E07E714E420E030E0F3
:10B6400040E85FE365E17EE083ED98E2A9D980916F
:10B65000E005882309F44FCF0F900F900F900F90C3
:10B66000DF91CF911F910F91FF90EF90DF90CF90DE
:10B67000BF90AF909F908F907F906F9008952F9282
:10B680003F924F925F926F927F928F929F92AF9272
:10B69000BF92CF92DF92EF92FF920F931F93CF93BF
:10B6A000DF93CDB7DEB729970FB6F894DEBF0FBE94
:10B6B000CDBF1C0179876887CA01B901E982FA8286
:10B6C0000B831C83DE82CD82AF8220E030E040E23B
:10B6D00051E40F949D5D6B017C0120E030E040E07F
:10B6E00057EC0F94625D18162CF0C12CD12CE12C74
:10B6F00027ECF22EC701B6010F94CE5B2B013C0163
:10B7000020E030E040E251E469817A818B819C81C4
:10B710000F949D5D4B015C0120E03EEF4FEF56E43E
:10B720000F945F5B87FD07C0812C9EEF992EAA24A2
:10B73000AA9496E4B92E20E030E040E251E4E88596
:10B74000F98560817181828193810F949D5D6B0188
:10B750007C01C301B2010F94015C9B01AC01C701E4
:10B76000B6010F94855A0F94D35B69837A838B83D8
:10B770009C83C501B4010F94CE5B7B018C01E4185E
:10B78000F50806091709FF81FF938D809E808DE2E1
:10B79000A82E8FE4B82EC980DA80A30192016885B3
:10B7A0007985C1010E94937F0F9029960FB6F89476
:10B7B000DEBF0FBECDBFDF91CF911F910F91FF90E4
:10B7C000EF90DF90CF90BF90AF909F908F907F9041
:10B7D0006F905F904F903F902F9008959F92AF92FF
:10B7E000BF92CF92DF92EF92FF920F931F93CF936E
:10B7F000DF9300D01F92CDB7DEB761E081E00E94F9
:10B80000388190901406B12C91101AC080911306C3
:10B81000811104C00E944B858111D4C08091230204
:10B82000882309F4C7C081E090911306911180E04C
:10B8300004E024E049EB58E26B2D0E94CC46BAC0EC
:10B8400081E098122CC080911306813021F40E946F
:10B850004B858111BFC080912302882309F4AAC0BF
:10B8600011E080911306813009F010E080914D0EB7
:10B8700090914E0EA0914F0EB091500E89839A83F5
:10B88000AB83BC83CE0101960F94785400E09C01F9
:10B8900045EA58E26B2D812F0E94FB468BC082E067
:10B8A00098122CC080911306823021F40E944B859F
:10B8B0008111ACC080912302882309F47BC011E080
:10B8C00080911306823009F010E08091510E909122
:10B8D000520EA091530EB091540E89839A83AB837C
:10B8E000BC83CE0101960F94785400E09C0141E99D
:10B8F00058E26B2D812F0E94FB465CC083E09812BA
:10B900002CC080911306833021F40E944B85811155
:10B9100099C080912302882309F44CC011E08091E2
:10B920001306833009F010E08091550E9091560E69
:10B93000A091570EB091580E89839A83AB83BC8334
:10B94000CE0101960F94785400E09C014DE758E237
:10B950006B2D812F0E94FB462DC084E098122AC0D7
:10B9600080911306843021F40E944B85811186C09A
:10B97000809123028823F1F011E080911306843036
:10B9800009F010E08091590E90915A0EA0915B0E33
:10B99000B0915C0E89839A83AB83BC83CE01019600
:10B9A0000F94785400E09C0149E658E26B2D812FFA
:10B9B0000E94FB46B394939485E0B81225CFB092D1
:10B9C000120677C00E942B508091E005882309F46D
:10B9D00025CF6FC081E00E944085A12C65E3C62E73
:10B9E0006FE4D62EE12C1CE3F12E0CE116E420E0EE
:10B9F00030E040EA50E46DE47EE08FEA98E23FDE1A
:10BA00008091E005882309F426CF53C081E00E948D
:10BA10004085A12C45E3C42E4FE4D42EE12C1CE339
:10BA2000F12E0CE116E420E030E040EA50E461E55C
:10BA30007EE08BE998E223DE8091E005882309F41B
:10BA400039CF37C081E00E944085A12C25E3C22E6A
:10BA50002FE4D22EE12C1CE3F12E0CE116E420E0C1
:10BA600030E040EA50E465E57EE087E898E207DEF2
:10BA70008091E005882309F44CCF1BC081E00E942F
:10BA80004085A12C85E3C82E8FE4D82EE12C1CE341
:10BA9000F12E0CE116E420E030E040EA50E469E5E4
:10BAA0007EE083E798E2EBDD8091E005882309F4EE
:10BAB0005FCF0F900F900F900F90DF91CF911F915C
:10BAC0000F91FF90EF90DF90CF90BF90AF909F903D
:10BAD00008950F93CF93DF9361E081E00E94388156
:10BAE000C0911406D0E0C11118C0809113068111D5
:10BAF00004C00E944B858111B5C080912302882328
:10BB000061F081E090911306911180E004E024E05F
:10BB10004DEF5BE26D2F0E94CC468091840D8770C3
:10BB2000873009F058C0C130D9F4809113068130B4
:10BB300021F40E944B8581119EC0809123028823AD
:10BB400009F4C1C081E090911306913009F080E0C2
:10BB500003E02EE346EF5BE26D2F0E94CC46B3C0BC
:10BB6000C230D9F480911306823021F40E944B85B3
:10BB700081118BC080912302882309F4A4C081E045
:10BB800090911306923009F080E003E02EE34FEE2F
:10BB90005BE26D2F0E94CC4696C0C330D1F58091F8
:10BBA0001306833021F40E944B85811178C0809167
:10BBB0002302882309F487C081E090911306933013
:10BBC00009F080E003E02EE348EE5BE26D2F0E9477
:10BBD000CC4684E03EC0C130F1F480911306813040
:10BBE00021F40E944B85811164C080912302882337
:10BBF00009F46BC081E090911306913009F080E068
:10BC000000E22EE34AED5BE26D2F0E94CC4682E01B
:10BC100020C084E001C082E0C8131BC080911306DD
:10BC20008C1304C00E944B85811151C08091230266
:10BC3000882371F081E0909113069C1380E003E06B
:10BC40002EE340ED5BE26D2F0E94CC468C2F01C0AD
:10BC50008C2FDF5FCF5FD53009F045CF8F5F8093AA
:10BC600012063EC081E00E9452808091E005882348
:10BC700009F443CF35C086E992E60E941F4B8091BC
:10BC8000E005882309F459CF2BC08BE992E60E9486
:10BC90001F4B8091E005882309F46CCF21C080EA16
:10BCA00092E60E941F4B8091E005882309F47FCF24
:10BCB00017C084EE9BE20E94917F8091E00588236B
:10BCC00009F493CF0DC084E0C4CF82E0C2CF85EAEF
:10BCD00092E60E941F4B8091E005882309F4A6CFCD
:10BCE000DF91CF910F910895CF92DF92EF92FF9263
:10BCF000CF93C82F0E9487306B017C0124EA30E784
:10BD00004DE75FE360912B0670912C0680912D0624
:10BD100090912E060F945F5B87FD05C04AEF50E0BF
:10BD200060E070E003C040E050E0BA01C40ED51EF0
:10BD3000E61EF71EC0922706D0922806E09229063A
:10BD4000F0922A06C0932402CF91FF90EF90DF90EB
:10BD5000CF9008952F923F924F925F926F927F9271
:10BD60008F929F92AF92BF92CF92DF92EF92FF920B
:10BD70001F93CF93DF93CDB7DEB728970FB6F89414
:10BD8000DEBF0FBECDBF1C01162F0E944B8588233E
:10BD900031F01092420680E00E945280DDC0209176
:10BDA0003A0630913B063E832D83232B09F4A0C035
:10BDB000E4E01E9FC001112498878F83FC01E259A3
:10BDC000FD4F80809180A280B38020E030E04AE780
:10BDD00054E4C501B4010F94855A2B013C0120E0C5
:10BDE00030E04AE754E4C501B4010F94865A6B0170
:10BDF0007C01809163028823B9F1113029F198F018
:10BE0000123091F540905B0250905C0260905D02B0
:10BE100070905E02C0905F02D0906002E09061027C
:10BE2000F090620221C040904B0250904C02609012
:10BE30004D0270904E02C0904F02D0905002E090A0
:10BE40005102F090520210C04090530250905402A0
:10BE50006090550270905602C0905702D0905802E0
:10BE6000E0905902F0905A022D813E81B901330FC2
:10BE7000880B990B0F94015C20912B0630912C06B6
:10BE800040912D0650912E060F949D5D9B01AC01B3
:10BE9000C501B4010F94865A9B01AC018F8198852E
:10BEA00082599D4F5C01FC0120833183428353837F
:10BEB0008D819E8197FF0CC0C301B2010F94625D1A
:10BEC00018168CF4F50140825182628273820BC095
:10BED000C701B6010F945F5B87FF05C0F501C08203
:10BEE000D182E282F382812FFFDE81E08093230200
:10BEF00010923B0610923A0680912302882361F14A
:10BF000024E0129FF0011124E259FD4F80819181BC
:10BF1000A281B38189839A83AB83BC832DEC3CECF3
:10BF20004CEC5DE360912B0670912C0680912D0600
:10BF300090912E060F94625D87FD05C0CE0101969B
:10BF40000F94EA5105C060E2CE0101960F9462524F
:10BF5000BC01C1010E945A4728960FB6F894DEBF73
:10BF60000FBECDBFDF91CF911F91FF90EF90DF907B
:10BF7000CF90BF90AF909F908F907F906F905F9089
:10BF80004F903F902F90089560E08EE79CE2E2CEC4
:10BF900061E087E79CE2DECE62E080E79CE2DACEF9
:10BFA000CF93DF9300D01F92CDB7DEB70E944B85B1
:10BFB000882331F01092420680E00E94528057C0E0
:10BFC00060913A0670913B066115710569F1072E83
:10BFD000000C880B990B0F94015C20912B0630917B
:10BFE0002C0640912D0650912E060F949D5D9B01CD
:10BFF000AC0160917A0270917B0280917C029091F9
:10C000007D020F94865A60937A0270937B0280932C
:10C010007C0290937D0283E067DE81E080932302BF
:10C0200010923B0610923A06809123028823F9F081
:10C03000209148053091490540914A0550914B05A2
:10C0400060917A0270917B0280917C0290917D02D6
:10C050000F94855A69837A838B839C83CE010196E2
:10C060000F94EA51BC0184E09CE20E945A470F9071
:10C070000F900F900F90DF91CF91089521E02093C2
:10C08000420660932B0670932C0680932D069093A6
:10C090002E0620E040E060E070E08091460590913F
:10C0A00047050C941F8060E070E080E291E4E6CFE9
:10C0B00060E070E080E89FE3E1CF6DEC7CEC8CEC1D
:10C0C0009DE3DCCF6DEC7CEC8CEC9CE3D7CF8F92C6
:10C0D0009F92AF92BF92CF92DF92EF92FF920F9317
:10C0E0001F93CF93DF93CDB7DEB76E970FB6F8945B
:10C0F000DEBF0FBECDBFD82E7093470560934605B7
:10C1000061E081E00E943881F09014068CE0C82E36
:10C11000E12C91E02EE0A22E2CE2B22E9E012F5FA8
:10C120003F4F490131E0D31659F1D31628F082E090
:10C13000D81609F449C06CC0F110D2C0992389F017
:10C140008091130618166CF020913A0630913B0648
:10C150002F5F3F4F30933B0620933A068F5F8093CB
:10C16000130680912302882309F432C100E010E015
:10C1700021E041E069E67CE28E2D0E946D4628C1F7
:10C18000F110AEC0992389F08091130618166CF057
:10C1900020913A0630913B062F5F3F4F30933B068C
:10C1A00020933A068F5F80931306809123028823A1
:10C1B00009F411C100E010E021E041E062E67CE218
:10C1C0008E2D0E946D4607C1F1108AC0992389F017
:10C1D0008091130618166CF020913A0630913B06B8
:10C1E0002F5F3F4F30933B0620933A068F5F80933B
:10C1F000130680912302882309F40BC100E010E0AC
:10C2000021E041E06BE57CE28E2D0E946D4601C18C
:10C2100040917A0250917B0260917C0270917D0284
:10C22000409348055093490560934A0570934B0528
:10C23000F11020C0992389F08091130618166CF034
:10C2400020913A0630913B062F5F3F4F30933B06DB
:10C2500020933A068F5F80931306809123028823F0
:10C2600049F000E010E021E041E061E57CE28E2D44
:10C270000E946D4693E0D91233C06091B20C709168
:10C28000B30C8091B40C9091B50C2091770C2111D6
:10C2900027C00F94CE5B2091390230913A02621789
:10C2A0007307F4F421E0F21219C080911306813073
:10C2B00021F40E944B858111C0C080912302882304
:10C2C00069F081E090911306913009F080E004E07C
:10C2D00024E041E45CE26E2D0E94CC4682E0A2C0E4
:10C2E00031E0F3121BC080911306813021F40E94CB
:10C2F0004B858111ABC080912302882309F468C06B
:10C3000081E090911306913009F080E004E024E090
:10C3100047E35CE26E2D0E94CC465AC082E0F812E0
:10C320001BC080911306823021F40E944B8581113D
:10C3300096C080912302882309F49BC081E09091EC
:10C340001306923009F080E003E02EE34DE25CE258
:10C350006E2D0E94CC468DC093E0F9121BC08091D7
:10C360001306833021F40E944B85811186C0809191
:10C370002302882309F4C3C081E09091130693300F
:10C3800009F080E003E02EE344E25CE26E2D0E94BF
:10C39000CC46B5C024E0F2121BC080911306843055
:10C3A00021F40E944B85811172C080912302882361
:10C3B00009F4A5C081E090911306943009F080E063
:10C3C00003E02EE349E15CE26E2D0E94CC4697C06B
:10C3D00032E0D31611F085E025C085E0F81219C0CF
:10C3E00080911306853021F40E944B85811159C03C
:10C3F00080912302882369F081E0909113069530A3
:10C4000009F080E003E02EE348E15CE26E2D0E943B
:10C41000CC4680912302882321F095E0F91609F497
:10C420004AC086E0E394F3942CE0C20E90E035E03D
:10C43000E31278CE8093120666C081E00E9452809B
:10C440008091E005882309F438CF5DC081E00E9427
:10C4500052808091E005882309F44DCF54C083E5D4
:10C4600090E60E941F4B8091E005882309F461CF7C
:10C470004AC082E0D812AFCFCCCF88E590E60E94C8
:10C480001F4B8091E005882309F471CF3CC08DE5F6
:10C4900090E60E941F4B8091E005882309F485CF28
:10C4A00032C082E690E60E941F4B8091E00588230F
:10C4B00009F49ECF28C06C2D86E00E9421428E0197
:10C4C0000B5E1F4F23E041E06DEC7CEC8CEC9CE3B9
:10C4D0000F940E5F9F938F93BF92AF929F928F9214
:10C4E0000F942064B40188E094E00E94BA3B0F905E
:10C4F0000F900F900F900F900F9086E093CF92E0E7
:10C50000D91269CF86CF6E960FB6F894DEBF0FBEF4
:10C51000CDBFDF91CF911F910F91FF90EF90DF90F2
:10C52000CF90BF90AF909F908F9008954FEF64ECA5
:10C530007FE580E0CCCD4FEF68EC7FE581E0C7CDB3
:10C540004FEF6CEC7FE582E0C2CD4FEF60ED7FE511
:10C5500083E0BDCD0F93CF93DF9361E081E00E9434
:10C560003881D0911406C0E0D1111AC08091130611
:10C57000811104C00E944B858111A9C080912302C2
:10C58000882309F49BC081E090911306911180E00B
:10C5900004E024E04BEC5BE26C2F0E94CC468EC0A2
:10C5A000D130D9F480911306813021F40E944B855B
:10C5B000811196C080912302882309F47FC081E015
:10C5C00090911306913009F080E003E02EE341ECF6
:10C5D0005BE26C2F0E94CC4671C0D230D9F48091BE
:10C5E0001306823021F40E944B85811183C0809113
:10C5F0002302882309F462C081E0909113069230EF
:10C6000009F080E000E22EE346E75BE26C2F0E9437
:10C61000CC4654C0D330D9F480911306833021F432
:10C620000E944B85811170C080912302882309F4F8
:10C6300045C081E090911306933009F080E000E25C
:10C640002EE348E65BE26C2F0E94CC4637C0D43024
:10C65000D1F480911306843021F40E944B8581111E
:10C660005DC080912302882349F181E090911306F7
:10C67000943009F080E000E22EE347EB5AE26C2FA1
:10C680000E94CC461BC0D530C9F48091130685307A
:10C6900021F40E944B8581114BC080912302882395
:10C6A00069F081E090911306953009F080E000E296
:10C6B0002EE342EA5AE26C2F0E94CC46CF5FDF5F46
:10C6C000C53009F051CF86E0809312063AC081E070
:10C6D0000E9452808091E005882309F44FCF31C039
:10C6E00089E69DE50E941F4B8091E005882309F4AF
:10C6F00061CF27C083E89BE20E94917F8091E00593
:10C70000882309F474CF1DC082E79BE20E94917FC9
:10C710008091E005882309F487CF13C086EC9AE264
:10C720000E94917F8091E005882309F49ACF09C087
:10C7300083EB9AE20E94917F8091E005882309F4BF
:10C74000ACCFDF91CF910F910895CF92DF92EF920E
:10C75000FF920F931F938091D108811103C083E151
:10C7600099E002C081ED98E02AECC22E2CE2D22E94
:10C770007C010DEB1CE22CEC33E64FEC53E666EB50
:10C780007CE280EB9CE20E9446821F910F91FF9019
:10C79000EF90DF90CF90089580E00C94528083E179
:10C7A00099E00E9433900E944B800C946B8B0E9406
:10C7B000D59421E030E0811102C020E030E03093D8
:10C7C0003B0620933A061092140681E08093E00520
:10C7D00083E0809323020895EF92FF920F931F93BB
:10C7E000CF93DF9380913C06882331F00E94E5953A
:10C7F00090934D0580934C0561E081E00E94388163
:10C80000C0911406D0E0C11118C0809113068111A7
:10C8100004C00E944B85811197C080912302882318
:10C8200061F081E090911306911180E004E024E032
:10C830004BEA5CE26D2F0E94CC468091200985FD79
:10C840001FC083FF1DC0C130C9F480911306813021
:10C8500021F40E944B85811180C08091230288239E
:10C8600069F081E090911306913009F080E000E2D8
:10C870002EE347EA5CE26D2F0E94CC4692E001C0B5
:10C8800091E080912302882309F456C0E12CF12C19
:10C8900011E01C0F20914C0530914D05E216F30676
:10C8A00008F04AC0C91343C0C901019760E070E0B5
:10C8B0008E199F090E94A8919091200980911306DA
:10C8C00094FF1CC08C1350C00E944B85882309F430
:10C8D0004BC083E199E00E947A941092140682E0A2
:10C8E00090E090933B0680933A0681E08093E005C8
:10C8F00010923D0683E08093230254C08C1304C041
:10C900000E944B8581113FC080912302882369F0EA
:10C9100081E0909113069C1380E000E02EEE37E159
:10C9200045E85CE26D2F0E945048912F01C09F5F47
:10C930008FEFE81AF80AAECFDF5FCF5FD53009F08E
:10C9400062CF909312062EC081E00E9452808091A7
:10C95000E005882309F461CF25C029DF8091E00537
:10C96000882309F47ACF1EC0809123028823E9F23C
:10C9700081E0909113069C1380E001E02EEE37E1F8
:10C9800046E95CE2CFCF0E946C7F20E040E060E0AF
:10C9900070E085EA93E60E941F808091E00588237D
:10C9A00009F4B2CFDF91CF911F910F91FF90EF90DB
:10C9B0000895CF93DF93EC01CB01BA010F94015C92
:10C9C0000F94CE5B79836883DF91CF91089569EDF1
:10C9D00074E680E795E60C9476800F931F93CF93CF
:10C9E000DF9361E081E00E943881C0911406D0E0BD
:10C9F00081E0C11122C0882389F0809113061816A6
:10CA00006CF020913A0630913B062F5F3F4F3093F8
:10CA10003B0620933A068F5F809313068091230292
:10CA2000882309F441C000E010E020E041E06FE21B
:10CA30007EE28D2F0E946D4637C0C130D1F48091C7
:10CA40001306813021F40E944B85811137C08091FB
:10CA50002302882349F181E090911306913009F077
:10CA600080E000E22EE344E25EE26D2F0E94CC46BD
:10CA70001BC0C230C9F480911306823021F40E9499
:10CA80004B85811122C080912302882369F081E0C7
:10CA900090911306923009F080E000E22EE340E12D
:10CAA0005EE26D2F0E94CC46DF5FCF5F80E0D53025
:10CAB00009F09FCF83E0809312060DC0C093F60B60
:10CAC0008091E005882319F206C0C093F60B80918F
:10CAD000E0058823C1F2DF91CF911F910F91089556
:10CAE0000F94015C0F94CE5BCB010D942450EF9218
:10CAF000FF920F931F93CF93DF93CDB7DEB72B97A2
:10CB00000FB6F894DEBF0FBECDBF7C0140914F053C
:10CB1000842F042E000C990B20915005223051F0E7
:10CB2000233019F02EE53EE20AC047FF06C02AE690
:10CB30003EE205C02CE73EE202C023E73EE29F93BF
:10CB40004F933F932F938E010F5F1F4F1F930F93B0
:10CB50000F94206440913702509138024F50510990
:10CB600097010F900F900F900F900F900F904E1510
:10CB70005F050CF49A013093B70C2093B60C80E05B
:10CB80000E94C0BAC8010E9423822B960FB6F89467
:10CB9000DEBF0FBECDBFDF91CF911F910F91FF90F0
:10CBA000EF900895E0914F0587E1E802F00111242C
:10CBB000E255F34F808591859ACF7F928F929F9215
:10CBC000AF92BF92CF92DF92EF92FF920F931F939B
:10CBD000CF93DF93782E8093500560934F0561E0EB
:10CBE00081E00E943881D0911406C0E081E0D1112B
:10CBF0002EC0882389F08091130618166CF02091BE
:10CC00003A0630913B062F5F3F4F30933B0620930F
:10CC10003A068F5F8093130680912302882309F4DC
:10CC200094C022E0721649F033E0731203C060E44E
:10CC30007EE205C060E37EE202C060E57EE200E0E5
:10CC400010E021E041E08C2F0E946D467EC0D13083
:10CC5000D9F480911306813021F40E944B85811113
:10CC60007DC080912302882309F46FC081E09091F8
:10CC70001306913009F080E004E024E04BEB5EE223
:10CC80006C2F0E94CC4661C0D230D9F4809113063B
:10CC9000823021F40E944B85811169C0809123026A
:10CCA000882309F452C081E090911306923009F074
:10CCB00080E000E22EE34FEA5EE26C2F0E94CC4659
:10CCC00044C0D330D1F480911306833021F40E9404
:10CCD0004B85811157C0809123028823B1F181E0F7
:10CCE00090911306933009F080E000E22EE343EACE
:10CCF0005EE26C2F0E94CC4628C0D43031F5809182
:10CD00001306843021F40E944B85811146C0809126
:10CD100023028823D1F011E080911306843009F0BA
:10CD200010E020914F0537E12303F0011124E25573
:10CD3000F34F808591850F94245000E09C0145E8D5
:10CD40005EE26C2F812F0E94FB46CF5FDF5F80E0A9
:10CD5000C53009F04CCFC09312065CC081E00E9440
:10CD600052808091E005882309F47BCF53C08091E5
:10CD7000570590915805BBDE8091E005882309F4A2
:10CD80008DCF48C08091590590915A05B0DE8091B1
:10CD9000E005882309F49FCF3DC081E00E944085D3
:10CDA00000914F0527E1020380011124F801E255AB
:10CDB000F34F60857185072E000C880B990B0F943B
:10CDC000015C20E030E040EF52E40F94855A0F946C
:10CDD000D35BF801EA54F34F1F9282ED882E85E66B
:10CDE000982E97EEA92E94E6B92E6B011AEAE12E41
:10CDF000F12C00E010E028E730E040E050E0BF0117
:10CE000084E99EE20E94937F0F908091E005882341
:10CE100009F47DCFDF91CF911F910F91FF90EF909B
:10CE2000DF90CF90BF90AF909F908F907F900895AC
:10CE300060E081E0C2CE8F929F92AF92BF92CF927C
:10CE4000DF92EF92FF920F931F93CF93DF934C01EA
:10CE50005B016A0160E085E00E943881D091140690
:10CE6000F12C82E0E82ED1111AC080912302882390
:10CE700021F180912802823041F0833019F465EE6F
:10CE80007DE205C063ED7DE202C065EF7DE200E07A
:10CE900010E021E041E08F2D0E946D460EC0D130A0
:10CEA00061F480912302882341F000E010E020E04B
:10CEB00041E0B4018F2D0E946D46A114B10481F0B0
:10CEC000D23081F480912302882309F46EC000E0FF
:10CED00010E020E041E0B5018F2D0E946D4665C055
:10CEE000C2E001C0C3E0C114D10491F0DC130FC053
:10CEF00080912302882351F000E010E020E041E01F
:10CF0000B6018F2D0E946D46CD2F01C0CD2FCF5F72
:10CF100021E030E0A114B10411F420E030E081E020
:10CF200090E0C114D10411F480E090E0820F931FCF
:10CF3000029781F0DC130DC080912302882349F011
:10CF400000E010E020E041E06EE07EE28F2D0E94E4
:10CF50006D46CF5FDC1314C080912302882371F0EB
:10CF600000E010E021E040E063E07EE28F2D0E94CF
:10CF70006D4660914E058F2D0E940E46E092230271
:10CF8000F394DF5F85E0F8126ECFCF5FC093120697
:10CF9000DF91CF911F910F91FF90EF90DF90CF9095
:10CFA000BF90AF909F908F900895C3E0C114D104BB
:10CFB00009F0ADCFADCF40E050E060E070E088EC2C
:10CFC0009DE239CF4FEB5DE26FEA7DE286EA9DE2BA
:10CFD00032CF40E050E066E97DE28DE89DE22BCF64
:10CFE00040E050E06EE77DE28FE69DE224CF40E036
:10CFF00050E060E67DE283E59DE21DCF47E45DE21F
:10D0000066E37DE286E29DE216CF40E050E068E113
:10D010007DE28FE09DE20FCF40E050E06FEF7CE2D9
:10D0200082EF9CE208CF40E050E065EE7CE284EEC7
:10D030009CE201CF40E050E065ED7CE28CEC9CE2AC
:10D04000FACE61116093280240934E05082E000C21
:10D05000990BAA0BBB0B8C309105A0F5FC0188271E
:10D06000EA56FF4F8F4F0D94E75E82EE97E61FC0A2
:10D0700089EE97E61CC08CE098E619C08EEF97E623
:10D0800016C085E098E613C08AE198E610C083E1F7
:10D0900098E60DC087EF97E60AC080EF97E607C0D5
:10D0A0001092F60B8DEE94E602C08BED97E600979A
:10D0B00049F021E02093420620E040E060E070E08B
:10D0C0000C941F800C944B80CF92DF92EF92FF92D2
:10D0D0000F931F938CE8C82E8FE2D82EE12CF12CF1
:10D0E00001E81FE22CEC33E64BE85BE86CE77FE2FB
:10D0F00087E79FE20E9446821F910F91FF90EF9079
:10D10000DF90CF9008959091200993FB882780F9B4
:10D1100093FF06C081E090915007911101C080E01B
:10D120000895EF92FF920F931F93CF93DF9361E0E7
:10D1300081E00E943881C091140610E0C11118C02E
:10D1400080911306811104C00E944B858111C8C1D2
:10D1500080912302882361F081E090911306911160
:10D1600080E004E024E04BE65FE2612F0E94CC46C1
:10D170008091200982FB002700F982FD07C0D1E0E1
:10D180009091E217913019F0D0E001C0D02F83FBCD
:10D19000EE24E0F883FF03C0B6DFF82E01C0F12CC7
:10D1A000DD2309F458C0C130D9F4809113068130D1
:10D1B00021F40E944B8581119CC180912302882318
:10D1C00009F4A9C181E090911306913009F080E043
:10D1D00000E22EE34FE55FE2612F0E94CC469BC147
:10D1E000C230D9F480911306823021F40E944B851D
:10D1F000811187C180912302882309F48CC181E0C9
:10D2000090911306923009F080E003E02EE344E5AC
:10D210005FE2612F0E94CC467EC1C33009F063C03B
:10D2200080911306833021F40E944B85811175C1D2
:10D2300080912302882309F46EC181E09091130646
:10D24000933009F080E003E02EE34FE45FE2612FCA
:10D250000E94CC4660C18091E217823029F053DFF2
:10D260008823F9F001111DC0C130E9F48091130643
:10D27000813021F40E944B85811159C18091230294
:10D28000882309F45CC181E090911306913009F084
:10D2900080E000E22EE342E45FE2612F0E94CC4690
:10D2A0004EC1D1E001C0D2E0CD131BC08091130666
:10D2B0008C1304C00E944B85811143C180912302CD
:10D2C000882371F081E0909113069C1380E003E0C5
:10D2D0002EE34BE35FE2612F0E94CC46DC2F01C0BE
:10D2E000DC2FDF5F01C0D4E0CD131BC0809113069B
:10D2F0008C1304C00E944B8581112DC180912302A3
:10D30000882371F081E0909113069C1380E003E084
:10D310002EE34FE25FE2612F0E94CC46DC2F01C07A
:10D32000DC2F81E08D0FC81318C0809113068C1379
:10D3300004C00E944B85811118C18091230288236B
:10D3400061F081E0909113069C1380E003E02EE3EE
:10D3500041E25FE2612F0E94CC4682E08D0F409156
:10D36000B60C5091B70C9091770C911107C0209199
:10D37000390230913A0242175307DCF0C81333C028
:10D38000809113068C1304C00E944B858111F7C055
:10D3900080912302882339F181E0909113069C1338
:10D3A00080E000E22EE349E05FE2612F0E94CC467C
:10D3B0001AC0C81318C0809113068C1304C00E94B1
:10D3C0004B858111E6C080912302882361F081E0C2
:10D3D000909113069C1380E003E02EE349EF5EE298
:10D3E000612F0E94CC46DD5FCD1318C080911306DB
:10D3F0008C1304C00E944B858111D5C080912302FB
:10D40000882361F081E0909113069C1380E003E093
:10D410002EE34BEE5EE2612F0E94CC4691E09D0F21
:10D42000EE2009F43BC0F11053C0C91318C080911D
:10D4300013068C1304C00E944B858111BEC08091DD
:10D440002302882361F081E0909113069C1380E011
:10D4500000E22EE34AED5EE2612F0E94CC4682E0BC
:10D460008D0FC81318C0809113068C1304C00E943E
:10D470004B858111ACC080912302882361F081E04B
:10D48000909113069C1380E003E02EE349EC5EE2EA
:10D49000612F0E94CC4693E09D0F1AC0C91316C09D
:10D4A000809113068C1302C00E944B858091230249
:10D4B000882361F081E0909113069C1380E000E2E4
:10D4C0002EE340EC5EE2612F0E94CC4692E09D0F7D
:10D4D0001F5FCF5F153009F031CE9093120680C0E8
:10D4E00081E00E9452808091E005882309F430CECB
:10D4F00077C00E949E8B8091E005882309F45DCE61
:10D500006FC084E698E60E941F4B8091E005882357
:10D5100009F470CE65C0D4E004CF8FE49CE60E948D
:10D520001F4B8091E005882309F482CE59C00E94E8
:10D53000AF8B8091E005882309F4A0CE51C0D2E0E2
:10D54000D0CE8AEA92E60E941F4B8091E0058823A4
:10D5500009F4B4CE45C089EE90E70E941F4B80913C
:10D56000E005882309F4CACE3BC08FE79EE70E94FE
:10D570001F4B8091E005882309F4DFCE31C089E19B
:10D580009FE20E94917F8091E005882309F400CFFB
:10D5900027C088E197E60E941F4B8091E005882311
:10D5A00009F411CF1DC088E390E70E941F4B8091C2
:10D5B000E005882309F422CF13C087EE9EE20E9483
:10D5C000917F8091E005882309F439CF09C08CEE62
:10D5D00093E60E941F4B8091E005882309F44BCF0E
:10D5E000DF91CF911F910F91FF90EF90089560917F
:10D5F000A70C70E080E00C9475B560918E0270917C
:10D600008F02072E000C880B990B0F94015C2AE007
:10D6100037ED43E25CE30F949D5D60938A02709363
:10D620008B0280938C0290938D020895CF93DF93A9
:10D63000EC01CB01BA010F94015C0F94D35B6883BA
:10D64000DF91CF91089580E00C94C0BA66E17BE64B
:10D650008CE29BE60C9476800F94015C0F94D35B74
:10D66000862F0D94A84FEF92FF920F931F93CF93A5
:10D67000DF9300D01F92CDB7DEB7082F7B010E9449
:10D680004B85882331F01092420680E00E94528040
:10D690003BC060913A0670913B066115710551F0EF
:10D6A00010923B0610923A0681E080932302802F6D
:10D6B0000E94D0AD80912302882331F184E0089F3D
:10D6C00080011124075E114F6091E00B7091E10B16
:10D6D000072E000C880B990B0F94015C9B01AC0189
:10D6E000F80160817181828193810F949D5D6983CE
:10D6F0007A838B839C8360E2CE0101960F94F9526A
:10D70000BC01C7010E945A470F900F900F900F90D5
:10D71000DF91CF911F910F91FF90EF90089567E0F7
:10D7200070E380E0A0CF6CEF7FE281E09CCF20E04F
:10D7300040E060E070E00E941F8081E0809342063C
:10D740001092E10B1092E00B08958FE89BE6EFCF6B
:10D7500083E99BE6ECCF2F923F924F925F926F92BC
:10D760007F928F929F92AF92BF92CF92DF92EF9271
:10D77000FF920F931F93CF93DF93CDB7DEB7299717
:10D780000FB6F894DEBF0FBECDBF1C017987688746
:10D7900069011A830983EB82BA01550F880B990B33
:10D7A0000F94015C4B015C0120E030E040E057EC5D
:10D7B0000F94625D18162CF0812C912CA12C27EC73
:10D7C000B22EC501B4010F94CE5B2B013C01B60112
:10D7D000DD0C880B990B0F94015C4B015C0120E080
:10D7E0003EEF4FEF56E40F945F5B87FD07C0812C3F
:10D7F0009EEF992EAA24AA9496E4B92EE885F9857D
:10D8000060817181072E000C880B990B0F94015CCD
:10D810006B017C01C301B2010F94015C9B01AC015F
:10D82000C701B6010F94855A0F94D35B6C837D8337
:10D830008E839F83C501B4010F94CE5B7B018C0165
:10D84000E418F50806091709FB81FF9389809A807F
:10D8500087EEA82E84E6B82ECC80DD80A30192014D
:10D8600068857985C1010E94937F0F9029960FB634
:10D87000F894DEBF0FBECDBFDF91CF911F910F9106
:10D88000FF90EF90DF90CF90BF90AF909F908F90E0
:10D890007F906F905F904F903F902F9008958F9260
:10D8A0009F92AF92BF92CF92DF92EF92FF920F932F
:10D8B0001F93CF93DF9361E081E00E943881D09184
:10D8C0001406C0E0D1111AC080911306811104C062
:10D8D0000E944B85811121C180912302882309F484
:10D8E00013C181E090911306911180E004E024E0DF
:10D8F00047EF5FE26C2F0E94CC4606C1D13011F594
:10D9000080911306813021F40E944B8581110EC154
:10D9100080912302882309F4F7C011E08091130657
:10D92000813009F010E080916802909169020F94B3
:10D93000245000E09C014BEE5FE26C2F812F0E948F
:10D94000FB46E2C0D23011F580911306823021F4FB
:10D950000E944B858111FCC080912302882309F429
:10D96000D3C011E080911306823009F010E080915D
:10D97000B60C9091B70C0F94245000E09C014DED33
:10D980005FE26C2F812F0E94FB46BEC0D33011F5A1
:10D9900080911306833021F40E944B858111EDC0E4
:10D9A00080912302882309F4AFC011E0809113060F
:10D9B000833009F010E080918D0C90918E0C0F94C3
:10D9C000245000E09C0145ED5FE26C2F812F0E9406
:10D9D000FB469AC0D43001F580911306843021F4BF
:10D9E0000E944B858111DEC080912302882309F4B7
:10D9F0008BC011E080911306843009F010E0809113
:10DA0000A70C0F94A84F00E09C014DEB5FE26C2F38
:10DA1000812F0E94FB4678C0D53011F58091130606
:10DA2000853021F40E944B858111DFC08091230253
:10DA3000882309F469C011E080911306853009F04C
:10DA400010E080918E0290918F020F94245000E09C
:10DA50009C0143EB5FE26C2F812F0E94FB4654C078
:10DA6000D630D9F480911306863021F40E944B857C
:10DA70008111CDC080912302882309F445C081E043
:10DA800090911306963009F080E003E02EE348EA17
:10DA90005FE26C2F0E94CC4637C0D730D1F4809122
:10DAA0001306873021F40E944B858111BAC0809102
:10DAB0002302882349F181E090911306973009F001
:10DAC00080E003E02EE34DE95FE26C2F0E94CC463C
:10DAD0001BC0D830C9F480911306883021F40E940D
:10DAE0004B858111A8C080912302882369F081E0D1
:10DAF00090911306983009F080E003E02EE34EE8A1
:10DB00005FE26C2F0E94CC46CF5FDF5FC53009F02B
:10DB1000D9CE89E08093120697C081E00E9452809E
:10DB20008091E005882309F4D7CE8EC0E12C00E077
:10DB300010E027EE33E04AE050E068E672E081EF63
:10DB40009FE209DE8091E005882309F4E1CE7CC0E4
:10DB500081E00E944085E12C03E21BE622E231E0F5
:10DB600040E050E066EB7CE084EE9FE2F4DD8091E3
:10DB7000E005882309F4F0CE67C081E00E9440856B
:10DB8000E12C0DE01BEB2CE830E040E050E06DE8CC
:10DB90007CE089ED9FE2DFDD8091E005882309F4D8
:10DBA000FFCE52C081E00E944085C090A70CD12CCE
:10DBB0001F9287EF882E8AE6982E96E2A92E9BE682
:10DBC000B92EE12CF12C8701EA9420E030E0A90184
:10DBD00067EA7CE089EC9FE20E94937F0F9080913E
:10DBE000E005882309F400CF2FC0E12C0DEF1AE6E1
:10DBF00027EE33E04AE050E06EE872E088EB9FE207
:10DC0000AADD8091E005882309F410CF1DC085EAC4
:10DC10009BE60E941F4B8091E005882309F42ACFE0
:10DC200013C088EA9BE60E941F4B8091E005882381
:10DC300009F43DCF09C08EE991E80E941F4B809105
:10DC4000E005882309F44FCFDF91CF911F910F9109
:10DC5000FF90EF90DF90CF90BF90AF909F908F900C
:10DC600008950E944B85882329F01092420680E097
:10DC70000E94528080E00C949F450E944B8588232F
:10DC800041F020E040E060E070E081E39EE60E9429
:10DC90001F8080E00C947EA54F925F926F927F92DE
:10DCA000AF92BF92CF92DF92EF92FF92CF93DF932A
:10DCB000EB01FC0160817181828193812CE3C22E92
:10DCC000D12CE12CF12CA70196010F94A95EB62E60
:10DCD000A72ECA01B901A70196010F94A95E6B0195
:10DCE0007C01CA01B90128E130E040E050E00F9426
:10DCF000A95E2B013C01C9016DE671E00F94825EC3
:10DD000061157105D9F0AF92BF92DF92CF925F9209
:10DD10004F929F938F937F936F9384E690E39F93AB
:10DD20008F93DF93CF930F9420648DB79EB70E9699
:10DD30000FB6F8949EBF0FBE8DBF61C00097C9F0AB
:10DD4000AF92BF92DF92CF925F924F929F938F9349
:10DD500084E590E39F938F93DF93CF930F94206498
:10DD6000EDB7FEB73C960FB6F894FEBF0FBEEDBF01
:10DD700046C04114510461047104B9F0AF92BF92DE
:10DD8000DF92CF925F924F9288E490E39F938F93BC
:10DD9000DF93CF930F9420648DB79EB70A960FB68A
:10DDA000F8949EBF0FBE8DBF2AC0C114D104E104F8
:10DDB000F104A9F0AF92BF92DF92CF9280E490E39A
:10DDC0009F938F93DF93CF930F942064EDB7FEB7AB
:10DDD00038960FB6F894FEBF0FBEEDBF10C0AF92DD
:10DDE000BF928CE390E39F938F93DF93CF930F9435
:10DDF00020640F900F900F900F900F900F90DF9175
:10DE0000CF91FF90EF90DF90CF90BF90AF907F9039
:10DE10006F905F904F9008952F923F924F925F9234
:10DE20006F927F928F929F92AF92BF92CF92DF922A
:10DE3000EF92FF920F931F93CF93DF93CDB7DEB78F
:10DE40006F970FB6F894DEBF0FBECDBF0E944B8513
:10DE5000882321F081E00E945280F1C02090D90CEB
:10DE60003090DA0C8091DB0C9091DC0C9F8F8E8FC0
:10DE70008091DD0C9091DE0CA091DF0CB091E00C54
:10DE80008A8F9B8FAC8FBD8F4090E10C5090E20C3D
:10DE90006090E30C7090E40C8090E50C9090E60CA0
:10DEA000A090E70CB090E80C60E085E00E9438811B
:10DEB000E0901406F12CDE0111966D01E1100DC009
:10DEC000809123028823E1F0C1010F945A508C0104
:10DED00020E040E069EC70E310C0B1E0EB1210C04C
:10DEE00080912302882361F08E8D9F8D0F945A506C
:10DEF0008C0120E040E06DEB70E38F2D0E946D46B9
:10DF00008A8D9B8DAC8DBD8D8E8B9F8BA88FB98F8D
:10DF1000B601CE014696C0DE92E0E9120BC08091B8
:10DF200023028823B1F000E010E020E040E06BEA3B
:10DF300070E30CC0A3E0EA120CC080912302882396
:10DF400041F0860120E040E068EA70E38F2D0E94F6
:10DF50006D464E8A5F8A688E798EB601CE014696EE
:10DF60009BDEB4E0EB120BC0809123028823B1F05A
:10DF700000E010E020E040E066E970E30CC085E0DE
:10DF8000E8120CC080912302882341F0860120E032
:10DF900040E063E970E38F2D0E946D4620E030E0A1
:10DFA00048EC52E4C501B4010F94665B0F94CE5B5C
:10DFB000CB016AE070E00F94965E9F938F9320E010
:10DFC00030E04AE754E4C501B4010F94665B0F9456
:10DFD000CE5B9F938F937F936F93ABE8B0E3BF9338
:10DFE000AF93DF92CF920F9420640FB6F894DEBF08
:10DFF0000FBECDBFB6E0EB120BC080912302882389
:10E00000B1F000E010E020E040E06BE770E30CC00E
:10E0100087E0E8120CC080912302882341F086013A
:10E0200020E040E068E770E38F2D0E946D46F39496
:10E03000E39495E0F91242CF88E0809312066F9640
:10E040000FB6F894DEBF0FBECDBFDF91CF911F9109
:10E050000F91FF90EF90DF90CF90BF90AF909F9087
:10E060008F907F906F905F904F903F902F9008958A
:10E070000F93CF93DF9361E081E00E943881D091CC
:10E080001406C0E0D11117C080911306811104C09D
:10E090000E944B85811166C080912302882309F478
:10E0A00058C081E090911306911180E004E024E0D3
:10E0B00047E350E34BC0D130C1F480911306813067
:10E0C00021F40E944B85811156C080912302882340
:10E0D00009F43FC081E090911306913009F080E08F
:10E0E00003E02EE346E250E331C0D230B9F4809130
:10E0F0001306823021F40E944B85811146C0809125
:10E100002302882331F181E090911306923009F0C7
:10E1100080E003E02EE348E150E318C0D630C9F4B4
:10E1200080911306863021F40E944B85811137C0FF
:10E1300080912302882369F081E090911306963044
:10E1400009F080E003E02EE342E150E36C2F0E94EF
:10E15000CC46CF5FDF5FC53009F094CF87E0809376
:10E16000120625C081E00E9452808091E00588233C
:10E1700009F492CF1CC08DE39EE60E941F4B809154
:10E18000E005882309F4A1CF12C08CE09FE60E942D
:10E190001F4B8091E005882309F4B1CF08C085E3C7
:10E1A0009BE40E941F4B8091E005882309F2DF91D8
:10E1B000CF910F91089560E070E080E00E9475B506
:10E1C00060E070E081E00E9475B50E945ABB0C943B
:10E1D0004B808F929F92AF92BF92CF92DF92EF923D
:10E1E000FF920F931F93CF93DF9361E081E00E9432
:10E1F0003881D0911406C0E0D1111AC08091130665
:10E20000811104C00E944B858111ABC08091230213
:10E21000882309F474C081E090911306911180E085
:10E2200004E024E04EE051E36C2F0E94CC4667C02E
:10E23000D13011F580911306813021F40E944B8575
:10E24000811198C080912302882309F458C011E0FD
:10E2500080911306813009F010E08091B60C909106
:10E26000B70C0F94245000E09C0140E051E36C2F68
:10E27000812F0E94FB4643C0D23009F580911306DE
:10E28000823021F40E944B8581119AC08091230233
:10E290008823A9F111E080911306823009F010E083
:10E2A00080918D0C90918E0C0F94245000E09C0175
:10E2B00048EF50E36C2F812F0E94FB4620C0D330E3
:10E2C000F1F480911306833021F40E944B85811173
:10E2D0009CC080912302882391F011E08091130665
:10E2E000833009F010E08091A70C0F94794F00E083
:10E2F0009C0140EE50E36C2F812F0E94FB468091E1
:10E30000B60C9091B70C20918D0C30918E0C232B74
:10E3100011F4892BE9F0D430C9F4809113068430CC
:10E3200021F40E944B858111A1C080912302882392
:10E3300069F081E090911306943009F080E000E2EA
:10E340002EE347ED50E36C2F0E94CC4685E001C0E0
:10E3500084E0CF5FDF5FC53009F04ECF80931206B7
:10E360008BC081E00E9452808091E005882309F4EF
:10E370004DCF82C081E00E944085C090B60CD09005
:10E38000B70C1F9263E2862E6BE6962E77EEA72ED1
:10E3900074E6B72E12E2E12EFF24F39400E010E0C1
:10E3A00020E030E0A90166EB7CE087E091E30E9489
:10E3B000937F0F908091E005882309F443CF5CC0E0
:10E3C00081E00E944085C0908D0CD0908E0C1F92F1
:10E3D0003DE0832E3BEB932E47EEA42E44E6B42E75
:10E3E0001CE8E12EF12C00E010E020E030E0A90173
:10E3F0006DE87CE08CEF90E30E94937F0F9080911A
:10E40000E005882309F442CF37C081E00E944085AF
:10E410006091A70C70E080E090E00F94FF5B29EC26
:10E4200038EC48EC5EE30F949D5D0F94D35B1F9234
:10E4300087EF882E8AE6982E9BEFA92E9BE4B92EB3
:10E440006B0114E6E12EF12C00E010E020E030E05A
:10E45000A90167EA7CE08CEE90E30E94937F0F9025
:10E460008091E005882309F434CF06C0A4DE8091B2
:10E47000E005882309F459CFDF91CF911F910F91C7
:10E48000FF90EF90DF90CF90BF90AF909F908F90D4
:10E49000089580E095E290936B0580936A058CE483
:10E4A00091E090936F0580936E0580EC9EEF9093C2
:10E4B0006D0580936C059091660580E2890F863723
:10E4C00040F080EF890F20E431E030936D05209318
:10E4D0006C0510926805809369058FEF809367053E
:10E4E00008958F929F92BF92CF92DF92EF92FF9208
:10E4F0000F931F93CF93DF931F92CDB7DEB7F7D75C
:10E50000882309F4D6C180913A06863214F085E258
:10E5100002C087FD80E0282F082E000C330B3093BB
:10E520003B0620933A06982F990F890F8093660532
:10E530008091CA05882309F4BCC120916C053091F3
:10E540006D050091680510916905020F131FE09099
:10E550006A05F0906B0580916E0590916F05E80E4D
:10E56000F91E01304FE7140768F031952195310904
:10E5700030936D0520936C056CED70E085E090E0C4
:10E580000F948955F7FE15C080916E0590916F0527
:10E5900091958195910990936F0580936E0568E13F
:10E5A00071E085E090E00F94895581E080936705E4
:10E5B00017C081E0E81680E4F80694F06BE470E0A0
:10E5C00084EF91E00F94895580915C058150809390
:10E5D0005C05882311F05DDF6CC11092CA0569C12A
:10E5E00020916E0530916F05C7019A50813093419B
:10E5F00008F098C08F2D992787FD9A950A9765E0B6
:10E6000070E00F94965E812F17FF02C087E0810FA4
:10E61000482F45954595459581E090E0A0E0B0E014
:10E6200004C0880F991FAA1FBB1F4A95D2F7FB0190
:10E63000EE0FFF1FE25AFA4F408151818A010823F1
:10E640001923012B09F419C18095909584239523F2
:10E650009183808384E090E0861B970B4091CB05EB
:10E660005091CC05840F951F9093CC058093CB05DA
:10E6700080915D05815080935D05811103C082E02A
:10E680008093CA05932F9095991F9927991F809180
:10E690006705881F8827881F9817F1F03195219505
:10E6A000310930936F0520936E0520E130E040E0A2
:10E6B00050E060EF7FEF8FEF9FEF0E94143B2091BF
:10E6C0006C0530916D05620F731F70936D0560933B
:10E6D0006C0560E773E021C080916C0590916D0539
:10E6E00091958195910990936D0580936C0520E13A
:10E6F00030E040E050E060EF7FEF8FEF9FEF0E944F
:10E70000143B20916E0530916F05620F731F70935B
:10E710006F0560936E0560E872E085E090E00F940D
:10E720008955ABC0121613060CF0A7C0FDE3FF1A03
:10E7300041E0E41642E0F40608F09FC080916605CF
:10E74000181B103108F099C031952195310930938B
:10E750006F0520936E0560E773E083E090E00F940F
:10E7600089558FEF8093670521E012300CF020E08F
:10E770008EEF810F8C30A0F080916C0590916D052B
:10E7800041E050E01816190614F040E050E030E087
:10E790004217530709F055C091958195910927C0FB
:10E7A000143050F520E030E0A90160EC7FEF8FEFEE
:10E7B0009FEF0E94143B20916C0530916D05620F14
:10E7C000731F70936D0560936C0561157E4F34F473
:10E7D00080E09EEF90936D0580936C0580916C05B1
:10E7E00090916D058130924064F180E092E09093C9
:10E7F0006D0580936C0525C01C301CF120E430E0D1
:10E8000040E050E060E070E0CB010E94143B2091BA
:10E810006C0530916D05620F731F70936D056093E9
:10E820006C0561157E4F34F480E09EEF90936D058A
:10E8300080936C0580916C0590916D0581309240BC
:10E84000A4F68091CA058230C1F480E480935D050E
:10E850008FEF9FEF90935F0580935E059093610526
:10E86000809360059093630580936205909365059E
:10E870008093640581E08093CA05209168053091FA
:10E88000690580916C0590916D05820F931F90939F
:10E8900069058093680520916A0530916B05809128
:10E8A0006E0590916F05820F931F90936B05809377
:10E8B0006A0561E08CE094E00E94AB3580914004F1
:10E8C0008E3130F0809140048E3308F456C05AC027
:10E8D000809142048A30B0F38CE5E82E85E0F82E72
:10E8E0009AE0892E912CB82C8091400490E09401FC
:10E8F0002C5F3F4F281739075CF442E0E40EF11C0F
:10E9000085E0880E911CEEE18E16910461F7DACF56
:10E9100080914204881588F330E0C12CD12CF70196
:10E9200082819381A0E0B0E00C2C04C0B695A7953D
:10E93000979587950A94D2F780FD07C0FFEFCF1A0D
:10E94000DF0A385F303859F7D8CF00E010E0A8016F
:10E95000480D591D8091400490E0481759073CF03C
:10E960008091420490E0841795070CF056C00F5F29
:10E970001F4F0430110559F7E1CF809142048C33C9
:10E9800008F056C08091CA058823B1F080916B05CC
:10E99000482F582F550F550B9A0133272F5F3F4FA4
:10E9A0008091400490E0281739073CF080914204A0
:10E9B000841708F04EC001C0B3D5809140048B305D
:10E9C000D8F40091CB051091CC0569E080E00E945D
:10E9D0002142C8010E94264269E08EE60E9421423F
:10E9E00020915C0583E090E0821B91096FEF7FEF3F
:10E9F0008D5E9E4C0E947B420E944B85882391F144
:10EA00000F90DF91CF911F910F91FF90EF90DF90CA
:10EA1000CF90BF909F908F90C0C527E04B2D400FA7
:10EA2000632F8CE094E039830E94BC3739819FCFFB
:10EA300020E14DE3609166058CE094E00E94BC37D4
:10EA400020E14CE3609166058CE094E00E94BC37C5
:10EA500099CF6091690502E022E08CE094E00E9489
:10EA6000FD37ABCF0F90DF91CF911F910F91FF90AA
:10EA7000EF90DF90CF90BF909F908F90089561E7C7
:10EA800072E782E079D5ECE5F5E088E3828783E000
:10EA9000808380E48183138212821582148217821C
:10EAA000168211861086F5DC82E190E090933B0699
:10EAB00080933A0608958F929F92AF92BF92CF9221
:10EAC000DF92EF92FF926091870520E030E090E0C6
:10EAD00080E0F901E45AFA4FC7A4CC2011F061E0BC
:10EAE000620F8C29722F7295707F40E050E0D12C1C
:10EAF000E12CF12C46015701042E04C0B694A794D2
:10EB0000979487940A94D2F780FE08C0E92FF0E02A
:10EB1000E45AFA4FA72FA42BA2AB9F5F4F5F5F4F22
:10EB20004530510539F72F5F3F4F2330310589F6C6
:10EB30006093870540E050E020E090E0A0E0B0E086
:10EB40006C017D01042E04C0F694E794D794C79419
:10EB50000A94D2F7C0FE05C0209385052AE335E06C
:10EB600007C02E504F5F5F4F4530510549F7F4CF36
:10EB7000422F3150A0F0225F6C017D01032E04C0B2
:10EB8000F694E794D794C7940A94D2F7C0FEF0CFD6
:10EB90004093860580918805823069F403C02093F4
:10EBA0008605F8CF80918405181614F08CEF01C00B
:10EBB00084E080938405FF90EF90DF90CF90BF902A
:10EBC000AF909F908F90089580E090E0FC01E45A10
:10EBD000FA4F168203968E319105C1F70895ECE540
:10EBE000F5E010828AE0818383E080A78FE084A72C
:10EBF0008FE187A780AB81AB5EDFE6CF1F93CF931A
:10EC0000DF93EC01162FE0DF80915F058093810593
:10EC100087E38093820586E0809383056AE070E055
:10EC200088EE93E00F94895590915E0591509093F2
:10EC30005E05992351F010928005188310925F05AC
:10EC400010923B0610923A0601C01882DF91CF91D4
:10EC50001F9108952F923F925F926F927F928F92B1
:10EC60009F92AF92BF92CF92DF92EF92FF920F935B
:10EC70001F93CF93DF931F92CDB7DEB784E08093CD
:10EC8000230280913C06882309F470C280913A06E1
:10EC900090913B068E31910514F08DE190E097FF45
:10ECA00002C080E090E090933B0680933A06880F84
:10ECB000991F880F991F20915F05422F022E000C8B
:10ECC000550B4817590774F42D5FAC01421B5109CD
:10ECD00027FD5395423051051CF020935F0502C07B
:10ECE00080935F0520915F05422F022E000C550B8B
:10ECF000841795077CF42350422F022E000C550BED
:10ED0000481B590B423051051CF020935F0502C08F
:10ED100080935F058091CA05882309F427C220915A
:10ED20009E05222349F090919D05920F90939D0599
:10ED3000933F14F410929E05823070F081508093BE
:10ED4000CA05823011F44BDF11C2843609F00EC2BD
:10ED500081E08093CA050AC280918A058F5F809303
:10ED60008A054091880590E0242F30E0359527955D
:10ED7000281739070CF0B3C090919F0581E08927CF
:10ED800080939F0510928A05442309F4A8C09091AE
:10ED9000840580915C05890F20918505821724F0F8
:10EDA000209186052817D4F491959093840520919D
:10EDB0005D052B5F20935D0580935C058091870541
:10EDC0003AE08302C0011124820F911D27FD9A951C
:10EDD000C99724F064E18AEC95E010DF90918405F6
:10EDE00080915C05890F80935C058091880588235C
:10EDF00009F475C024E130E040E050E060E070E0EC
:10EE0000CB010E94143B672B682B692B09F067C06C
:10EE1000E2E6F5E080E090E0208121115AC09C01FB
:10EE2000220F331F8901080F191FC801805A9A4FFA
:10EE3000892B09F454C02091880530E02F5F3F4FA3
:10EE4000032E000C440B550B60E070E0CB010E94D8
:10EE5000143BFB01E45AFA4F42A9242F30E0B4E0FE
:10EE600035952795BA95E1F7F901E259FC4F808174
:10EE700090E0045A1A4F4F7050915C056EE0469F27
:10EE8000500D1124452FFC01E559FC4F5081450FD1
:10EE9000FC01E859FC4F90819695842F890FF80169
:10EEA000848380915D0582502F5F3F4FFAE02F9F52
:10EEB000800D1124F801858322E030E040E050E02D
:10EEC00060E070E0CB010E94143B6E5FF801668346
:10EED00006C0019633968A30910509F09DCF909136
:10EEE0008005992341F080917F05890F80937F05EC
:10EEF00087FD1092800580918005882309F4A2C0C7
:10EF000020917F05E0915D052E170CF49BC0022E29
:10EF1000000C330B0E2E000CFF0BCF014D96821709
:10EF200093070CF48FC010915C05E0907E05CE2C09
:10EF30000E2C000CDD08C601811B910917FD93956D
:10EF40006EE070E00F94965EF62E653008F07AC0A1
:10EF50002E1B3F0BC90102966AE070E00F94965E8B
:10EF6000062F633008F06EC0812C912C54018394DD
:10EF70000F2C04C0880C991CAA1CBB1C0A94D2F745
:10EF8000A62F660FBB0BBD01645A7A4FFB0197A5F4
:10EF9000892F882109F456C0FD01E259FC4FE08118
:10EFA0004E2F50E0812FFEE0FF9E800D11249A012C
:10EFB00025593C4FF901F080F80EEF140CF442C0D3
:10EFC000FA01E859FC4F1081412F50E04F0D511DBF
:10EFD000F7FC5A95C416D506ACF510928005282D7D
:10EFE00020952923FB0127A723E030E02A1B3B0BB8
:10EFF0008091CB059091CC05280F391F3093CC051B
:10F000002093CB056AE070E088E290E00F94895588
:10F0100020915D05FAE00F9F200D1124912F969508
:10F020008F2D890F8550809381052093820584E080
:10F03000809383058091880581508093880588237B
:10F0400021F039DD02E615E012C084E18093CA05A3
:10F05000BBDDF8CF8291890F808380346CF0F8019A
:10F0600010820D5F1F4FF5E000381F07E9F0F8012F
:10F0700090819923B1F3EECF87339CF3F801329757
:10F08000208180915F05281764F3022E000C330B5A
:10F09000082E000C990B0A968217930714F368E761
:10F0A0008AEC95E0ABDDDDCF80919E05811124C017
:10F0B00024EF31E040E050E060E070E0CB010E94DE
:10F0C000143B672B682B692BB9F422E030E040E059
:10F0D00050E060E070E0CB010E94143B672B682B8E
:10F0E000692B09F099C18FEF80939E05813009F457
:10F0F00095C18FE780939D05809180058823B1F1AC
:10F1000080919E05882391F180917F05873074F569
:10F1100020917E0580919D05281744F1022E000C58
:10F12000330B082E000C990B0C9682179307F4F002
:10F1300010929E05109280058091CB059091CC0590
:10F140000A969093CC058093CB056AE070E088E244
:10F1500090E00F94895580919D058F5F8093810584
:10F1600081E08093820584E080938305809144064A
:10F1700082FF04C080918905815001C08AE080939C
:10F1800089050E944B858823C1F08091CA058111B1
:10F1900003C01092890511C0813079F480918005F7
:10F1A00081110BC080915F058B5F80937E0584E3A6
:10F1B00080937F058CEF8093800580918905811174
:10F1C00001C0EBD161E08CE094E00E94AB3530915E
:10F1D0005D05632F032E000C770B80918705AB0133
:10F1E0002AE08202400D511D1124425051098091A4
:10F1F000400490E0841795072CF080919E058111C2
:10F200006BC06FC08091420490E086179707ACF303
:10F21000FEE66F2EF3E07F2EC12CD12CF30121915D
:10F220003F01432F032E000C550BBA01695F7F4F3E
:10F230008091400490E0681779074CF4365FFFEF47
:10F24000CF1ADF0A23E0C216D10441F7D6CF80914E
:10F25000420490E0841795078CF310915C0546E416
:10F26000542E510EA12CB12CC601845A9A4F4C0138
:10F27000822F90E01C01220C331CF40187A590E042
:10F28000A0E0B0E00A2C04C0B695A79597958795A5
:10F290000A94D2F780FF19C080919F057101E80E92
:10F2A000F11CC701E4E0880F991FEA95E1F7AC0172
:10F2B0004A5B5E4C7A0108E022E0432F612F8CE02C
:10F2C00094E039830E94D5353981125F5FEFA51A2A
:10F2D000B50A1511D2CFB2CF80914004883008F41E
:10F2E0009FC08091CA05882369F0909140049F33A4
:10F2F00048F490914204973328F0823008F49EC07D
:10F3000081FD9CC0809180058823B1F040917F05EC
:10F31000242F042E000C330BB9016D5F7F4F8091B9
:10F32000400490E0681779073CF08091420490E037
:10F33000821793070CF090C000E010E0F801E45A47
:10F34000FA4F8681882399F04581842F042E000C82
:10F35000990B2091400430E08217930744F0029704
:10F360002091420430E0281739070CF07DC00D5F72
:10F370001F4F0E31110511F7809183058823B1F0DD
:10F3800040918205242F042E000C330BB9016A5FD3
:10F390007F4F8091400490E0681779073CF080919E
:10F3A000420490E0821793070CF066C08091CA0572
:10F3B000811101C0B5D0809140048A3008F06EC040
:10F3C0000091CB051091CC0569E080E00E942142BC
:10F3D000C8010E94264280915E05882309F45EC020
:10F3E00011E060E1C62ED12C80915E05811708F4F2
:10F3F00055C0B601611B7109660F660F660F71E398
:10F40000E72E71E3F72E05E021E041E08CE094E087
:10F410000E94D5351F5FE8CF81E066CE83EF6ACECC
:10F4200029E1E22E21E3F22E05E022E042E06091A4
:10F430009D058CE094E00E94D53553CF96E3E92EEC
:10F4400091E3F92E08E022E047E360915F058CE04C
:10F4500094E00E94D53556CF24E060917E058CE083
:10F4600094E00E94DC3768CF425023E064818CE056
:10F4700094E00E94DC377BCF83E2E82E81E3F82E14
:10F4800007E022E0609181058CE094E00E94D53590
:10F490008091830581508093830588CF0F90DF9101
:10F4A000CF911F910F91FF90EF90DF90CF90BF9081
:10F4B000AF909F908F907F906F905F903F902F9034
:10F4C0000895CF93DF936AE276E784E155D0CCE5E7
:10F4D000D5E083E08A838AE08DA71CA280DB1B82B3
:10F4E00010923B0610923A06DF91CF9108958091D9
:10F4F0003C06882319F082E080935B0584E08093CA
:10F5000023028091CA05882349F090915B058FEF13
:10F51000890F80935B0581E019160CF080E0089557
:10F520000F9380914004853228F5809142048B31FD
:10F5300008F160E08CE094E00E94AB3509E028E33C
:10F540004BE164E28CE094E00E944D3861E08CE095
:10F5500094E00E94AB350E949486882359F063E2C0
:10F5600085E20E9421426FEF7FEF86EA91E30F91DF
:10F570000C947B420F910895FB011092CC051092E0
:10F58000CB058093CA0520E040E060E070E0CF0149
:10F5900056D581E08093420608951092420680E09D
:10F5A00081C5809161059091630589130DC080919B
:10F5B000620590916405891714F02FEF01C021E0D6
:10F5C000820F8093620508C0891714F02FEF01C0E5
:10F5D00021E0820F8093610589131BC02091C9052A
:10F5E00021502093C90530E0832F90E0DC01AA0F61
:10F5F000BB1FA45ABA4F880F991FFC01E25AFA4F59
:10F600008581968116969C938E9315973F5F23175D
:10F6100058F70895EF92FF921F93CF93DF931091C5
:10F62000C90520915E05E22E022E000CFF083091E4
:10F630005D05C32F032E000CDD0BE4E6F5E040E092
:10F64000411709F446C0CF010397DC019C91BF012B
:10F6500061507109DB018C9198131DC0692F092E2F
:10F66000000C770B61507109C617D70711F03913D9
:10F670002DC09081BF0162507109DB018C91582F20
:10F6800098170CF4592F25170CF189170CF4892FB2
:10F690008217E4F020C0BF0162507109DB015C9168
:10F6A000652F052E000C770B61507109E616F706E1
:10F6B00011F025130BC0582F98170CF4592F35173C
:10F6C0002CF089170CF4892F83172CF44F5F329696
:10F6D000B7CF80E001C081E0DF91CF911F91FF9013
:10F6E000EF90089528E130E040E050E060E070E005
:10F6F000CB010E94143B60935D052AE030E040E0BE
:10F7000050E060E070E0CB010E94143B60935E0526
:10F7100081DF8111E7CF089590915C05811102C0CE
:10F720008FEF01C081E0980F937090935C058091FA
:10F73000C9058F5F8093C90590E0FC01EE0FFF1FA4
:10F74000E45AFA4F2091C6052583880F991FFC01C2
:10F75000EE59FA4F8091C805808308951F93CF9387
:10F76000DF93CCE5D5E080E091E09093C6058093EF
:10F77000C50580E095E09093C8058093C705188281
:10F780001092C9051D8215E01E8381E0C5DF1B8331
:10F7900010923B0610923A061C82DF91CF911F9186
:10F7A0000895EF92FF920F931F93CF93DF93809171
:10F7B000C905843008F4DEC090E0FC01EE0FFF1FA5
:10F7C000E65AFA4F3581FC01EE0FFF1FE45AFA4F5B
:10F7D0006581AC0142505109361739F0C0E0880FFD
:10F7E000991FFC01E05AFA4F82C0F12CDC01AA0FEC
:10F7F000BB1FAE59BA4F880F991FFC01E05AFA4F50
:10F800008F2D90E0841795070CF0B4C0BC01660FF3
:10F81000771F645A7A4FEB016D818C01000F111F25
:10F82000025A1A4FE8012D816217F1F0722F621708
:10F830000CF4762F3717ECF126170CF4262F23172C
:10F84000C4F1880F991F8E599A4FEC01288191E0DD
:10F85000808128170CF090E081E06C9162170CF425
:10F8600080E0981731F188C0361323C07C91208145
:10F870008C01000F111F0C591A4FE8016881880F85
:10F88000991F8E599A4FEC018881122F72170CF430
:10F89000172F982F86170CF4962F911754F0922F4C
:10F8A00027170CF4972F68170CF4862F98170CF075
:10F8B00063C0F394A5CF7C01DFEFED1AFD0A8C0144
:10F8C000000F111F0E591A4FD8017C918C01000FA7
:10F8D000111F0C591A4FD8012C91721729F1A081D0
:10F8E000B22F72170CF4B72FAB173CF4CF5F8C2FED
:10F8F00090E084179507FCF23DC027170CF4272FE2
:10F900002A17A4F3880F991FDC01A45ABA4F159641
:10F910002C9191E023170CF090E081E062170CF439
:10F9200080E0981719F328C020812713DFCFD70173
:10F93000AA0FBB1FA45ABA4F15962C91880F991F76
:10F94000DC01A45ABA4F15968C91762F36170CF419
:10F95000732F982F82170CF4922F97173CF2962F43
:10F9600063170CF4932F28170CF4822F98170CF4BC
:10F97000BDCF02C080E001C081E0DF91CF911F9137
:10F980000F91FF90EF900895BF92CF92DF92EF9288
:10F99000FF920F931F93CF93DF931F92CDB7DEB7E4
:10F9A000A6DD882309F486C08091C5059091C6051F
:10F9B000392F4091C7055091C80520915C05213031
:10F9C00061F02CF4211116C0CA01C3970AC022307D
:10F9D00031F0233079F4C39709C0C39607C0CA0138
:10F9E000C3969093C8058093C70504C09093C6053D
:10F9F0008093C5051091C6050091C805311303C059
:10FA0000051709F457C0183110F40A3048F0109265
:10FA1000CA0568E270E080E991E00F9489554AC018
:10FA20008091C90590E0FC01EE0FFF1FE45AFA4FE8
:10FA30001583880F991FFC01EE59FA4F00838091BE
:10FA40003A0690916005282F291B39F080936005B4
:10FA500081E012160CF080E05FDE80915F05882364
:10FA600021F0815080935F0501C09BDD9ADE8111FA
:10FA7000CECF80915D0518131DC080915E050813DF
:10FA800019C06CED70E085E090E00F94895568E155
:10FA900071E085E090E00F9489558091CB059091BD
:10FAA000CC0501969093CC058093CB0582E08093A2
:10FAB0005F0518DE61E08CE094E00E94AB35809138
:10FAC0004004893058F4E090CB05F090CC0567E015
:10FAD00080E00E942142C7010E94264206E32CE7F3
:10FAE00049E062E08CE094E00E94FD3710E08091F4
:10FAF000C90530914004181708F084C0412F50E028
:10FB0000BA01660F771FFB01E45AFA4FA581FB018A
:10FB1000E25AFA4F2581CA010396A21351C0FB0194
:10FB2000EC59FA4F2081880F991FFC01E45AFA4FD3
:10FB3000C080DC2CC2160CF4D22E8D2D95E08902EB
:10FB4000A0011124425F5F4F832F90E048175907AF
:10FB50000CF456C02C150CF4C22EEC2DF5E0EF027F
:10FB600090011124265F3F4F8091420490E02817B6
:10FB700039070CF045C08C2D880F880F8C0DEBE0F9
:10FB8000BE2EB80ECB018F599A4F7C01DC14C4F104
:10FB90002B2D0B2C000C330BA9014D5F5F4F809177
:10FBA000400490E0481759073CF08091420490E0EF
:10FBB000821793070CF053C0C39495E0B90EE6CFBB
:10FBC000880F991FFC01E45AFA4F8081982F990FF2
:10FBD000990F890F5BE0E52EE80E4E2D0E2C000CE0
:10FBE000550BBA016D5F7F4F832F90E0681779073F
:10FBF0003CF06091420470E0641775070CF03EC061
:10FC00001F5F75CF40915E05842F880F880F480FC6
:10FC1000455F642F042E000C770BFB013396832F76
:10FC200090E0E817F9073CF08091420490E08617D5
:10FC300097070CF045C08091CA05811101C070DCA6
:10FC40002AD7882309F44AC00F90DF91CF911F91E2
:10FC50000F91FF90EF90DF90CF90BF909ECCF70177
:10FC60006081862F880F880F680F6C5F04E024E0A6
:10FC70004B2D8CE094E00E944D389ECFD22EA217DF
:10FC80000CF4DA2EC22E2A170CF4CA2EFD2CFF0C0F
:10FC9000FF0C8F2D8D0D30E094E0F92EF80ECD1471
:10FCA0000CF4AECF6F2D630F04E024E04E2D8CE0FA
:10FCB00094E039830E944D38D39439813B5FEFCF74
:10FCC00060915D05862F880F880F680F6C5F04E0D8
:10FCD00024E08CE094E00E94FD37ADCF0F90DF91DF
:10FCE000CF911F910F91FF90EF90DF90CF90BF9039
:10FCF000089564EC7CE781E03FDC30DDF3CC0F93CA
:10FD00001F93CF93DF9361E081E0B2D2D0911406CC
:10FD1000C0E0D11116C080911306811103C0BBD67B
:10FD200081119AC080912302882309F43CC081E0AC
:10FD300090911306911180E004E024E04FEF51E32D
:10FD40002FC0D130B1F480911306813019F4A3D6BD
:10FD500081118AC080912302882329F181E090914A
:10FD60001306913009F080E003E02EE34DEE51E3FD
:10FD700017C0D230C1F480911306823019F48BD6AB
:10FD800081117CC080912302882369F081E09091E9
:10FD90001306923009F080E003E02EE34EED51E3CC
:10FDA0006C2F0E94CC4634D1182FD330D1F48091DF
:10FDB0001306833019F46FD681116AC08091230233
:10FDC000882309F477C081E090911306933009F0FD
:10FDD00080E000E22EE34FEC51E36C2F0E94CC4612
:10FDE00069C0811169C0D430B1F4809113068430A8
:10FDF00019F451D6811153C080912302882319F13F
:10FE000081E090911306943009F080E000E22EE347
:10FE100041EC51E315C0D530B1F480911306853023
:10FE200009F444C080912302882369F081E0909115
:10FE30001306953009F080E000E22EE340EB51E339
:10FE40006C2F0E94CC4686E0CF5FDF5FC53009F0A3
:10FE500060CF809312063BC081E024D18091E00501
:10FE6000882309F45FCF33C08EE493E50E941F4BD3
:10FE70008091E005882309F46DCF29C08EE991E8CF
:10FE80000E941F4B8091E005882309F47BCF1FC09F
:10FE9000E2D28091E005882309F490CF18C0DED229
:10FEA0008091E005882309F4A7CF11C0F4D5811112
:10FEB00005C0B8CF112339F284E0C6CF0E9401DF1C
:10FEC00081E028D28091E005882309F4ABCFDF914F
:10FED000CF911F910F910895E091E105E63000F573
:10FEE00081E08E0F8093E10580913A0690913B0668
:10FEF000A0E0B0E0309114062091120648E0E49FA3
:10FF0000F0011124EE51FA4F40913506509136061A
:10FF10005183408382839383A483B583368327836D
:10FF200008950D943C442F923F924F925F926F92AE
:10FF30007F928F929F92AF92BF92CF92DF92EF9279
:10FF4000FF920F931F93CF93DF9300D000D0CDB7D4
:10FF5000DEB71C012B833C834D835E8369837A83E8
:10FF6000BBDF83E0809323023092DF052092DE0521
:10FF700069817A817093DD056093DC052B813C817A
:10FF80004D815E812093D8053093D9054093DA05E1
:10FF90005093DB05E092D405F092D5050093D60589
:10FFA0001093D705D0923B06C0923A06B09236061F
:10FFB000A09235069092D3058092D2058C8D8093C5
:10FFC000D10526960FB6F894DEBF0FBECDBFDF91E8
:10FFD000CF911F910F91FF90EF90DF90CF90BF9046
:10FFE000AF909F908F907F906F905F904F903F90D9
:10FFF0002F900895FB01908181E08927808383E021
:020000021000EC
:10000000809323024115510511F0FA0119940895C6
:100010008091870E9091840E891B8F7071F490915E
:10002000200992FB882780F992FD08C081E0909119
:10003000E217913019F080E0089581E00895E09191
:100040003506F0913606E817F90721F1309145069B
:1000500037FD1092450690933606809335067093CF
:100060003B0660933A0640931406209312068B5A7F
:10007000944821F4109242061092E1050E940D4628
:1000800082E08093230281E08093E00510923D0698
:100090001092CD05089520E040E060E070E08BEA2A
:1000A00094E8CDCFE091E105EE23F9F0E150E09343
:1000B000E10598E0E99FF0011124DF01AE51BA4F4C
:1000C00017962C911797811108C016964C91169788
:1000D00012966D917C91139703C040E060E070E050
:1000E000EE51FA4F80819181AACFD5CFCF93DF9384
:1000F000FC01EB0180913A0690913B0697FF04C00A
:1001000010923B0610923A064091D4055091D505C5
:100110006091D6057091D70580913A0690913B0683
:10012000092E000CAA0BBB0B481759076A077B075F
:1001300024F450933B0640933A068091230288238F
:10014000D1F020913A0630913B068091D8059091EC
:10015000D905A091DA05B091DB05BC01CD01620F94
:10016000731F811D911D1995BC018091DE05909131
:10017000DF050E945A4780912F06811108C08091A7
:10018000D105882389F180912302882369F1809128
:10019000DC059091DD05009791F020913A063091B1
:1001A0003B064091D8055091D9056091DA057091D0
:1001B000DB05420F531F611D711DFE011995E09172
:1001C000D205F091D305309741F08091D10581118E
:1001D00003C080912F06811119955DD4882321F0E9
:1001E00080E0DF91CF915ECFDF91CF9108950F93A3
:1001F0001F93CF93DF9380912302882359F060915E
:10020000CE057091CF0500E010E020E041E081E0F4
:100210000E946D468091D00581111CC081E08093C1
:10022000D005C0913506D091360620E040E060E070
:1002300070E087EF90E803DF0E9495FB1092D005F5
:1002400020E040E060E070E0CE01DF91CF911F91AF
:100250000F91F5CEDF91CF911F910F9108950097E7
:1002600011F483E192E39093CF058093CE05BFCF45
:10027000282F1092340680913A0690913B068130E7
:10028000904820F010923B0610923A0680913C066E
:10029000882331F080913A06809313061092E0058E
:1002A000809112061816BCF4082E000C990B821BC4
:1002B000910920911306022E000C330B28173907E1
:1002C00054F097FF02C080E090E080931306909373
:1002D0003B0680933A06809113066623C1F0909105
:1002E0001406891714F48093140620911406022E24
:1002F000000C330B2C5F3F4F482F082E000C550B82
:100300002417350734F4845080931406089580939D
:1003100014060895882361F063E972E084E690E0B2
:100320000F9489556AEB72E084E690E00D9489554C
:1003300068EB71E084E190E00D948955CF92DF92F3
:10034000EF92FF92CF93DF93A6D3882361F00E94B0
:100350004CA51092420680E0DF91CF91FF90EF9084
:10036000DF90CF909FCE81E080934206C0913A0605
:10037000D0913B06209709F442C010923B061092A0
:100380003A06BE010D2E000C880B990B0F94015CF0
:100390002091210E3091220E4091230E5091240E77
:1003A0000F949D5D20915D0D30915E0D40915F0D2C
:1003B0005091600D0F94865A6B017C0120E030E073
:1003C00040E050EC0F94625D87FD19C020E030E002
:1003D00040EA50E4C701B6010F945F5B18167CF049
:1003E000BE0182E00E94D0ADC0925D0DD0925E0D44
:1003F000E0925F0DF092600D82E080932302809185
:1004000023028823C9F08DE59DE00F948650BC013E
:1004100084E092E30E945A4760915D0D70915E0DF9
:1004200080915F0D9091600DDF91CF91FF90EF90E3
:10043000DF90CF900C947E48DF91CF91FF90EF90AA
:10044000DF90CF90089521E02093D0050F94414490
:100450001092D00508950E943BDB5CCF0E9492E988
:1004600059CF20913A0630913B062115310559F0BC
:1004700081E0121613060CF080E08093CD051092F7
:100480003B0610923A068091CD0508954F925F92F7
:100490006F927F928F929F92AF92BF92CF92DF9294
:1004A000EF92FF920F931F93CF93DF931F921F92B0
:1004B000CDB7DEB75C014A01390128018701760119
:1004C00069837A83CEDFD82EE6D2C82E69817A81FD
:1004D000811104C0809123028823F9F092014D2DEF
:1004E000C5010E942548CC20C1F0DD2011F0F401A7
:1004F00001C0F3010F900F90DF91CF911F910F91E9
:10050000FF90EF90DF90CF90BF90AF909F908F9033
:100510007F906F905F904F9019940F900F90DF91A4
:10052000CF911F910F91FF90EF90DF90CF90BF90F0
:10053000AF909F908F907F906F905F904F900895B5
:10054000FC0180810895FC01849108954F925F928F
:100550006F927F928F929F92AF92BF92CF92DF92D3
:10056000EF92FF920F931F93CF93DF936C017B0168
:100570005A012901672B31F088248394912CC0E023
:10058000D0E019C0F8011182108227C03701680C31
:10059000791C76946794E3012197A201BE01C601FC
:1005A000F50119951816190654F0892BC9F0430165
:1005B000FFEF8F1A9F0AE814F90440F702C07E018A
:1005C000FACFCE15DF0530F4CE01029688169906D3
:1005D00020F02196F801D183C0838FEF9FEF05C0F3
:1005E000F801D183C08380E090E0DF91CF911F912B
:1005F0000F91FF90EF90DF90CF90BF90AF909F90C2
:100600008F907F906F905F904F9008958F929F9200
:10061000AF92BF92CF92DF92EF92FF920F931F9310
:10062000CF93DF93EC016B017A01FB01199587FDF4
:1006300006C0082F10E020E030E0219620C1982F5E
:10064000907E903CC1F4082F0F7110E020E030E064
:100650004801590186E0880C991CAA1CBB1C8A958C
:10066000D1F7CE010196F60119958F73950184019A
:10067000082B229604C1982F907F903E19F58F7019
:10068000882E912CA12CB12C16E0880C991CAA1C48
:10069000BB1C1A95D1F7CE010196F60119958F73FF
:1006A000882A06E0880C991CAA1CBB1C0A95D1F765
:1006B000CE010296F60119958F7395018401082BDE
:1006C0002396DDC0982F987F903F81F58770882E04
:1006D000912CA12CB12CF6E0880C991CAA1CBB1CF7
:1006E000FA95D1F7CE010196F60119958F73882AF4
:1006F000A6E0880C991CAA1CBB1CAA95D1F7CE01B8
:100700000296F60119958F73882AB6E0880C991C19
:10071000AA1CBB1CBA95D1F7CE010396F601199518
:100720008F7395018401082B2496A9C0982F9C7F74
:10073000983FE9F58370882E912CA12CB12C56E0BE
:10074000880C991CAA1CBB1C5A95D1F7CE010196A6
:10075000F60119958F73882A66E0880C991CAA1CEB
:10076000BB1C6A95D1F7CE010296F60119958F73DD
:10077000882A76E0880C991CAA1CBB1C7A95D1F7B4
:10078000CE010396F60119958F73882AE6E0880C4E
:10079000991CAA1CBB1CEA95D1F7CE010496F60160
:1007A00019958F7395018401082B259668C0982FA1
:1007B0009E7F9C3F09F04AC08170882E912CA12C0D
:1007C000B12C86E0880C991CAA1CBB1C8A95D1F719
:1007D000CE010196F60119958F73882A96E0880C50
:1007E000991CAA1CBB1C9A95D1F7CE010296F60162
:1007F00019958F73882A26E0880C991CAA1CBB1CAB
:100800002A95D1F7CE010396F60119958F73882AA0
:1008100036E0880C991CAA1CBB1C3A95D1F7CE0176
:100820000496F60119958F73882A46E0880C991C66
:10083000AA1CBB1C4A95D1F7CE010596F601199565
:100840008F7395018401082B269619C0982F907CF0
:10085000903849F4082F007C003871F42196CE01BD
:10086000F6011995F7CF082F0E7F0D3F28F021963E
:10087000CE01F6011995F7CF00E010E09801E114E0
:10088000F10429F0F7010083118322833383CE0121
:10089000DF91CF911F910F91FF90EF90DF90CF905C
:1008A000BF90AF909F908F9008951F93CF93DF9349
:1008B00000D01F92CDB7DEB710E0AE014F5F5F4FA3
:1008C00060EA72E8A3DE49815A816B817C81452B05
:1008D000462B472B11F01F5FF0CF812F0F900F9009
:1008E0000F900F90DF91CF911F9108951F93CF9399
:1008F000DF9300D01F92CDB7DEB710E0AE014F5F9F
:100900005F4F63EA72E882DE49815A816B817C81A4
:10091000452B462B472B11F01F5FF0CF812F0F90F7
:100920000F900F900F90DF91CF911F910895FC01D0
:10093000A081B1811C92A281B3818C918F5F8C9335
:100940000280F381E02D80816CE0689F600D1124AE
:1009500080E00C9421421092340680912F06109270
:100960002F06882349F020E040E060E070E081E954
:1009700098E665DB0C94DD452091680230916902B0
:1009800040913A0650913B06C901840F951F2436C9
:10099000310551F44730510514F0069720C04A3F05
:1009A0005F4F64F506961BC02436310524F4853666
:1009B000910524F504C08436910524F41FC08A30C3
:1009C00091053CF0883E43E094072CF087EE93E0DD
:1009D00002C08AE090E02817390731F40DC08A3050
:1009E000910584F78AE090E0909369028093680211
:1009F00010923B0610923A060C94154284E690E061
:100A0000E1CFCF93DF931F92CDB7DEB78091D108AE
:100A1000811103C083E199E02FC0211103C081ED52
:100A200098E02AC08DE0815048F0440F411DE82F26
:100A3000F0E0ED5EF64F90814927F5CF80912606D4
:100A40008417A9F04093260681ED98E069832DDF95
:100A500090E06981861B910997FF02C080E090E0D9
:100A6000809337061092380688E0809325028091A3
:100A7000380690E08F52974F0F90DF91CF910895F5
:100A8000809334061092300610923106109232068E
:100A900010923306089580912F0610922F06089524
:100AA0007F928F929F92AF92BF92CF92DF92EF92FE
:100AB000FF920F931F93CF93DF93CDB7DEB72897A5
:100AC0000FB6F894DEBF0FBECDBF7C014B016A01AB
:100AD0005901FB0180816CE0689F600D1124F701D2
:100AE0008081982F990F890F880F0E942142C1148D
:100AF000D10409F496C0FE82ED8298868F8201119E
:100B000003C01C2D0D2D74C09D2C0C2D1D2DD12C22
:100B100088248394AE014F5F5F4FB5018C2D992DD2
:100B200075DDC82E992E89819A81AB81BC8177248D
:100B300073940097A105B105C9F0712C803291051D
:100B4000A105B10581F0AC01BD014D52510961090A
:100B50007109423051056105710540F08B97A1057F
:100B6000B10589F503C0DD2009F455C0F7012081E6
:100B70008D2D90E0820F911D46972CF0253018F0B6
:100B8000CE010596D4DE372D3825D30EF7018081AE
:100B90008D0D8083DD2089F0DA94AE014F5F5F4FC9
:100BA000B501C80133DD8C0169817A818B819C811B
:100BB0004FEF5FEF0E942C42EDCF711032C00C2D31
:100BC000192DD12CA7CFD3940115110509F0A2CF6F
:100BD0000C2D192D9FCF4FEF5FEF0E942C42F70194
:100BE00020812F5F2083253118F0CE0105969FDEEE
:100BF000AE014F5F5F4FB501812F902F07DD182F9A
:100C0000092F69817A818B819C816115710581052C
:100C1000910509F706C00115110589F20F5F1F4FF5
:100C2000D3CF28960FB6F894DEBF0FBECDBFDF91AD
:100C3000CF911F910F91FF90EF90DF90CF90BF90D9
:100C4000AF909F908F907F900895AF92BF92CF9278
:100C5000DF92EF92FF920F931F93CF93DF931F9238
:100C60001F92CDB7DEB75C016B017A013FDE182F12
:100C7000E114F10419F0C70139DE01C080E01A82E5
:100C80001982C114D104C1F4412F50E090E09A01BF
:100C9000280F391F263131057CF425E130E0241B73
:100CA000350B281B390B37FF02C02F5F3F4F35959F
:100CB00027952A8381E0898301E023EA32E8A501B0
:100CC000BE016F5F7F4FCE010296EADEC114D104F0
:100CD00089F08A81882321F01A8289818F5F898334
:100CE00000E020EA32E8A601BE016F5F7F4FCE012F
:100CF0000296D6DEE114F10451F000E023EA32E876
:100D0000A701BE016F5F7F4FCE010296C9DE0F9033
:100D10000F90DF91CF911F910F91FF90EF90DF9097
:100D2000CF90BF90AF900895CF92DF92EF92FF9255
:100D30000F931F930E948730009122061091230683
:100D400020912406309125066B017C01C01AD10A3E
:100D5000E20AF30AF7FC13C02091210620952093A4
:100D60002106DC01CB018A549C4FAF4FBF4F8093CB
:100D7000220690932306A0932406B093250681E0D3
:100D800090912106911101C080E01F910F91FF9079
:100D9000EF90DF90CF900895CF9393E0909323024C
:100DA0008111109244060E948730DC01CB018C50E7
:100DB0009E4FAF4FBF4F80933E0690933F06A09348
:100DC0004006B093410668E873E182E090E00F943A
:100DD0008955C6E0C15049F00F94285562E070E093
:100DE00080E090E00E94B830F5CFCF910895AF92A7
:100DF000BF92CF92DF92EF920F931F93CF93DF9327
:100E000000D01F92CDB7DEB7809124028F3F09F446
:100E100044C00E9487300091270610912806209137
:100E2000290630912A06DC01CB01801B910BA20B15
:100E3000B30BB7FD32C09091840E8091870E8F5F07
:100E40008F70981751F1E091240284E0E802F001DC
:100E50001124EF58FC4F20E030E040E752E460817D
:100E60007181828193810F94665B69837A838B831E
:100E70009C83A12CB12C6501E12C8E010F5F1F4FCB
:100E80002AE732E046E752E062E772E08EE692E05F
:100E90000F9407098FEF809324020F900F900F900B
:100EA0000F90DF91CF911F910F91EF90DF90CF9036
:100EB000BF90AF9008950F931F930E9487300091C9
:100EC0003E0610913F062091400630914106DC011C
:100ED000CB01801B910BA20BB30BB7FD0FC0809110
:100EE000030185FB992790F981E0892790910301FF
:100EF00096FF8260629B84608093440680914406E2
:100F000081709091440691FD826090911506891739
:100F100041F18130A9F028F0823041F0833059F05E
:100F20001EC0913089F09230A9F019C0992361F068
:100F3000933081F014C0913069F0923081F404C094
:100F4000992341F0933059F4909139069F5F909323
:100F5000390605C0909139069150909339068093D7
:100F600015061F910F910895CF93DF930E94DD45E1
:100F7000E4E0F1E080818F7D8083C5E0D1E088816D
:100F800080958072A3E0B1E08C9380818F7B808319
:100F90008881809580748C936A98729A54985C9A30
:100FA00082E08093430687DF10923906DF91CF916C
:100FB0000895CF93C0918A0686E496E076DCC81740
:100FC00090F480918A068F5F21E0280FE82FF0E0EF
:100FD000EA5BF94F9081907C903811F4822FF4CF26
:100FE00080938A0602C010928A06CF9108950F93CB
:100FF0001F93CF93DF938C01C0918A06D0E0CA5B28
:10100000D94FCE0152DCF8018083CE01DF91CF9120
:101010001F910F91089581E090914606911101C0B2
:1010200080E00895CF93DF9320918906211120C09D
:10103000FC0101900020E9F73197EF01C81BD90BA3
:10104000C334D10534F031972081207C2038D9F386
:10105000F4CFBC01DD27AE0186E496E00F94066470
:10106000CA5BD94F188210928A0683E080932302CC
:10107000DF91CF910895CF93DF93CDB7DEB78E8107
:1010800090918906891790F0809389069E01275FC9
:101090003F4F4F81588562E470E086E496E00F94FC
:1010A0004F6410928A0683E080932302DF91CF91F0
:1010B00008950F931F93CF93DF938C0167FF03C0B5
:1010C0001092890660E08091890690E0262F062E16
:1010D000000C330B281739071CF160938906C801EF
:1010E0000F946863F801E80FF91FEF01C01BD10BE3
:1010F000C334D10534F031978491807C8038D9F3A2
:10110000F4CFDD27AE01B80186E496E00F94896341
:10111000CA5BD94F188210928A0683E0809323021B
:10112000DF91CF911F910F9108954F925F926F922F
:101130007F928F929F92AF92BF92CF92DF92EF9267
:10114000FF920F931F93CF930E9487306B017C0116
:101150004EDEB1DE8091440682FF15C080912006EC
:10116000811113C091E0909320062091ED17211179
:1011700003C08091D005892780932F061092ED1728
:1011800081E00ADE02C010922006C9B1C295C1708A
:1011900081E0C82780914306C81779F10E948B45EA
:1011A000882359F110914306C0934306CC2309F4D8
:1011B000B2C164EF71E080E090E00E94D6A50E9489
:1011C0000B95123009F0A2C10E94E2950E94DD4504
:1011D00083E0809323020E9487306B017C01DC0155
:1011E000CB018C599F4FAF4FBF4F80931C069093FC
:1011F0001D06A0931E06B0931F0680911C069091B9
:101200001D06A0911E06B0911F06A7019601281B7E
:10121000390B4A0B5B0B57FF05C080913D068823B5
:1012200009F433C2D701C6018C599F4FAF4FBF4F4E
:1012300080931C0690931D06A0931E06B0931F0674
:1012400060913906062E000C770B77FF03C071956D
:1012500061957109062E000C770B880B990B0F9482
:10126000015C2B013C0120E030E040E050E40F94B1
:10127000625D87FF05C080912F0681117DC08DC002
:1012800080913406882309F456C0809030069090EF
:101290003106A0903206B090330681149104A10467
:1012A000B104E1F120E030E040E05FE3C301B201CE
:1012B0000F949D5D2B013C01C701B60168197909A6
:1012C0008A099B090F94FF5B9B01AC01C301B2012A
:1012D0000F94665B20E030E04AE754E40F949D5D94
:1012E0004B015C0120E030E040EA52E40F94625D83
:1012F00087FF0FC020E030E040EF51E4C501B401AA
:101300000F94625D87FD0AC02AE030E040E050E0C3
:1013100009C024E630E040E050E004C021E030E0C5
:1013200040E050E0C0923006D0923106E0923206A2
:10133000F092330604C021E030E040E050E0A0919C
:10134000390600913A0610913B060A2E000CBB0BA1
:101350000F94085F22E030E040E050E00F94CB5E55
:10136000DA01C901800F911FA11DB11D90933B06A9
:1013700080933A0610923906D701C6018856954CDB
:10138000AF4FBF4F8093180690931906A0931A068B
:10139000B0931B0681E080932302209135063091A3
:1013A000360644E82B3A340741F48091250288231D
:1013B00009F4BCC08150809325022C5E334651F560
:1013C00080912502882321F081508093250222C03C
:1013D00084E080932502809138068F5F80933806E1
:1013E00090913706981728F4109238068CE0809375
:1013F000250281E080932302D701C6018856954CCF
:10140000AF4FBF4F8093180690931906A0931A060A
:10141000B0931B0680916F0081FB222720F981FF8A
:1014200005C080916F008D7F80936F008091950D36
:101430009091960DA091970DB091980D222329F0CF
:1014400020916F00226020936F003AE0B695A79537
:10145000979587953A95D1F7009721E0A207B105B6
:1014600020F08FEF9FEFA0E0B0E096958795209158
:101470002302211105C030913D06311102C139C04E
:10148000009739F0409116065091170648175907F2
:1014900080F580913D06811103C0223008F056C0CE
:1014A000C1E080913506909136068B5A944809F038
:1014B000C0E08C2F0E941742CC2309F453C04BDAB2
:1014C00010922F060E948730DC01CB018C199D09F8
:1014D000AE09BF09009116061091170620E030E012
:1014E000081719072A073B0720F4909317068093E3
:1014F000160680913506909136068B5A944809F469
:1015000083C08091420681117FC0AAC060E084E957
:1015100092E3CFDD5BCE18D6123009F457CE60E0EF
:1015200086E892E3C6DD0E944B8050CE8CE080932B
:101530002502809116069091170601979093170641
:101540008093160681E08093230237CF243030F059
:10155000243009F0A5CF10922302A2CF81E080931E
:1015600023029ECF80913D06811114C080914504D5
:10157000811107C081E0809345048CE094E00E94D3
:1015800052358CE094E00E94893581E080933C06DE
:1015900080933D0683E00E94704561E08CE094E01A
:1015A0000E94AB35E0913506F09136061995109200
:1015B0003C0680913D06882309F482CF8CE094E0BC
:1015C0000E948D3591E0811101C090E090933D061D
:1015D000992309F475CF0E948730DC01CB018C1967
:1015E0009D09AE09BF09C0901606D0901706E12CE0
:1015F000F12CC816D906EA06FB0608F046C09093FF
:1016000017068093160641C058E9C50E5AE3D51E49
:10161000E11CF11CC0921806D0921906E0921A063D
:10162000F0921B0680913D0681112FC0809123020C
:10163000813099F0833049F5CF911F910F91FF9040
:10164000EF90DF90CF90BF90AF909F908F907F9062
:101650006F905F904F900C940D461092230215C02E
:101660008091180690911906A0911A06B0911B0658
:10167000C81AD90AEA0AFB0AF7FCD4CF0E944B80A9
:10168000D1CF009709F40CCFFDCECF911F910F91D0
:10169000FF90EF90DF90CF90BF90AF909F908F9092
:1016A0007F906F905F904F90089561E002DD0C9401
:1016B0004B80CF93DF931F921F92CDB7DEB7898304
:1016C0009A8352DC89819A81F0DF0F900F90DF912D
:1016D000CF910C94E2458091200982FD05C0809154
:1016E000E217823061F410C08091D108811103C0EB
:1016F00083E199E002C081ED98E061E093CC813014
:1017000031F082E592E305C089E792E302C08DE6FD
:1017100092E36FEFCECC1092ED171092950280916C
:1017200020098064809320090E9433B50E94CCCDAB
:1017300060E084E492E3BDDC0C944B8088E392E3A8
:101740000E942F8160E08BE292E3B3DC40E061E035
:1017500080E00E94216881E292E30D943C44BBDF6B
:101760001092ED17109295020E948368882321F051
:101770008091200982FF04C00E942BB50C94AFCD4C
:101780008DE192E30F943C44F7CF8091200982FFD2
:101790002AC00E948368882319F18091DB0690910A
:1017A000DC06A091DD06B091DE060097A105B1052B
:1017B000B9F0BC01CD016D597F4F8F4F9F4F24E68B
:1017C00030E040E050E00F94A95E6091D706709140
:1017D000D8068091D9069091DA060F94A95E01C0CF
:1017E00020E020934506809145068F7708958BEA87
:1017F00094E89093360680933506089561E0FC01E5
:1018000080810E94B7328FEF0C94C8A6CF93DF93EC
:10181000EC018A810E948AA660E08881DF91CF91E5
:101820000C94B7328F929F92AF92BF92EF92FF9239
:101830000F931F93CF93DF93EC018B017A010E94EA
:1018400087304B015C012CE2820E21E0921EA11C2C
:10185000B11C0E94A2A68B838F3F61F40E94873047
:10186000DC01CB0188199909AA09BB09B7FDF1CFA1
:1018700081E10DC08E3F51F4B701C8010E94A9A6B5
:101880000E94A2A60E94A2A611E003C08FE0898355
:1018900010E0CE01B3DF812FDF91CF911F910F9127
:1018A000FF90EF90BF90AF909F908F900895CF9250
:1018B000DF92EF92FF926A017B010E948730C60E91
:1018C000D71EE81EF91E0E94A2A68F3F61F00E945B
:1018D0008730DC01CB018C199D09AE09BF09B7FD2A
:1018E000F2CF80E001C081E0FF90EF90DF90CF90D9
:1018F0000895EF92FF921F93CF93DF9300D01F9232
:10190000CDB7DEB77C01162F29833A834B835C83E6
:101910007DDF48E552E060E070E0C701C8DF812F5D
:1019200080640E94C8A68C810E94C8A68B810E94F8
:10193000C8A68A810E94C8A689810E94C8A61123D0
:1019400011F087E801C085E90E94C8A61C3011F497
:101950000E94A2A610E00E94A2A6F701838387FF3F
:1019600004C01F3F11F01F5FF6CF0F900F900F9034
:101970000F90DF91CF911F91FF90EF9008958F927C
:101980009F92AF92BF92CF92DF92EF92FF920F930E
:101990001F93CF93DF93EC01162F1C82198248838B
:1019A0000E9487306B017C0120EDC20E27E0D21E21
:1019B000E11CF11CA89561E088810E94B73261E0CA
:1019C00088810E947B320E949BA685E08A830E94C8
:1019D0008AA60AE08FEF0E94C8A60150D9F7A89501
:1019E00020E030E0A90160E0CE0183DF8B8381300D
:1019F00061F00E948730DC01CB018C199D09AE0992
:101A0000BF09B7FDEDCF81E055C0A8952AEA31E0C6
:101A100040E050E068E0CE016CDF853011F481E0F9
:101A200009C004E00E94A2A68B830150D9F78A3A2C
:101A300051F482E08C83A8958C81823081F0812CD6
:101A4000912C540111C00E948730DC01CB018C190C
:101A50009D09AE09BF09B7FDD9CF82E02BC0812C0B
:101A6000912CA12C80E4B82E20E030E0A90167E39E
:101A7000CE013FDFA501940169E2CE013ADF8B83FD
:101A8000882361F00E948730DC01CB018C199D090D
:101A9000AE09BF09B7FDE8CF8AE00CC08C81823067
:101AA000D1F420E030E0A9016AE3CE0122DF8823EF
:101AB00029F088E08983CE01A1DE16C00E94A2A68B
:101AC000807C803C11F483E08C830E94A2A60E945B
:101AD000A2A60E94A2A6CE0191DE173018F41A83A6
:101AE00081E003C088E1898380E0DF91CF911F917D
:101AF0000F91FF90EF90DF90CF90BF90AF909F90AD
:101B00008F9008950F931F93CF93DF93EC0189017A
:101B10008C81833039F089E0440F551F661F771F91
:101B20008A95D1F79A01AB0161E1CE01E2DE811124
:101B300009C040E052E0B801CE01DF91CF911F9182
:101B40000F9170CE84E08983CE0158DE80E0DF9172
:101B5000CF911F910F910895CF93DF93EC01862FC2
:101B6000BA010E94CDA68FEF0E94C8A68FEF0E94F7
:101B7000C8A60E94A2A68B83982F9F71953031F042
:101B800083E18983CE013ADE80E001C081E0DF910C
:101B9000CF9108950F931F93CF93DF93EC018901A9
:101BA0008C81833039F089E0440F551F661F771F01
:101BB0008A95D1F79A01AB0168E1CE019ADE8111D5
:101BC0001EC0A8016EEFCE01C7DF8823E1F048E513
:101BD00052E060E070E0CE016ADE882371F020E020
:101BE00030E0A9016DE0CE0184DE81110AC00E94BF
:101BF000A2A6811106C011E007C087E103C086E0FC
:101C000001C086E1898310E0CE01F8DD812FDF91EC
